:10000000F01F0010E1BA0000DDBA0000DDBA000008
:10001000DDBA0000DDBA0000DDBA0000000000001B
:10002000000000000000000000000000DDBA000039
:10003000DDBA000000000000DDBA0000A9B1000038
:10004000D1B10000D1B10000D1B10000D1B10000A8
:10005000D1B10000D1B10000D1B10000D1B1000098
:10006000D1B10000D1B10000D1B10000D1B1000088
:10007000D1B10000DBBA0000DBBA000061AF0000C4
:1000800091B1000079B1000061B1000049B10000F8
:10009000DBBA0000D9B00000DBBA0000DBBA000018
:1000A000DBBA0000DBBA0000DBBA0000DBBA0000FC
:1000B000DBBA0000DBBA0000DBBA0000DBBA0000EC
:1000C0000223184A10B5116801240B431360202342
:1000D000154A164811680B431360154B1968014007
:1000E0001960196821431960124B13491A680240BC
:1000F0001A601A6822431A606C22104B1A60104B67
:1001000018680BF02BFF80220E4B120218600E4B6A
:1001100018600E4B20001A6080234022DB051A6015
:1001200010BDC0460480044080800440F8FCFFFFFE
:100130003040044034400440400D030018000040AB
:1001400048040010140000401000004000E100E0EE
:10015000802208201021094BD20510B511601860CB
:100160000023074814680C4201D0834204D105489B
:1001700098428041404210BD0133F3E7180000402F
:10018000FF0F0000FE0F0000802100222020134BF3
:10019000C90510B55A609A60DA600860104958685D
:1001A000012807D08A4203D1FFF7D2FF002010BDFB
:1001B0000132F4E78A42F7D000211A69013A5868FF
:1001C000FF2801D95868F2E71869904202D01A69ED
:1001D00059690A3158698142F1D1E5E748040010B4
:1001E000FF0F0000F8B5060003250C4B0C4C1F78E0
:1001F0000223A222A361013BE361E318DA77013312
:10020000DE77084BDF77FFF7BFFF0223FF3398420B
:1002100002D0013D002DEBD1F8BDC0464CE70000F7
:10022000480400104B040010064A537BD318D873BF
:10023000537B0133DBB253735BB2002B01DA002333
:100240005373704748140010C143094A53699942D7
:1002500009D2591C08185169994200D27047516956
:100260008842FCD8F7E75169C91A8142FBD3F5E708
:10027000480400108022114B10B5DA679218DA6733
:100280008022D200DA6780225201DA6780221201CE
:10029000DA6780229200DA6700230121084A494286
:1002A0001360084A1160084A1360084A136001226B
:1002B000074B1A60FFF704FF10BDC04604E100E0E1
:1002C000048204400882044004C000403CC0004056
:1002D00000C000404023044A11680B431360012210
:1002E000024B30331A70704780800440480400107D
:1002F000084B70B530331B7804000D00002B01D182
:10030000FFF7E8FF182223689343236023681D4307
:10031000256070BD480400100E4B70B530331B785B
:1003200006000D001400002B01D1FFF7D3FF701E53
:1003300002280AD8084B8000C25801231168AB403C
:10034000012C04D10B43136070BD044AF5E79943B7
:100350001160F9E74804001050E70000FC3F00502E
:100360000F4B70B530331B7806000D001400002BC6
:1003700001D1FFF7AFFF701E02280BD8094B800098
:100380001818C26801231168AB40012C04D10B433B
:10039000136070BD044AF5E799431160F9E7C04660
:1003A0004804001050E700000080005010B50C4CCD
:1003B000606B002806D00220FFF714FF0238FF38D8
:1003C00043425841230038331A780A235106490F13
:1003D0004B430F210A4048349B186370E07110BDF5
:1003E00048040010F8B505000E000324A227094BAD
:1003F000B21C9A610022DA610133DF770133DD77C5
:10040000FFF7C2FE0223FF33984202D0013C002CCA
:10041000EDD1F8BD4804001010B50120FFF7E2FE51
:100420000223FF33984210D1094B01201A003832C1
:1004300014785863220706D0032203332240DA7768
:100440000100FFF7CFFF200010BD01246442FAE74E
:100450004804001070B50D4C636B002B13D0D5B25F
:10046000E31CDD77130A251DDBB2EB77130CDBB23F
:10047000651D120E0634EB77E277FFF7B3FF023803
:10048000FF3843424341180070BDC0464804001085
:1004900010B5FFF7C1FF0220FFF7A4FE0223FF33D0
:1004A000984220D1104B1A00383212787F2A15D981
:1004B0005A6B002A12D01A0000210820012422328F
:1004C0009070D47051701170142226330638D97090
:1004D00018705C709A700731FFF784FF034A04219B
:1004E0000920FFF7B7FF10BD48040010808080800E
:1004F000012210B510000B21FFF732FF00220B2163
:100500000120FFF709FF012202210320FFF728FF46
:10051000002202210320FFF7FFFE10BD70B5060088
:100520000024064D1835605D054B3100C0180134BC
:10053000FFF7DEFE0A2CF6D170BDC04650E7000082
:1005400000400440F8B500241020FFF7E7FF0B4DF2
:1005500022352B19665D5F78002239003000FFF7E5
:10056000FFFE0234012239003000FFF7D5FE142CC3
:10057000EFD10122024B5A65F8BDC04650E700009A
:1005800048040010F8B51B4C0600636D002B01D128
:10059000FFF7D8FF002E09D0012207210220FFF724
:1005A000DFFE002207210220FFF7B6FE23003033D2
:1005B0001B78002B01D1FFF78DFE0F4D01272B6813
:1005C0001B0509D530342378002B01D1FFF782FEBB
:1005D00001272B68DB0A9F43002E09D00022072148
:1005E0000220FFF7BDFE012207210220FFF794FE43
:1005F0003800F8BD48040010FC3F0050F0B5012061
:1006000089B0FFF7BFFF0123049300284FD10400F6
:100610001D0004902A4E630001330393330037001A
:100620002233E25C1B195B78019219002A000198C1
:100630000293FFF795FE002202990198FFF76CFEE6
:10064000204B343630333C37069607933B787E7820
:100650000593079B1B78002B01D1FFF73BFE059B01
:10066000032B0DD818000BF06FFC02252729164B21
:100670002A00B2401B6813405A1E9341002B02D13E
:100680006B461B7B0493039B023F01330393069B42
:100690009F42DBD1002202990198FFF761FE0234EC
:1006A0002A0002990198FFF737FE142CB2D1049862
:1006B00009B0F0BD054BDBE7054BD9E7054BD7E7A4
:1006C00050E7000048040010FC3F0050FC3F015080
:1006D000FC3F0250FC3F0350F8B54A0007000400FD
:1006E0001E48520D1518132D18DC002D09DACB0FFA
:1006F000DB070022691C01D119490B4319001000C6
:1007000017E0184E2E4132000A40144312D08022C6
:1007100012032A415318B3430022EFE7332D0BDDB8
:100720008023DB009D4205D13A000B0038000CF01D
:100730008BFA07003800F8BD01260B4876421218E4
:10074000D6403E42F6D03322551B323AAA40D21947
:10075000BA42A44164420B19B243CFE701FCFFFF48
:100760000000F03FFFFF0F00EDFBFFFF07B5002289
:1007700000280CD090231B06009201930098019949
:10078000802300225B050DF085F903B000BD8023B6
:100790005B05F1E707B5002200280CD0F0231B060B
:1007A0000092019300980199E0230022DB050DF0EF
:1007B00071F903B000BDE023DB05F1E7F0B5D34AE2
:1007C0004B0089B007000E000C005B0893423CD937
:1007D000CF4A934200D8F5E1CE4A93420DD90B039C
:1007E0001B0B034304D002000B000CF02DFA0EE0AB
:1007F00000290EDA0027C84E0BE0C84AC84B0BF0A0
:10080000C1FC002800D1DDE10020FFF7C3FF070095
:100810000E003800310009B0F0BDC24AC24B3800AA
:1008200031000CF011FA002200230BF097FC002895
:10083000E0D1BE4ABE4B380031000DF02BF9002C40
:1008400000DAA8E00024BB4DA7E0BB4A934200D8E1
:10085000C5E0BA4A9342ECD8B94ABA4B002900DA4B
:100860008FE00DF089FB012304000D000093B64AD0
:10087000B64B02920393029A039B200029000DF0CD
:100880007BFB02000B0007000E00200029000DF08A
:1008900073FB029A039B0DF06FFB02900391002201
:1008A000A44B380031000DF0F5F8049005910200DA
:1008B0000B00380031000DF0EDF804000D00A44AE3
:1008C000A44B0DF0E7F8A44AA44B0CF0BDF92200AC
:1008D0002B000DF0DFF8A24AA24B0DF04DFB2200D9
:1008E0002B000DF0D7F8A04AA04B0CF0ADF9220078
:1008F0002B000DF0CFF89E4A9E4B0DF03DFB2200E1
:100900002B000DF0C7F800229B4B0CF09DF9020064
:100910000B0006900791049805990DF0BBF80200B2
:100920000B00002095490DF027FB02000B000490FE
:100930000591069807990DF01FFB049A059B0690F8
:100940000791380031000DF0A5F802000B000020DF
:100950008B490DF011FB02000B00069807990CF073
:100960008FFC2B0022000DF095F8009B002B4CD142
:1009700002000B00380031000DF08CF822002B0033
:100980003AE00CF061F901235B42009304000D0092
:100990006D4A7C4B6DE700247B4D02000B0020006C
:1009A00029000CF051F90DF02FFE00900DF062FEC1
:1009B000634A644B029003910DF06CF802000B0047
:1009C000380031000DF0D8FA5F4A04000D0002989B
:1009D00003995E4B0DF05EF8029003914BE7002106
:1009E0006A4A0091934200D959E7694A694B31003C
:1009F0000CF02AF902000B000DF0BEFA02000B0009
:100A0000380031000DF0B8FA01E7029A039B0DF0AF
:100A1000B3FA3A0033000DF03DF8029A039B0DF053
:100A2000ABFA2B0022000DF0A7FA009B04000D008A
:100A300001330CD102000B00380031000DF09CFA9C
:100A400000223C4B0DF026F800223A4BDAE7009BDF
:100A5000012B26D10022504B380031000BF07EFBD9
:100A6000002811D00022334B380031000CF0ECF894
:100A700002000B00200029000DF07EFAC0230022A6
:100A80001B060DF007F8C2E622002B0038003100EB
:100A90000DF072FA02000B000CF0D6F80022364B73
:100AA000A3E6009B1B050293009B0133392B0FD952
:100AB0003A0033000DF060FA02000B0000202E49CE
:100AC0000DF05AFA029C0022631819002A4B99E78C
:100AD000009B132B62DC8023009A9B0313410020B0
:100AE000254AD11A009001913A00330020002900D4
:100AF0000DF042FA02000B00009801990DF03CFA4B
:100B0000029C070063181E0083E6C04679684340D4
:100B1000412E8640FFFFEF7F0000F0BFEF39FAFE65
:100B2000422E864059F3F8C21F6EA501FE822B6546
:100B30004715F73F0000E03F422ED63FB1A2F03FFD
:100B40000000E0FE422EE63F763C7935EF39EA3D83
:100B50002DC3096EB7FD8ABE3952E686CACFD03E94
:100B6000B7DBAA9E19CE143F8555FE19A0015A3F46
:100B7000F41011111111A13F0000F03F00000840D6
:100B800000001840EF39EABD0000E0BFFFFF8F3CD6
:100B90009C7500883CE4377E0000D0BF00980E4969
:100BA0000022091A0B05200029000CF04DF8020064
:100BB0000B00380031000DF0DFF90022074B0CF07C
:100BC00043F89DE7002C00DA27E6054A054B38007C
:100BD00031000CF05FFF35E6FF0300000000F03F3E
:100BE000FE822B654715F73FF0B54A005708914A3A
:100BF00089B005000C00CE0F97422DD98E4A97423E
:100C000011D90B031B0B034306D002000B00280075
:100C100021000CF019F810E0002E00D006E12800A9
:100C2000210009B0F0BD854A854B0BF0ABFA01906D
:100C3000002805D00020FFF7ADFD05000C00EEE711
:100C4000804A814B280021000BF088FA002807D049
:100C50000198FFF78BFDF0E77C4B9F4200D89BE0AB
:100C60007B497C4BF2008F426FD89F183A6C7B6CAB
:100C7000280021000DF080F93B6D7C6D012502906C
:100C80000391AD1B04930594AB1B0193049A059B40
:100C9000029803990DF070F905000C002A0023005A
:100CA000280021000CF0F6FE06000F006A4A6B4B8C
:100CB0000CF0F0FE6A4A6B4B0DF05EF932003B001F
:100CC0000CF0E8FE684A694B0BF0BEFF32003B00B7
:100CD0000CF0E0FE664A674B0DF04EF932003B0027
:100CE0000CF0D8FE644A654B0BF0AEFF32003B00BF
:100CF0000CF0D0FE02000B00280021000DF03CF9A2
:100D00000B00020006000F00280021000CF0C2FEBC
:100D1000019B06900791002B53D180230022DB0515
:100D2000300039000DF028F902000B0006980799F1
:100D30000CF0A6FA2A0023000DF01EF902000B00A9
:100D400000204F490DF018F977E79E1828004D4A0A
:100D50004D4B21000CF09EFE326E736E0BF074FF53
:100D60000DF052FC01900DF085FC484A484B0600FE
:100D70000F000CF08FFE02000B00280021000DF088
:100D8000FBF8444A02900391434B300039000CF0C9
:100D900081FE0490059179E7404B9F420CD8404A70
:100DA000404B0BF051FF0022354B0BF0EBF90028C4
:100DB00005D00022324B2AE7002301936EE7019011
:100DC0006CE7802132003B000020C9050DF0D4F80B
:100DD00002000B00069807990CF052FA02000B0073
:100DE000049805990DF0C8F8029A039B0DF0C4F819
:100DF00002000B00002022490DF0BEF82A4B019A98
:100E00009A4205DB019C0500260573181C0006E7C5
:100E1000FA25AD00AC46019C0022644426057318F7
:100E20001900B8235B040CF035FE06E700252C0002
:100E3000F5E6C046412E8640FFFFEF7FEF39FAFE10
:100E4000422E864051302DD5104987C0422ED63FC4
:100E5000B1A2F03F50E70000D0A4BE726937663EF1
:100E6000F16BD2C541BDBB3E2CDE25AF6A56113FAA
:100E700093BDBE166CC1663F3E5555555555C53F91
:100E80000000F03FFE822B654715F73F0000E0FEB3
:100E9000422EE63F763C7935EF39EA3DFFFFEF3DE4
:100EA0009C7500883CE4377E03FCFFFFF0B5BA4B2D
:100EB0008DB00E00994223DC4B005B08034307D141
:100EC000002200230020B5490CF0DAF90DB0F0BD86
:100ED000002906DA02000B000DF04EF80022002374
:100EE000F2E7AF4B00220CF0D5FD36230E005B423B
:100EF000AC4A964206DD02000B000BF0A5FEE5E7CA
:100F00000023F5E7A84C321512193603A74CD21866
:100F1000330B02931C1980235B032340A44C029DD6
:100F20005C401B159B18254300930022A04B290011
:100F30000DF022F8029B060002331B030F001B0B6F
:100F40000022022B64DC00230BF002F9002819D0E8
:100F5000009B002B00D11CE118000DF08BFB954A83
:100F6000954B04000D000CF095FD944A06000F000F
:100F7000934B200029000CF08DFD02000B00300087
:100F80003900BAE78F4A904B300039000CF082FDEF
:100F900002000B0000208D490CF0EEFF320004002F
:100FA0000D003B00300039000CF074FD0B00020016
:100FB000290020000CF06EFD009B02900391002B95
:100FC00006D102000B00300039000CF0D5FF7DE7A0
:100FD00000980DF04FFB774A774B04000D000CF0A2
:100FE00059FD764A00900191754B200029000CF0C4
:100FF00051FD02000B00029803990CF0BDFF320076
:101000003B000CF0B9FF02000B0000980199DCE7EF
:101010008023DB050BF018FE02000B0030003900C6
:101020000CF02EF90490059100980DF023FB049A22
:10103000059B06900791100019000CF02BFD644AE7
:10104000029B944663440B9302000B0008900991A5
:101050000CF020FD04000D005E4A5F4B0CF01AFD01
:101060005E4A5F4B0BF0F0FD22002B000CF012FDEE
:101070005C4A5D4B0BF0E8FD22002B000CF00AFDF2
:101080005A4A5B4B0BF0E0FD089A099B0CF002FDFD
:10109000584A08900991584B200029000CF0FAFC9E
:1010A000564A574B0BF0D0FD22002B000CF0F2FCFF
:1010B000544A554B0BF0C8FD22002B000CF0EAFC03
:1010C00002000B00089809990BF0BEFD029A4F4BE5
:1010D00004009B1A0B9A0D001343002B34DD0022F1
:1010E0003A4B300039000CF0D5FC32003B000CF0DC
:1010F000D1FC0290039102000B00200029000BF0AC
:10110000A3FD049A059B0CF0C5FC009B04000D0098
:10111000002B06D102000B00029803990CF02CFF63
:101120004FE7244A244B069807990CF0B3FC234A56
:101130000090019106980799214B0CF0ABFC22001E
:101140002B000BF081FD54E702000B00300039004A
:101150000CF012FF049A059B0CF09CFC009B040011
:101160000D00002B02D102000B002CE7114A124B9C
:10117000069807990CF08EFC104A00900191069891
:1011800007990F4B0CF086FC02000B002000290091
:1011900033E70020002199E6FFFF0F00000050C355
:1011A00000005043FFFFEF7F01FCFFFF645F090079
:1011B0000000F03F0000E0FE422EE63F763C79352D
:1011C000EF39EA3D555555555555D53F0000E03F9F
:1011D00086EBF9FF44523EDF12F1C23FDE03CB96AD
:1011E0006446C73F599322942449D23F935555559D
:1011F0005555E53F9FC678D0099AC33FAF788E1DFD
:10120000C571CC3F04FA97999999D93F51B8060016
:10121000434218434900C00F490801430348401A9C
:10122000414201430120C90F401A70470000F07F7E
:10123000564BF0B51A0085B005000C000A409A42E2
:101240000FD102000B000CF025FC02000B0028005F
:1012500021000BF0F9FC05000C002800210005B06E
:10126000F0BD0200002910DC4B005B080343F4D002
:101270000020814200D180E00B0028000CF07CFEB1
:1012800002000B000BF0FCFFE5E7081575D0404BA2
:101290000903C0188023090B5B031943C30703D557
:1012A000D30F4900C918520000244310490003938A
:1012B000D30FCB1880211625200052008903461831
:1012C0009E4202DC70189B1B6418D60F5B00013D28
:1012D0009B1952004908002DF1D1202680272900B2
:1012E00001963F067E19B446834202DC14D1964231
:1012F00012D865466646ED190290002E03DAEE43D9
:10130000F60F861902961B1A6245804140421B1A4D
:101310006046121A0298C919D60F5B00F318019E95
:101320005200013E7F080196002EDBD1134303D00B
:101330004B1C27D131000134164B6010C0184908EE
:10134000E30702D580231B061943039B0D001C05F0
:1013500023181C0081E7D10A153B52050029FAD059
:101360008024640321420AD020241600241AE64077
:10137000451E82403143581B89E70023EEE74900B0
:101380000130EFE7012301319943D5E70000F07FF9
:1013900001FCFFFF0000E03FF0B54F005E008DB0A4
:1013A0007F087608B74205DA3C00370026000400C3
:1013B00010002200330000920193F0223900040053
:1013C0003D00BB1B9204934206DD009A019B0BF08B
:1013D0003BFC04000D0017E0804B9F4200DCA1E0C5
:1013E0007F4B9F4214DD3F033F0B074305D0009A1C
:1013F000019B0BF029FC04000D007A4B5E40009B22
:101400001E4301D1009C019D200029000DB0F0BDBC
:10141000754BF618FF18009A019B33000092019358
:1014200096233D009B000893704B9E421BDC704B43
:101430009E4200DD78E0009B3343E5D0009801999F
:1014400000226C4B0CF026FB002200900191694BAE
:10145000200029000CF01EFB674A040094460D0092
:10146000089B63440893009A019B200029000CF01C
:1014700083FD0200099102900B00049100980199EC
:101480000AF06CFE002200285ED03B0010003900FC
:1014900016000CF0FFFA009B049005919C46009A00
:1014A000019B8020614600068446029101996144B7
:1014B0000391029803990CF0EDFA3200009001912B
:1014C0003B00200029000BF0BFFB3200029003918B
:1014D0003B00200029000CF04FFD02000B00029899
:1014E00003990CF0D7FA02000B00009801990CF058
:1014F00043FD02000B00049805990CF03DFDFFF739
:1015000097FE089B04000D00002B00D17CE7002013
:101510003A4A1B0599180B000200290020000CF024
:10152000B9FA56E700237EE79623354A9B05944691
:10153000FF18F618089B3D0063440893009A019B2E
:101540003300009201938EE73300802106920793C7
:10155000002249037B180698079916001F000CF01B
:1015600099FA0A900B918020000684460299049B08
:1015700004910999029A61440591049805990CF027
:1015800089FA2200029003912B00200029000BF021
:101590005BFB32003B000CF0EFFC009A019B0CF06F
:1015A00079FA069A079B04000D00009801990CF047
:1015B000E3FC32003B000CF06DFA02000B0020004F
:1015C00029000BF041FB02000B00029803990CF07C
:1015D000D3FC02000B000A980B998EE70000305FE5
:1015E000FFFFEF7F0000F07F000080DAFFFFAF20F9
:1015F000FFFF0F000000D07F02FCFFFF0000F03F64
:10160000A8FDFFFFF0B589B002920393464A4B0054
:1016100005000C005B08934203DC0CF0F5FF00288A
:101620004CD02A002300280021000CF033FA0600D9
:101630000F0002000B00280021000CF02BFA3B4A9F
:10164000009001913A4B300039000CF023FA394AEE
:10165000394B0CF091FC32003B000CF01BFA374A7E
:10166000374B0BF0F1FA32003B000CF013FA354A1D
:10167000354B0CF081FC32003B000CF00BFA334B85
:10168000334A0BF0E1FA0E9B04900591002B19D11F
:1016900002000B00300039000CF0FCF92D4A2E4BF3
:1016A0000CF06AFC009A019B0CF0F4F902000B00AC
:1016B000280021000BF0C8FA05000C0028002100CA
:1016C00009B0F0BD002202980399244B0CF0E2F916
:1016D000049A059B06900791009801990CF0DAF99D
:1016E00002000B00069807990CF046FC32003B0004
:1016F0000CF0D0F9029A039B0CF03EFC154A060050
:101700000F0000980199144B0CF0C4F902000B0073
:10171000300039000BF098FA02000B00280021007D
:101720000CF02AFCC8E7C046FFFF3F3E7CD5CF5AED
:101730003AD9E53DEB9C2B8AE6E55A3E7DFEB15752
:10174000E31DC73ED561C119A0012A3F1111813F98
:10175000A6F81011495555555555C53F0000E03FB5
:10176000F8B50022324B0CF095F900220023060058
:101770000F000AF0EDFC002854D100222D4B300060
:1017800039000AF0E5FC00284FD132003B00300060
:1017900039000CF07FF904000D00274A274B0CF0AC
:1017A00079F9274A274B0CF0E7FB22002B000CF0BD
:1017B00071F9254A254B0BF047FA22002B000CF05B
:1017C00069F9234A234B0CF0D7FB22002B000CF0C5
:1017D00061F9214A214B0BF037FA22002B000CF063
:1017E00059F91F4A1F4B0CF0C7FB22002B000CF0CD
:1017F00051F91D4A1D4B0BF027FA22002B000CF06B
:1018000049F91B4A1B4B0CF0B7FB22002B000CF0D4
:1018100041F9194A194B0BF017FA32003B000CF052
:1018200039F9F8BD00200021FBE700201449F8E752
:101830000000E03F0000D03F98456D69B8D1B93F46
:10184000722CC67097F7E63FA79ED5E9358F0E40FC
:101850000CD7D1DD74302E40CB90514883074540E2
:10186000437562CE2C2D53406EAA7567BC665440FA
:1018700052BE25E6BCAB4440182D4454FB21194010
:101880000000F03FF8B505000C00FFF7C1FC002890
:1018900000D0E3E000220023280021000AF05EFCD3
:1018A00000280BD0280080252D066119FFF7EAFFDC
:1018B0004919002200230BF0C7F9F8BD00220023CC
:1018C000280021000AF044FC061E02D0002001007E
:1018D000EFE70022644B280021000AF039FC0028C1
:1018E00000D0BEE00022614B280021000AF030FC4D
:1018F0000028EBD15E4A60002300400890420BDDD7
:101900002A00280021000BF09FF902000B000BF0C9
:10191000B7FC05000C000FE08027E20F2900D2077A
:10192000FF05B84215DC07D1002D12D1D20FD3002C
:10193000504AD218156F546F00224B4B28002100DB
:101940000AF016FC002857D028002100FFF708FFF6
:10195000AFE780241B031B0B64031C43464B00159D
:10196000C018464BE318002816D1002B00DA2300DC
:101970001C0001200C43D9D0414CA3421ADD414C3C
:10198000A0421DDB3D4C0D001B191A433E4BC018F5
:10199000000502431400CFE7002B05DA6400CB0FEB
:1019A0001C1949000138DCE71C000C43BED05B0069
:1019B000CC0FF5E7CD0F5B005B1949000138DCE780
:1019C000241A142C0ADC314DE14040191D008540D9
:1019D00023410D431A43110028009AE71F2C07DC0E
:1019E000E1402A4C001983400B431D001300F1E72E
:1019F0002749081A0341F8E700221C4B2800210060
:101A00000AF0B6FB002806D02A0023000020174960
:101A10000CF0B2FA9AE700221E4B280021000AF0CF
:101A2000A7FB002200280AD0280021000F4B0CF051
:101A3000A3FAFFF795FE80231B06C91839E7802318
:101A40002800DB0521000AF093FB002800D13DE7C8
:101A500080212A0023000020C905E8E700200E4964
:101A600027E73000014924E70000E03F0000F03F95
:101A7000FFFFEF7F50E7000000FCFFFF0000F0FFDA
:101A8000FFFF0F0002FCFFFFFF0300001E04000029
:101A9000E2FBFFFF0000F83F0000F87FF0B587B0E1
:101AA000049205934B005B080093009A484B050095
:101AB0000C009A4204DC0CF0A7FD002800D184E061
:101AC0002A002300280021000BF0E4FF0022414BF4
:101AD00006000F000BF0DEFF3F4A029003913F4BE0
:101AE000300039000BF0D6FF3D4A3E4B0BF0ACF80E
:101AF00032003B000BF0CEFF3B4A3C4B0CF03CFA73
:101B000032003B000BF0C6FF394A3A4B0BF09CF811
:101B100032003B000BF0BEFF374A384B0CF02CFA7A
:101B200032003B000BF0B6FF354A364B0BF08CF819
:101B300032003B000BF0AEFF32003B000BF0AAFF7F
:101B4000049A059B06000F00280021000BF0A2FF5D
:101B500002000B00300039000CF00EFA2A4B009AFC
:101B600004000D009A420DDC02000B00029803995C
:101B70000CF002FA020000200B0024490CF0FCF9E2
:101B800007B0F0BD224B009A00269A421BDC1300DE
:101B9000204A944663441F0032003B0000201B494A
:101BA0000CF0EAF9320000900191029803993B0091
:101BB0000CF0E2F922002B000CF0DEF902000B0021
:101BC00000980199DAE7144FE6E700200F49D7E7BC
:101BD000FFFF3F3E0000E03FD43888BEE9FAA8BDD1
:101BE000C4B1B4BD9EEE213EAD529C804F7E923E6C
:101BF0009015CB19A001FA3E7751C1166CC1563F22
:101C00004C5555555555A53F3233D33F0000F03F55
:101C10000000E93F0000E0FF0000D23F70B5140073
:101C20004A000B00520D0DD14B005B0803430FD04F
:101C3000224B00220BF02EFF214B9C4209DA214A55
:101C4000214B17E0214DAA4207D102000AF0FCFF08
:101C500070BD0B004A00520D363A1D4DAC420CDDF2
:101C6000C90F1C48C907084303001B4A190010008C
:101C7000184B194A0BF00EFFEAE7A218174CA242C4
:101C8000EEDC002A05DD164C120523401343190033
:101C9000DEE71400353408DAC90F0B48C9070843DA
:101CA0000300084A19001000C9E70D4C36322340E2
:101CB00012051A4311000B4B0022DBE700005043D2
:101CC000B03CFFFF59F3F8C21F6EA501FF070000EB
:101CD00050C300003CE4377E9C750088FE0700007E
:101CE000FFFF0F800000903CF0B54B00394A5B0DC0
:101CF00085B09E180D0004000390132E33DC002ED7
:101D000014DA354A354B0AF09FFF002200230AF00F
:101D100039FA002807D0002D58DA6B005B081C4305
:101D200001D000242E4D2000290026E02D4F374100
:101D30003B000B40034320D000900191264A274BE3
:101D4000009801990AF080FF002200230AF01AFA95
:101D50000028E8D0002D03DA80235B033341ED181F
:101D6000BD430024DFE7332E09DD8023DB009E42E4
:101D700003D102000B000AF067FF05B0F0BD012798
:101D8000194A7F429B18DF403842F6D000900191FB
:101D9000114A124B009801990AF056FF00220023C5
:101DA0000AF0F0F90028BED0002D02DA142E02D17C
:101DB0000135BC43B7E734239E1B333BB340E418E3
:101DC000039B9C429B415B42ED18F2E700242500F7
:101DD000A9E7C04601FCFFFF9C7500883CE4377E04
:101DE0000000F0BFFFFF0F00EDFBFFFFF0B5D14C8F
:101DF000A54408900991D01E1821140002930AF0FE
:101E0000ADF81823421C5B4253431B190024009376
:101E1000029B05905D1EDF1C451BC74BAE00F618EC
:101E2000EC4200D5F1E0A300F0580CF023FCE300F5
:101E300022AAD318013418605960A742F0DA0024AE
:101E4000029BDB00D3180793079B00261D19002374
:101E500000270693069B089ADB00E91A0839D31875
:101E60001A685B68086849680BF014FE02000B00F2
:101E7000300039000AF0E8FE069B060001330693A5
:101E8000069A029B0F009342E4D172AB1B190834EF
:101E90001E605F60282CD7D10426059BA64A9B00B4
:101EA0009B180A93370072AAF300D3181C685D6868
:101EB0000EA9B3005B1805930B9200229F4B2000E4
:101EC00029000BF0E7FD0CF09FFB0CF0D3FBBB00EF
:101ED0005B42079300229A4B029003910BF0DAFDCC
:101EE00002000B00200029000CF046F80CF08CFBDF
:101EF000059B079A013F98500B9AFB00D3181A686C
:101F00005B68029803990AF09FFE04000D00002F01
:101F1000D3D1009AFFF782FEFF2300229B05040025
:101F20000D000BF0B7FDFFF7DFFE0022854B0BF035
:101F3000B1FD02000B00200029000CF01DF80D007F
:101F400004000CF061FB07900CF094FB0B00020006
:101F5000290020000CF010F8009B04000D00002B5D
:101F600056DD721E92000EAB9B5818211F00009880
:101F7000091A0F410798C0198F40DF1B0EAB9F5005
:101F80001723009A07909B1A1F410597059B002B6A
:101F90004FDD079B00270133079380235B043A0042
:101FA0009C4691000EABCB58002F00D0A5E0002B33
:101FB00004D06746FB1A0EAFCB510127013296427F
:101FC000EFD1009B002B05DD012B00D19AE0022B05
:101FD00000D1A1E0059B022B2BD122002B00002079
:101FE00059490BF0C9FF04000D00002F21D0009AC1
:101FF00000205549FFF712FE02000B0020002900C7
:102000000BF0BAFF04000D0013E0002000210EE7E2
:10201000009B002B06D1731E9B000EAAD758FB1500
:102020000593B3E70022494B0AF0B6F8002861D1C6
:10203000059700220023200029000AF089F80028D3
:1020400000D1E0E00022731E0293013B022B00D07E
:102050006AE0002A00D19BE0009B0EAA183B009387
:10206000029B9B009B58002B00D1C8E0009A0020E7
:102070003549FFF7D3FD06000F00029C002C00DB62
:10208000FCE00025029B324FDC0072AB1C19029B66
:102090005B1B00D40AE100263500029C002C00DB0B
:1020A00029E1059B2900002B02D080231B06E9189B
:1020B0000B003200099901240A604B604A984B9941
:1020C0002B000BF059FF029BA34200DB20E1059B94
:1020D000002B02D080231B06C91802000B0007202A
:1020E00009998A60CB60079B034018009B239B00E3
:1020F0009D44F0BD022305934BE71648C31A0EA872
:102100000B505BE7721E92000EAB9B5802935B0272
:102110005B0A0EA98B505DE7721E92000EAB9B58B6
:1021200002939B029B0AF4E799000EA809184968DC
:102130000A438AE794FDFFFF78F000000000703E3C
:1021400000007041000020400000F03F0000E03F30
:10215000D0E70000FFFFFF0001339A008A1A1269DE
:10216000002AF9D0721C0292069A00249219D20019
:102170000792079922AA8C4662440C92F318F20047
:102180000D920593029B059A934204DD160089E6A1
:1021900001230EA9E1E7079B0A9A1D1922AB5D19DD
:1021A000029B00269B00D0580CF064FA00272860A0
:1021B000696000250C9B1B190B93089AEB00D11842
:1021C0000B9A08684968D31A1A685B680BF062FCBE
:1021D0000B000200390030000AF036FD069B013585
:1021E00006000F00AB42E8D10D9B72AA1B19D31851
:1021F0009E60DF60029B083401330293C2E7029BBA
:10220000013B029328E7009B20005A422900FFF778
:1022100005FD0022434B04000D0009F0BDFF00281E
:1022200023D00022404B200029000BF033FC0CF09F
:10223000EBF907000CF01EFA00223A4B0BF02AFCD7
:1022400002000B00200029000BF096FE0CF0DCF9D8
:102250000EABB200D050731C0293009B0EAA183331
:102260000093029B9B009F5000E7200029000CF088
:10227000CBF9B7000EABF8500296F7E6E50072AB6B
:102280000EAA5D19A30098580CF0F4F932003B0037
:102290000BF000FC002228606960234B30003900FD
:1022A0000BF0F8FB013C06000F00E7E600220023DC
:1022B000002600920193B54213DBF300F918E318EE
:1022C0001A685B68086849680BF0E4FB02000B00C1
:1022D000009801990AF0B8FC013600900191052E92
:1022E000E9D1EB004AAAD31801350099019A083CBC
:1022F00019605A60CBE6E3004AAAD31830001A6886
:102300005B6829000AF0A0FC013C06000D00C5E650
:10231000E3004AAAD3181A685B680AF095FC0134F6
:10232000D1E6C046000070410000703E49004B08F5
:1023300019007047F7B54B005B080193019A3F4BBA
:102340009A4204DD02000B000BF0A4FB2BE03C4B97
:10235000019A9A422DDCFFF7E9FFFEF72FFA0022DF
:10236000384B06000F000AF06FFC374B019A04004F
:102370000D009A4219DD32003B00300039000BF0AD
:1023800089FB220006000F002B00200029000AF024
:102390005BFC02000B00300039000AF071FF0022E4
:1023A000284B0AF051FC04000D002000290003B066
:1023B000F0BD264B019A9A4216DCFFF7B7FFFEF7F5
:1023C00013FC0022224B04000D000BF063FB2200E3
:1023D00006000F002B0000201D490AF051FF0200EB
:1023E0000B0030003900DCE71A4B019A9A4206DCF8
:1023F000FFF79CFFFEF7F8FB0022154BA4E7164BF6
:10240000019A9A4205DD154B9A4213D1144A904223
:1024100010D8FFF78BFF00220D4B0BF03BFBFEF7B4
:10242000E3FB04000D000022094B0BF033FB2200FC
:102430002B0089E70020FEF7ADF9B4E7FFFFEF7F3F
:10244000422ED63F0000F03FFFFF7F3CFFFF3540AC
:102450000000E03F412E8640CD338640CE3386409B
:102460007DF8B98FF0B54C4A4E0085B005000C00E0
:102470000B007608964208DD02000AF0E5FB050035
:102480000C002800210005B0F0BD0022002944DA2C
:10249000424B00920193424B9E424FDC414B9E4285
:1024A0000BDC414A414B280021000AF0CDFB002201
:1024B0003F4B09F067FE0028E3D128002100FFF719
:1024C00035FFFEF77BF93B4B04000D009E4226DCF6
:1024D00002000B000AF0B8FB2200029003912B00CF
:1024E000200029000BF0D6FA002206000F00304B26
:1024F000200029000AF0A8FB02000B003000390080
:102500000AF0BEFE02000B00029803990BF034FDA6
:10251000009A019B0BF0BEFAB1E7274BB9E7002206
:10252000234B0AF091FB02000B00200029000AF067
:10253000A7FE22002B000AF087FBE9E71F4B9E4213
:1025400006DC28002100FFF7F1FEFEF74DFBDFE778
:102550001B4B9E4205DD1B4B9E4217D11A4A9542EA
:1025600014D828002100FFF7E1FE0022124B0BF0E7
:1025700091FAFEF739FB04000D0002000B000098F1
:1025800001990BF087FA22002B00C3E7064A074B9C
:1025900028002100BEE7C046FFFFEF7F0000E0BF3C
:1025A000FFFF3540FFFF2F3E3374AC3C1F7BAC7FF9
:1025B0000000F03FFFFFEF3F0000E03F412E86406C
:1025C000CD338640CE3386407DF8B98FF7B51700FE
:1025D0001E0004000D00FFF7A9FE00221B4B09F0AE
:1025E000C7FD00280CD020002900FFF7A3FE3860AB
:1025F000796020002900FFF735FF30607160F7BD7A
:1026000020002900FEF7F0FA04000D0002000B0084
:1026100000200E490AF034FE0022009001910B4B7D
:10262000200029000BF036FA009A019B04000D00EF
:102630000BF0A2FC220030607160009801992B0021
:102640000AF002FB38607960D9E7C0460000E03F3D
:1026500082B0F0B58BB001901092119300221298C5
:102660001399002309F074FD0022002300283ED0B6
:102670001098119909F06CFD00280CD0129813994C
:10268000002200230BF006FA002200230AF0DCFAF5
:10269000129C139D19E010981199FFF747FEFEF761
:1026A000C7FD0022002304000D001098119909F0C5
:1026B00055FD00220023002812D0200029000BF035
:1026C000E9F9002200230AF0BFFA019B1860596063
:1026D0009C60DD6001980BB0F0BC08BC02B01847EC
:1026E000129813990BF0D6F922002B00CEE7109820
:1026F000119909F02DFD002830D012981399FFF799
:1027000015FE0022764B0BF0C5F9FEF791FD002275
:10271000002305000C000BF0BDF9002206000F009D
:1027200012981399002309F02DFD32003B00002878
:1027300004D0280021000AF087FA06E028002100D2
:102740000BF01AFC80231B06E418019B2A0018607A
:102750005960230001998A60CB60BBE710981199FA
:10276000FFF7E4FD00225F4B09F00CFD00280AD1C1
:1027700012981399FFF7DAFD00225A4B09F002FD77
:10278000002800D175E0109811990022564B0BF0EB
:1027900081F90022544B04000D00129813990BF09C
:1027A00079F98023002202900391DB0504920593BE
:1027B00002980399002200230BF06CF922002B00F1
:1027C0000AF042FA029A039BFEF7E6FD0022444B10
:1027D0000BF060F9002206900791414B2000290080
:1027E0000BF058F9002206000F00029803993C4BA9
:1027F0000BF050F9002208900991002320002900D5
:1028000009F0C0FC32003B00002846D0069807992A
:102810000AF01AFAFEF70CFD02000B0006000F008A
:10282000089809990AF02CFDFFF780FD049A059B92
:102830000BF030F932003B0005000C0004980599BC
:102840000BF028F906000F000022002328002100C9
:102850000BF020F9002204900591029803990023BF
:1028600009F07CFC049A059B002835D03000390023
:1028700066E70022109811991C4B0BF00BF900220F
:102880001A4B04000D00129813990BF003F9F92369
:102890000290039100229B0588E7069807990BF0A8
:1028A0006BFBFEF7C5FC02000B0004000D0008984E
:1028B00009990AF0E5FCFFF739FD049A059B0BF036
:1028C000E9F822002B0006000F00049805990BF090
:1028D000E1F805000C00B7E7300039002BE7C046EF
:1028E0000000E03F000010400000D03F00005043D7
:1028F000F0B593B002920393039B0E0002995D0022
:1029000004930B006D0807002B4319D180210903A4
:10291000714002000B0092185B419B498B4206D824
:1029200001D000F0C7FC002A01D100F0C3FC029ADC
:10293000039B380031000AF087F9009001917CE098
:10294000924B74000896009064089C469C4207DCF9
:1029500001D1002804D1654502DC0CD100290AD040
:102960008B4BF3183B43E2D1802103980903484085
:10297000029A0300CFE700230693002E17DA854A58
:1029800095424BDC844A954211DD844B2A15D218BE
:10299000142A23DD3420821A0298D0400300934089
:1029A0008B4204D1012210409218131A0693002979
:1029B0005ED1654521D1764BE3181F4301D100F06C
:1029C00079FC754B9C422BDD049B002B01DA00F057
:1029D00075FC029B039C009301942EE0002947D1D3
:1029E00014239A1A2B00134119009140A94204D1D3
:1029F000012213409218D31A0693694B9D4220D1AD
:102A000038003100049B00900191002B15DA3A0048
:102A10003300002062490AF033FC8EE70223C5E749
:102A2000049B002B01DB00F049FC80221206944637
:102A3000029B0093039B634401930098019913B098
:102A4000F0BD8023049ADB059A4206D13A00330098
:102A5000380031000BF01EF86FE7524B049A9A428F
:102A600006D1002E04DB38003100FEF7E1FB64E7FD
:102A700038003100FFF75AFC00900191002F2ED151
:102A8000002C04D0464AB3009B08934227D1049BF4
:102A9000002B07DA009A019B002041490AF0F0FB65
:102AA00000900191089B002BC7DA394BE418069B74
:102AB0001C4308D1009A019B100019000BF05CFA2E
:102AC00002000B00A7E7069B012BB6D100988021DE
:102AD000020001980906431800920193ADE7F20F36
:102AE000069B013A134304D13A0033003800310009
:102AF000E4E7069B013B13430022002B14D0284B34
:102B0000069207938423DB059D4200DC0AE1264BF5
:102B10009D4212DD204B9C4208DC049B002B08DA0E
:102B20000020FDF737FE08E7204BE9E7049B002B68
:102B3000F6DC0020FDF71AFEFFE61D4B9C420FDC81
:102B4000069807990023002209F008FB431E9841CC
:102B500001244042049B04402000002BEADAE0E715
:102B60000F4B9C4226DD069807990023002209F0AE
:102B7000F5FA431E984101244042049B0440200082
:102B8000002BCEDCD6E7C0460000F0FF0000F07F4F
:102B9000000010C0FFFF3F43FFFFEF3F01FCFFFFBE
:102BA0000000F03F0000E03F0000F0430000F0BFF5
:102BB000FEFFEF3F0098019900224F4B0BF0DCF92C
:102BC000C0224E4BD20506000F000AF063FF4C4AAC
:102BD000049005914B4B300039000AF05BFF002256
:102BE00000900191484B300039000AF053FF020079
:102BF0000B00464846490BF0BFF932003B000AF093
:102C000049FF02000B00002042490BF0B5F93200E9
:102C100004000D003B00300039000AF03BFF0200C9
:102C20000B00200029000AF035FF3B4A334B0AF025
:102C300031FF02000B00009801990BF09DF9020092
:102C40000B0004000D000498059909F0FDFF049A9B
:102C5000059B0020009001910BF08EF902000B0003
:102C6000200029000BF088F9029C039D0024060037
:102C70000F000298039922002B000BF07DF9009AB7
:102C8000019B0AF007FF029A039B04900591300014
:102C900039000AF0FFFE02000B000498059909F0C4
:102CA000D3FF22002B0002900391009801990AF0B3
:102CB000F1FE06000F000B00020002980399049633
:102CC000059709F0C1FF154B05000C0008919942CA
:102CD00000DCCAE2124BCB18034300D1CCE10698CA
:102CE00007990023002209F039FA431E9841012474
:102CF00040420440200014E70000F03F4715F73F32
:102D000044DF5DF80BAE543E0000D03F555555559D
:102D10005555D53F0000E03FFE822B65FFFF8F40F9
:102D2000000070BFBB4B00229C420ADC0098019956
:102D30000022B94B0AF0AEFE352200900191019CB1
:102D40005242B64923155B189B182403B44DB54A6B
:102D50000E93230B1D430024934209DDB24A013434
:102D6000934205DD0E9B1B1900240E93AF4BED180B
:102D7000009801992900AE4AE300D3180F931A6C0A
:102D80005B6C0C900D910A920B930BF0F5F80C9A7A
:102D90000D9B06000F000A980B9909F055FF0200E1
:102DA0000B0000209E490AF06BFA1090119102006E
:102DB0000B00300039000AF06DFE08900991089A66
:102DC000099B802104920593002389056D100D4312
:102DD00080210493049A059B009201930022090329
:102DE0006D18A4042B190098019914001D000AF015
:102DF00051FE02000B00300039000BF0BDF80A9ABA
:102E00000B9B06000F00200029000BF0B5F8020014
:102E10000B000C980D990BF0AFF8009A019B0AF08B
:102E200039FE02000B00300039000BF0A5F8109AB3
:102E3000119B0AF02FFE089A099B0A900B91100033
:102E400019000AF027FE06000F007A4A7A4B0AF0B2
:102E500021FE7A4A7A4B09F0F7FE32003B000AF075
:102E600019FE784A784B09F0EFFE32003B000AF079
:102E700011FE764A764B09F0E7FE32003B000AF07D
:102E800009FE744A744B09F0DFFE32003B000AF081
:102E900001FE724A724B09F0D7FE320004000D00A9
:102EA0003B00300039000AF0F5FD02000B00200065
:102EB00029000AF0EFFD009A019B04000D0008981C
:102EC000099909F0C1FE0A9A0B9B0AF0E3FD220062
:102ED0002B0009F0B9FE009A019B0C900D91100097
:102EE00019000AF0D7FD00225E4B04000D0009F026
:102EF000ABFE0C9A0D9B09F0A7FE049E0F0032005A
:102F00000B00009801990AF0C5FD00220090019184
:102F1000544B300039000BF02FF822002B000BF03F
:102F20002BF802000B000C980D990BF025F8089A6D
:102F3000099B0AF0AFFD320004000D000A980B99BE
:102F40003B000AF0A7FD02000B002000290009F059
:102F50007BFE04000D0002000B000098019909F0AF
:102F600073FEE022049E12063F4B30000F000AF071
:102F700091FD08900991009A019B300039000AF0F8
:102F8000FBFF02000B00200029000AF0F5FF374A82
:102F9000354B0AF07FFD364A04000D00354B3000FA
:102FA00039000AF077FD02000B002000290009F02B
:102FB0004BFE0F9B1A6D5B6D09F046FE0A900B915C
:102FC0000E980BF057FB04000D00089809990F9B11
:102FD0001E6E5F6E0A9A0B9B09F036FE32003B00B4
:102FE00009F032FE22002B0009F02EFE0498220088
:102FF0002B00009001910AF0BFFF32003B000AF065
:10300000BBFF089A099B0AF0B7FF02000B000A9861
:103010000B9927E6FFFF0F000000404301FCFFFF74
:103020000000F03F8E98030079B60B000000F0FF1F
:10303000D0E70000EF4E454A287ECA3F65DBC993C2
:103040004A86CD3F01411DA96074D13F4D268F5165
:103050005555D53FFFAB6FDBB66DDB3F03333333E5
:103060003333E33F0000084009C7EE3FFD033ADC7D
:10307000F5015B14E02F3EBE924A934B02980399F0
:1030800009F0E2FD3200009001913B002800210090
:103090000AF072FF02000B000098019909F072F823
:1030A000002800D01BE60021884A63005B080091DD
:1030B000934225DD864A1B159B18802252039446B5
:1030C0001A4114196000834B400D834DC01805410F
:1030D0002100A9430B0061462403240B214314243F
:1030E000201A0141009108990022002902DA009972
:1030F00049420091300039000AF03EFF04900591EA
:10310000029A039B04980599002609F09DFD002270
:10311000724B30000F000AF0BDFC049A059B08902A
:103120000991300039000AF027FF02000B000298D5
:1031300003990AF021FF6A4A6A4B0AF0ABFC6A4A1B
:1031400004000D00694B300039000AF0A3FC0200B6
:103150000B002000290009F077FD04000D0002009B
:103160000B000898099909F06FFD089A099B060061
:103170000F000AF001FF02000B00200029000AF0F6
:10318000FBFE3200029003913B00300039000AF050
:1031900081FC04000D00564A564B0AF07BFC564A4F
:1031A000564B0AF0E9FE22002B000AF073FC544A49
:1031B000544B09F049FD22002B000AF06BFC524AE7
:1031C000524B0AF0D9FE22002B000AF063FC504A51
:1031D000504B09F039FD22002B000AF05BFC020085
:1031E0000B00300039000AF0C7FE04000D00020099
:1031F0000B00300039000AF04DFC8023049005914B
:103200000022DB05200029000AF0B6FE02000B00B8
:10321000049805990AF034F8029A039B04000D0003
:10322000300039000AF036FC029A039B09F00CFDCD
:1032300002000B00200029000AF09EFE32003B0035
:103240000AF09AFE02000B00002033490AF094FEB7
:10325000009B1B055B181A15002A29DC009AFEF753
:10326000DDFC069A079BFFF7F5FB2C4A4B005B0839
:10327000934200DC17E72A4BCB1803430CD0069887
:1032800007990023002208F069FF431E984101249A
:103290004042044020004DE432003B000AF06CFE46
:1032A000029A039B08F078FF002800D1FBE6E6E7CE
:1032B0001900D6E70023184CFFF78DFB00230024EC
:1032C000FFF789FBFE822B654715973C0000E03F26
:1032D00002FCFFFF01FCFFFFFFFF0F00432EE63F54
:1032E000EF39FAFE422EE63F396CA80C615C20BE35
:1032F000D0A4BE726937663EF16BD2C541BDBB3EFC
:103300002CDE25AF6A56113F93BDBE166CC1663FD9
:103310003E5555555555C53F0000F03FFFCB9040F9
:1033200000346F3FF0B5984B85B04E0004000D009F
:10333000039176089E4218DD944B9E4202DC0AD12E
:10334000002808D022002B002000290009F07CFC76
:1033500004000D0005E0039B8D4C002B00DC10E108
:103360008C4D2000290005B0F0BD8B4B9E420FDC38
:103370008A4B9E4209DC8A4A8A4B09F065FC00228E
:10338000894B08F0FFFE0028EBD101235B4225E0CA
:10339000FEF7CCFF854B04000D009E4200DDAAE045
:1033A000834B9E4200DD90E002000B0009F04CFCD4
:1033B00000227D4B0AF0E0FD802306000F00002272
:1033C000DB052000290009F03FFC0B00020039005A
:1033D000300009F055FF002304000D000293220085
:1033E0002B00200029000AF055FB02000B00009082
:1033F00001910AF04FFB06000F006E4A6E4B0AF077
:1034000049FB6E4A6E4B09F01FFC32003B000AF08C
:1034100041FB6C4A6C4B09F017FC32003B000AF090
:1034200039FB6A4A6A4B09F00FFC32003B000AF094
:1034300031FB684A684B09F007FC32003B000AF098
:1034400029FB664A664B09F0FFFB009A019B0AF0D4
:1034500021FB644A00900191634B300039000AF06F
:1034600019FB624A624B0AF087FD32003B000AF00A
:1034700011FB604A604B0AF07FFD32003B000AF00E
:1034800009FB5E4A5E4B0AF077FD32003B000AF012
:1034900001FB5C4A5C4B0AF06FFD32003B000AF016
:1034A000F9FA02000B000098019909F0CDFB2B00FE
:1034B00022000AF0EFFA029B013343D102000B0015
:1034C000200029000AF058FD42E70022364B0AF09E
:1034D00053FD002206000F00334B2000290009F0A5
:1034E000B3FB0B0002003900300009F0C9FE0123D4
:1034F00004000D0072E7454B9E4219DC0022444B4C
:103500000AF03AFD002206000F00414B200029007E
:103510000AF0C0FA0022244B09F096FB0B000200CF
:103520003900300009F0ACFE022304000D0055E71D
:103530000B0002003749002009F0A2FE032304001B
:103540000D004BE7029B344FDE00344BBF199E1930
:10355000326973690AF010FD22002B000AF00CFD9D
:103560000B000200386F796F0AF006FD039B040020
:103570000D00002B00DBF4E6802109066B181D000E
:10358000EFE6274DEDE6C046FFFF0F440000F07F59
:10359000182D4454FB21F93FFFFFDB3FFFFF1F3E87
:1035A0009C7500883CE4377E0000F03FFFFFF23F4F
:1035B000FFFFE53F11DA22E33AAD903FEB0D7624B1
:1035C0004B7BA93F513DD0A0660DB13F6E204CC54D
:1035D000CD45B73FFF8300922449C23F0D55555555
:1035E0005555D53F2F6C6A2C44B4A2BF9AFDDE52CC
:1035F0002DDEAD3F6D9A74AFF2B0B33F711623FE6E
:10360000C671BC3FC4EB98999999C93FFF7F0340AD
:103610000000F83F0000F0BFD0E7000050E80000D5
:10362000FB21F9BFF7B554425E001443484F7608BA
:10363000E40F00933443BC4209D844424D00044394
:103640006D08E40F009101902C43BC4203D909F0AE
:10365000FBFA03B0F0BD3F4C1C19144302D1FFF735
:1036600061FEF6E79C17A446022467463C40009F93
:10367000FF0F3C43019F2F4306D1022C62D0032C45
:10368000E7D135483549E4E73700174305D1009BBA
:103690003148002B59DA3249DBE72D4FBE421BD1AE
:1036A000B5420ED1022C06D0032C07D02A48012C9B
:1036B00046D12C49CDE72C482C49CAE72A482C4949
:1036C000C7E7022C3ED0032CDBD000200021012CC8
:1036D000BFD180210906BCE71D4FBD42D7D0AD1B2D
:1036E0002D153C2D16DC002B01DA3C3515DB09F0DD
:1036F000C7FDFEF71BFEFFF715FE012C10D0022CB4
:1037000013D0002CA5D01B4A1B4B0AF035FC124AE3
:103710001A4B12E010481A49EFE700200021ECE7AD
:10372000802424060B19190093E7124A124B0AF061
:1037300023FC02000B00084810490AF01DFC88E732
:10374000104986E704480D4983E70D4981E7C046E3
:103750000000F07F000010C0182D4454FB2109C068
:10376000FB21F9BFFB21E9BFD221337F7CD9024085
:103770007CD902C0075C143326A6A13CFB2109407A
:10378000FB21F93FFB21E93F82B0F0B589B00E92F1
:103790000F93019000220E980F99002308F0D8FC97
:1037A000002808D0109811990022704B08F0EAFC0C
:1037B000002800D0CCE00E9A0F9B100019000AF0F0
:1037C00069F90290039102000B00002067490AF09A
:1037D000D3FB109A119B04000D00100019000AF091
:1037E00059F902000B00200029000AF0C5FB0E9ACF
:1037F0000F9B04000D001000190009F025FA2200AB
:103800002B00FFF70FFF0022594B0AF043F9594AEA
:10381000594B0490059109F033FD00220023040068
:103820000D0008F0B9FC0022514B002800D18AE0BD
:103830002000290009F008FA00224C4B04000D007A
:10384000109811990AF098FB02000B000AF022F977
:10385000029A039B09F0F8F90022002306900791D1
:1038600008F076FC002800D072E0290020000AF061
:10387000CBFE0AF0FFFE002206000F0010981199FF
:103880003A4B09F0E1F902000B000AF003F9029A41
:10389000039B09F0D9F9069A079B09F0F1FCFDF7A3
:1038A00005FB0022354B0AF0F5F8354A02900391EA
:1038B000344B300039000AF0EDF8A8220690079149
:1038C000D2052D4B300039000AF0E4F802000B005D
:1038D000049805990AF050FB802204000D0052055F
:1038E000294B300039000AF0D5F802000B00200007
:1038F00029000AF041FB002206000F0002980399FC
:1039000000230AF0C7F8069A079B04000D00300058
:1039100039000AF031FB02000B002000290009F0F9
:1039200093F9019B002218605960029803990023C3
:1039300009F08AF9019B9860D960019809B0F0BC40
:1039400008BC02B01847200029000AF015FB73E7F5
:103950000E4B0198196B5A6BDC6B9B6B01604260DC
:10396000029303948360C460E7E7C0460000F03F21
:103970000000E03F182D4454FB2109400000D03FD7
:103980006EC0453163626A3C460B213E50E8000040
:1039900082B0D3B5069207930400089A099B069853
:1039A0000799FDF7F9FCFDF781FA069A079B00904D
:1039B000019108980999FFF735FE002200230600BF
:1039C0000F000AF067F8009A019B09F03DF9A66024
:1039D000E760206061602000D6BC08BC02B01847D8
:1039E00082B0F0B593B004001A981B9918921993FD
:1039F000002200230AF04EF8189A199B09F024F9C6
:103A000000260200002700200B004549029603977C
:103A1000049005911A981B99009001910EA808F046
:103A2000C5FB0E9A0F9B08920993109A119B0A925C
:103A30000B93189A199B1000190009F005F91A9AAE
:103A40001B9B0AF027F80D00079032003B000798F7
:103A500029000AF01FF81A9A1B9B06000F001898FD
:103A600019990AF089FA1A9A1B9B0C900D911898D3
:103A7000199909F0E9F802000B000C980D990AF069
:103A800009F832003B0009F0DFF802000B000020CB
:103A900023490AF071FA32003B000AF06DFA8023E4
:103AA0001B06ED180B0007990200019500910EA866
:103AB000FEF7CEFD0E9A0F9B0898099909F0C4F8FD
:103AC000109A119B06000D000A980B9909F0BCF89A
:103AD00032002B00019100900EA8FFF759FF002241
:103AE000104B0EA804920593802300221B0602921D
:103AF0000393109A119B009201930E9A0F9B08F06A
:103B000055FB0E9A0F9B200022606360109A119B58
:103B1000A260E36013B0F0BC08BC02B01847C04616
:103B20000000F03F0000F0BF82B0F0B589B00F9305
:103B3000159B0E9207930600109A119B0E980F99F1
:103B4000FDF72AFC00220023149F0290039108F045
:103B5000FFFA002810D0474B196C5A6CDC6C9B6C38
:103B600031607260009301943000B360F46009B07A
:103B7000F0BC08BC02B01847079B10981199069337
:103B80000E9A0F9BFFF74EFD129A139B049005911E
:103B900002980399FEF7ACFE374A00900191049811
:103BA0000599364B09F06CFB02000B001298139933
:103BB00009F070FF002204000D0000233800069970
:103BC00008F0C6FA00282AD1049A059B8020000636
:103BD000844607990497614405910498059909F072
:103BE00059FFFDF701F802000B000098019909F058
:103BF00051FF0090019102980399FDF757F93A009F
:103C0000069B09F047FF1C4A1C4B09F039FB0200D8
:103C10000B002000290009F017F804000D00200017
:103C20002900FDF72FFE009A019B09F033FF2200C7
:103C30002B0002900391002011490AF09DF9FDF735
:103C400021FE02000B000098019909F023FF0022D9
:103C500004000D0002980399002309F01BFF0B00DC
:103C600002002900200008F0EFFF029B039C306057
:103C7000716079E750E80000182D4454FB21094099
:103C80000000E03FF0B58FB000934B005B08069357
:103C90000292D34B069A05000C000B919A425DDC10
:103CA0000AF0B2FC0490002800D07CE0149B069A35
:103CB00001332B4313430FD128002100FEF736FBBD
:103CC00002000B000020C74909F0DAFA05000C00D9
:103CD000280021000FB0F0BD149B012BF8D0029AF0
:103CE000009B2800210008F0AFFF020004980B00A1
:103CF000069007910020BC4909F0C2FA2A000890FA
:103D0000099106980799089E099F23000AF034F943
:103D1000049E02000B00029800990AF02DF932006F
:103D20003B0009F0B7FE320004000D000698079929
:103D30003B0009F0AFFE0022AA4B08F085FF02000D
:103D40000B002000290008F07FFF089A099B09F06A
:103D5000A1FE32003B0008F077FFB7E7A34B069ABD
:103D60009A4220DD002907DA802109068C46631873
:103D70001C00009B634400932A0023009C489D493B
:103D80000AF0FAF806000F00029A009B9A489B4935
:103D90000AF0F2F83B00320008F056FF002305005D
:103DA0000C00029300932A0023002800210009F050
:103DB00071FE02000B000490059109F06BFE049A5D
:103DC000059B06000F002800210009F063FE8C4AC5
:103DD000089009918B4B3000390009F05BFE8A4A4C
:103DE0008A4B08F031FF32003B0009F053FE884A4D
:103DF000884B08F029FF32003B0009F04BFE864A51
:103E0000864B08F021FF32003B0009F043FE844A54
:103E1000844B08F019FF32003B0009F03BFE824A58
:103E2000824B08F011FF049A059B09F033FE804A8B
:103E30000C900D917F4B3000390009F02BFE7E4A2B
:103E40007E4B08F001FF32003B0009F023FE7C4A64
:103E50007C4B08F0F9FE32003B0009F01BFE7A4A69
:103E60007A4B08F0F1FE32003B0009F013FE784A6D
:103E7000784B08F0E9FE32003B0009F00BFE764A71
:103E8000764B08F0E1FE02000B000C980D9908F04B
:103E9000DBFE089A099B09F0FDFD029A009B08F0E1
:103EA000D3FE049A059B09F0F5FD029A009B08F0E9
:103EB000CBFE06000F0008980999694A694B09F082
:103EC000E9FD32003B0008F0BFFE029003910200C2
:103ED0000B002800210008F0B7FE444B069A0600AC
:103EE0000F009A423DDD14980AF0C4FB32000090A6
:103EF00001913B003000390009F0CCFD009A019B94
:103F0000049005913000390008F09EFE02000B007D
:103F10000498059909F0B4F9029A039B0AF02CF869
:103F200002000B00280021000AF026F802000B0016
:103F300008F08AFE02000B00009801990AF01CF8B4
:103F40000B9B0400981702231840013B181A0D0020
:103F50000AF090FB02000B002000290009F09AFDF6
:103F6000B4E6149B012B37D00023009601970093F1
:103F7000009A019B0492059302000B0000201A494D
:103F800009F07EF92A000690079104980599069E8B
:103F9000079F230009F0F0FF009E02000B0002982B
:103FA000039909F0E9FF32003B0009F073FD32008C
:103FB00004000D00049805993B0009F06BFD0022F8
:103FC000084B08F041FE02000B002000290008F019
:103FD0003BFE069A079BBAE605000C0078E6C04651
:103FE000FFFF2F3E0000F03F0000F0BF2794E53FA9
:103FF000182D4454FB21E93F075C143326A6813C6D
:10400000D47ABF74702AFB3EE9A7F0320FB8123F92
:1040100068108D1AF726303F1583E0FEC8DB573F46
:1040200093846EE9E326823FFE41B31BBAA1AB3F06
:10403000735360DBCB75F3BEA69237A0887E143F26
:104040000165F2F2D844433F280356C9226D6D3F03
:1040500037D60684F464963F7AFE10111111C13FE1
:10406000635555555555D53FF0B54B008FB05B089E
:1040700000931700DA4B009A040007919A4209DC7A
:1040800002000B003A607B6000220023BA60FB60F4
:10409000002624E0D34B009A9A4200DD6DE0D24A1C
:1040A000002935DDD14B09F067FF009B04001A00A1
:1040B000CE4B0D009A4215D0CD4ACE4B09F05CFF95
:1040C00002000B0020003A607B60290009F054FFD9
:1040D000C74AC84B09F050FF0126B860F9603000AC
:1040E0000FB0F0BDD322C34B520509F045FFC24AC1
:1040F000C24B04000D0009F03FFF02000B0020003E
:104100003A607B60290009F037FFBB4ABB4BE1E70F
:10411000B64B08F099FD009B04001A00B34B0D004C
:104120009A4214D0B24AB34B08F08EFD02000B0045
:1041300020003A607B60290009F01EFFAC4AAD4BBD
:1041400008F082FD0126B860F9607642C7E7D32205
:10415000A84B520508F078FDA74AA84B04000D00B3
:1041600008F072FD02000B0020003A607B6029001D
:1041700009F002FFA04AA14BE2E7A14B009A9A4244
:1041800000DDD0E0FEF7D2F89E4A9F4B04000D0000
:1041900009F080FC00229D4B08F056FD0AF034FA2D
:1041A00006000AF067FA904A904B0490059109F0D6
:1041B00071FC02000B002000290009F0DDFE8C4A92
:1041C00002900391049805998A4B09F063FC04005E
:1041D0000D0002000B000298039909F0CDFE1F2E7E
:1041E00028DC8B4A731E9B009B58009A934221D077
:1041F00002000B003A607B60029803997B683A6882
:104200000093009B09F0B8FE22002B0009F0B4FED9
:104210000B000200BA60FB60079B002B00DB5EE72F
:10422000802212069446009B891863447B60B86024
:10423000F9608AE7009B1B150693069A4B005B0DFD
:10424000D31A102BD4DD04980599D322694B52055B
:1042500009F020FC04000D0002000B0002980399F5
:1042600009F08AFE02000B00009001910298039968
:1042700009F082FE22002B0009F07EFE04000D00F2
:10428000049805995C4A5D4B09F004FC22002B0060
:1042900009F072FE02000B0004000D000098019965
:1042A00009F06AFE069A4B005B0DD31A312B08DC2D
:1042B00002000B003A607B60009A019B029203931C
:1042C0009AE7B8220498059992054C4B09F0E2FB55
:1042D00004000D0002000B000098019909F04CFE4B
:1042E00002000B00029003910098019909F044FE2E
:1042F00022002B0009F040FE04000D0004980599EF
:10430000444A454B09F0C6FB22002B0009F034FE5D
:1043100002000B0004000D000298039909F02CFE26
:104320003860796068E73D4B009A9A4208DD0200E8
:104330000B0009F021FEB860F96038607960A7E6EB
:10434000009B374A1B159B18009A02931B05D51A30
:1043500029000AF059F90AF08DF902000B0020003B
:1043600029000892099309F007FE00222D4B09F05D
:1043700091FB04000D000AF047F90AF07BF90200F6
:104380000B0008AEB260F3602000290009F0F4FDD4
:104390000022244B09F07EFB032430617161651E0D
:1043A000EB00F318186859680022002307F0D0FECC
:1043B000002813D123003000029A3900FDF716FDC2
:1043C000079B0600002B00DB89E680227B68120633
:1043D0009B187B60FB689B18FB60B6E62C00DEE751
:1043E000FB21E93F7BD9024000004054FB21F93F0B
:1043F0003163621A61B4D03D7370032E8A19A33BF6
:10440000FB21394183C8C96D305FE43F0000E03FC4
:10441000F8EF0000C14920259A837B39FFFFEF7F29
:10442000EAFBFFFF0000704130B5204A4B0087B027
:104430005B08934206DC0023002200930023FDF773
:10444000E1F806E01A4A934205DD02000B0009F08C
:1044500093FD07B030BD02AAFFF706FE049C059D40
:1044600003230340012B0AD002980399022B0DD09D
:10447000002B15D10133009322002B00DFE722002F
:10448000029803992B00FDF709FBE2E701232200C4
:1044900000932B00FDF7B6F880231B06C918D8E758
:1044A00022002B00FDF7FAFAF6E7C046FB21E93FB0
:1044B000FFFFEF7F30B51E4A4B0087B05B08934289
:1044C00004DC00220023FDF7E9FA06E0194A9342D2
:1044D00005DD02000B0009F04FFD07B030BD02AA58
:1044E000FFF7C2FD049C059D03230340012B08D068
:1044F00002980399022B0FD0002B12D122002B001F
:10450000E1E700932200029803992B00FDF77AF867
:1045100080231B06C918E0E722002B00FDF7BEFA36
:10452000F6E70123220000932B00FDF76BF8D4E798
:10453000FB21E93FFFFFEF7F82B0D0B586B00400DA
:104540000C980D990A920B9304AA02ABFEF73EF861
:104550000A980B99FFF7AEFF029A039B09F09AFAAB
:1045600006000F000A980B99FFF75EFF049A059B5F
:1045700009F090FA002200900191002330003900E8
:1045800009F088FA02000B000098019908F05CFB22
:10459000206061602000A660E76006B0D0BC08BC67
:1045A00002B0184782B0D3B506920793040006986C
:1045B0000799FCF719FB06000F0008980999FFF707
:1045C00033FF32003B0009F065FA00900191089832
:1045D0000999FFF76FFF32003B0009F05BFA0022F8
:1045E00006000F0000980199002309F053FA020019
:1045F0000B003000390008F027FB009A019B206077
:104600006160A260E3602000D6BC08BC02B018471D
:1046100082B0F0B50026002797B01D931E9B1F9D0A
:104620000E9304001C923B0032000E982900069560
:1046300007F08EFD002821D01C981D9932003B0008
:1046400007F096FD002819D01C981D99FDF74CFB2A
:104650001C9A1D9B07F07CFD00280FD032003B0008
:1046600000208B4908F00CFEA660E76020606160C6
:10467000200017B0F0BC08BC02B0184780231C987B
:104680001D991B06EB180F930022824B07F066FD65
:10469000002854D01C981D997F4A804B09F0FAF9E4
:1046A0007D4A06000D007D4B0E98069909F0F2F93F
:1046B00032002B000191009012A8FFF73DFF149AE1
:1046C000159B129E139F069207931C9A1D9B002018
:1046D0006F4909F051FC0B000F99020001910E99EE
:1046E00012A80091FFF794FF149A159B12A8049248
:1046F0000593129A139B02920393069A079B0092CA
:10470000019332003B0007F051FD149A159B04926F
:104710000593129A139B029203930022002312A87E
:10472000009201935C4A5D4B07F0B4FF129A139B11
:1047300022606360149A159BA260E36098E70022F0
:104740001C981D99524B09F017FC002200230C9273
:104750000D93012201254E4B089009910A920B936B
:104760004F4B50331093109AEB00D3181E685F68BC
:104770000E9A069B28000492059309F07BFF089A85
:10478000099B08F061FA0022002302900391009235
:10479000019312A832003B0007F07CFF129A139B92
:1047A0000A980B9908F050FA149A159B0A900B91ED
:1047B0000C980D9908F048FA01350C900D910B2DCD
:1047C000D1D1089809990022364B08F03DFA002211
:1047D000304B08F039FA0500109111912E483249FA
:1047E000FCF726FD002206000F0008980999294BC6
:1047F00008F02AFA0E9A069B029003910492059300
:10480000069B2A0001930E9B12A80093119BFFF7B1
:104810008BF91298139932003B0009F03BF93200F2
:1048200006900791149815993B0009F033F98022FE
:10483000120694460F0006000F9A109B01920E9AE2
:104840006344009212A82A00FFF7ACFE149A159B4D
:1048500012A804920593129A139B00960197029254
:104860000393069A079B07F0A1FC0C9A0D9B12A8D4
:10487000049205930A9A0B9B02920393149A159B38
:1048800000920193129A139B07F090FC4EE7C046EA
:104890000000F03F0000E03F182D4454FB21094088
:1048A00050E8000000002240FB211940F8B50D003F
:1048B00017001E00040009F0A7FE386009F0DAFEB8
:1048C00002000B002000290009F056FB0022104BCB
:1048D00009F0E0F804000D00FBF7FEFE09F094FE7D
:1048E000306009F0C7FE02000B002000290009F02B
:1048F00043FB0022074B09F0CDF8FBF7EDFE09F072
:1049000083FE002800D10130069B1860F8BDC04628
:1049100000408F400000594030B50A4B652804DD47
:10492000032287331A70002030BD000118180930A7
:10493000FF30026843688468C5680A604B608C6019
:10494000CD60F0E7C80C001070B505000C00002227
:1049500000232800210007F001FC002807D02800D0
:1049600080252D066119FDF7BFF9491970BD280092
:104970002100FDF7B9F9F9E7F7B505000E006F4220
:104980002F4373005B08FF0F1F432F4B0095DF1B66
:10499000FF0F54D128003100FCF73AFC041E50D11F
:1049A000002200232800310007F0D2FB00283AD172
:1049B000002200232800310007F0D0FB002806D099
:1049C0008021009A0906731815001E00D7E70022FF
:1049D0001E4B2800310007F0DFFB002815D0002215
:1049E0001B4B00920193009801992A00330007F0B5
:1049F000C9FB002817D1009801990022144B09F037
:104A000049F8013400900191EDE7124C124B0093EC
:104A100001940124009801992A00330007F0A8FBB3
:104A2000002802D064422000FEBD009801990022B7
:104A3000074B08F025FC013400900191EAE70024BF
:104A4000F1E73C00EFE7C0460000F07F0000F03FD8
:104A5000000024409999B93F9A9999990A4B10B549
:104A60001A007E321278002A0BD17F331B78002285
:104A7000002B07D0054B09F00DF8054A054B08F04F
:104A8000FFFB10BD044BF6E7C80C00100000794096
:104A9000182D4454FB211940008076400200082163
:104AA00003000120473A8A43D2B210B5824220D98E
:104AB0001A0004246F3AA243D2B2002A19D01A0075
:104AC000763A0A2A15D940221800904302000120A4
:104AD0002B2A0ED09A1F82420BD9073AA243D2B298
:104AE0000400002A05D000208B43433BDBB29C42EC
:104AF000404110BD70B50124084E094D305D0028BD
:104B000009D0FFF7CBFF431E98410019441CAC426B
:104B1000F4DDFA24E400200070BDC046F804001063
:104B2000CF07000070B504000D00FFF7E3FF154B41
:104B30001A1AAA4204DA0322134B87331A7070BD83
:104B40009C42FCDC2919FAD4002DF8D00ADD0021A2
:104B50000E4BED18A042F2DBC21816782E541170DD
:104B60000138F7E7FA2200230848D200121B09187F
:104B700024189A42E3DDE05CC8540020E05401337D
:104B8000F7E7C046CF070000C80C0010F80400107B
:104B9000F8B506000400064F351B002C05DD013C6E
:104BA000385DFFF77BFF0028F6D101202840F8BDD3
:104BB000F804001070B50A4E04B223B2002B01DCD9
:104BC000084809E0A5192B782B2B06D12000FFF708
:104BD000DFFF002801D1687870BD013CEDE7C046D9
:104BE000F8040010FFFFFF7F7C23F0B5124A83B06A
:104BF0000192D55A012D0FD90024104E6F1E02E0EC
:104C00000134BC4206D02B1B023BF05CFFF746FF91
:104C10000028F5D1E30709D40120002D04D07C231E
:104C20000020019A013DD55203B0F0BD7C23019ACA
:104C3000023DD5520020F7E7C80C0010F804001020
:104C400010B50122802806D8044980004358002B63
:104C500001D098470022100010BDC046F4ED0000BE
:104C6000F0B57C241D491E4B0A5B08209D5C2B007F
:104C7000473B8343DBB2012B22D92B0004266F3B39
:104C8000B343DBB2002B1BD02B00763B0A2B17D98A
:104C900040232F009F432B2F12D0AB1F012B0FD986
:104CA000073BB343DBB2002B0AD08543433D012DC4
:104CB00006D90C4B9A4206D8013200200A5306E06E
:104CC000094B9A4204D9872303220120CA54F0BD1C
:104CD0007C230232CA520020F9E7C046C80C0010FB
:104CE000F8040010CE070000CD070000F7B5114C06
:104CF000019123007C331B880F4D0700EA5C002ADA
:104D000001D1002B01D1FFF7ABFF7C3420880121BA
:104D1000FFF708FF26883800AF55FFF7BFFE0028D1
:104D200007D0701C0121FFF7FDFE2388ED18019BC1
:104D30006B70F7BDC80C0010F804001030B5FA24F1
:104D400000230849E400CD5C5A1C2B2D04D18D5C56
:104D5000854201D1981C30BD1300A242F3D100203E
:104D6000F9E7C046F804001010B5682802D8FFF72C
:104D7000E5FF10BD0A4BFE280CD1E922D2009B189A
:104D80001868596809F040FC03004042002BF0DB32
:104D9000D8B2ECE7032287331A700020E9E7C04657
:104DA000C80C001083280DD80F290BD88423CA08FB
:104DB000534318180723194079330B41024A115CF9
:104DC0000B4313547047C046D8140010F0B587B099
:104DD00003923C4A0493D3780C00834204D21378A4
:104DE0000193019807B0F0BD002153689278801AB2
:104DF0001A7888421ADC991C5B78009101938B1811
:104E000005930C9B002B02D0019BE41A0134049BF8
:104E1000E5B20027002B1BD10025E4B20295019BCF
:104E2000029A9342DDDD082600273DE002329B18FE
:104E30000131DDE7039B2800F118C9B2FFF7B2FF8B
:104E40000136204B5B789E42F4DB01350137EDB231
:104E5000019BBB42E0DD0026F3E7082E08D1059B4D
:104E6000009A9342BDD013000026013315780093B9
:104E700001231D4215D0039BF918049BC9B2002BD6
:104E80001CD0832C0DD80F290BD88422CB08534378
:104E90007D3A0A40802111410B481B19C25C8A43AC
:104EA000C2546D1001370136064B5B789F42D4DB4C
:104EB000029B013401330293E4B2B0E72000FFF714
:104EC00071FFEEE700000010D814001070B50D005F
:104ED00004000122FBF744FA290001222000FBF71D
:104EE0001BFA70BD0122F8B5082107001000FBF77E
:104EF00013FA07240826002231000120FBF70CFAE0
:104F00003A000125224102212A400020FBF704FA41
:104F10002A0031002800FBF7FFF9013CEBD2F8BD75
:104F2000002210B5040011000220FBF7F5F9200063
:104F3000FFF7D8FF10BDF7B5012300245026134D0D
:104F40000093019476426A46A300D058002730436C
:104F5000C0B2FFF7E5FF0020FFF7E2FF1020FFF7E8
:104F6000DFFFE020FFF7DCFF012200210220FBF73A
:104F7000D3F9E85D0137FFF7B5FF842FF4D184350D
:104F8000012C00D1F7BD0124DDE7C046D814001084
:104F9000704770470122024B80331A707047C04639
:104FA000C80C0010054B002219007C310A80190042
:104FB00086310A70A43301321A707047C80C001091
:104FC00010B5074C230085331B78002B03D00C2130
:104FD0007620FFF78BFE0123A434237010BDC0465A
:104FE000C80C0010044B84331A787F2A02D8FF22A1
:104FF0001A7070470022FBE7C80C001010B5064C71
:105000007C342388002B02D0FFF7EEFD10BDFFF7A4
:1050100071FD2080FAE7C046C80C001010B5074C9F
:10502000230085331B78002B03D00B217620FFF75C
:105030005DFE0123A434237010BDC046C80C0010CF
:105040008022024B52007E331A807047C80C001039
:105050000122024B7E331A807047C046C80C0010F4
:105060000022024B7E331A807047C046C80C0010E5
:1050700070470022014B80331A707047C80C001033
:105080000122024BA4331A707047C046C80C0010AE
:105090000122024BA4331A707047C046C80C00109E
:1050A0000022054B84339A56002A02DC01221A7032
:1050B00070470022FBE7C046C80C0010054B0021DA
:1050C0001A008132117082331A7851424A411A70A3
:1050D0007047C046C80C0010054B00211A008232F0
:1050E000117081331A7851424A411A707047C04694
:1050F000C80C001070B5114C114923007C331A887C
:10510000885C002803D1002A01D0188070BD2300DC
:1051100085331B78002B02D0FFF7A2FDF6E72500B0
:10512000012386352B70FFF78BFD2B78002B01D0E8
:10513000FFF796FD002386342370E7E7C80C0010C4
:10514000F8040010F7B516001F000090019100222E
:105150001B4B3000390007F001F8002801D0002671
:10516000174F0024164D009A019B3000390006F0BD
:10517000FFFF002803D12000290003B0F0BD20006C
:10518000290032003B0008F085FC04000D002000DF
:105190002900FCF73DF80028EDD1634223436A0063
:1051A0005208DB0F1343074AD31AE4D43000390006
:1051B0000022034B07F048FD06000F00D3E7C0466E
:1051C0000000F03F0000F07FF0B585B004000191D1
:1051D00015008A4206DD00220023026043600020A1
:1051E00005B0F0BD0268436828000292039309F0FD
:1051F00041FA02000B0000201749FDF779FB060079
:105200000F000298039907F009FD02900391300006
:10521000390007F0E5FC07F001FD0B0002000298E1
:10522000039908F02DF8FBF757FA07F0D9FC019B1A
:1052300003C49D4203D10843411E8841D0E707F0D3
:10524000EDFCFFF799FB019BC1175D1BEB0FA8421B
:1052500059410800C4E7C0460000244073B51D0052
:10526000104B14001E001A00B836C832009001918D
:1052700010685168306071609068D168B060F1600A
:105280001E00A833D836306871689C60DD601060FD
:105290005160B068F1689060D1600099019A19601E
:1052A0005A6073BDC80C001073B514000C4A00900E
:1052B000019116001D000B4B983618685968103B79
:1052C000186259629869D9699862D962B342F4D177
:1052D00000980199A8329460D5601060516073BD48
:1052E000C80C0010900D0010F8B51F00074B04000B
:1052F000A4331B780D001600002B05D020002900D8
:1053000032003B00FFF7D0FFF8BDC046C80C0010CC
:10531000D0B5164C164A23000833DB6F13400CD16E
:10532000144AA534916D002902DD21709365D0BD2A
:105330002378936504232370F9E7230086331B78D1
:10534000002BF4D00B4B5869EF23DB00E358A43457
:10535000C01A09F0C9F90022074B07F091FF00239A
:105360000022FFF7C1FF0123E5E7C046C80C00108B
:1053700000FFFF004804001000408F40F8B5FBF725
:105380003DF9584F0400031EFE6D574D3FD1032ECB
:105390002DD12B0085331B78002B05D12B007A33C0
:1053A0001B78002B00D134002B0081331A78002A9F
:1053B00003D0052E01D000221A702B0082331A78F8
:1053C000002A03D0092E01D000221A702B000022DF
:1053D00084339A56002A05D02F2E0FD0572E0DD089
:1053E00000221A703A2E09D1FFF792FF06E0532EE1
:1053F00002D12B008533D3E7002ED5D12A0000231C
:105400007A3279351370FB652B703B663DE02A00DC
:1054100081321278002A21D02834FB22053B134226
:1054200004D12000282106F07FFE0C00B44242D1B6
:10543000032C2CD12B0085331B78002B15D0002595
:105440003B6E022B32DD642D1FDC0120FAF7FCFEDF
:10545000FBF7D4F8002810D00135F1E72A0082329A
:105460001278002AD9D05034D7E7204C0120FAF71F
:10547000EBFEFBF7C3F8002801D1002405E0013C56
:10548000002CF3D101237A352B702000F8BD532C6A
:10549000D5D0174D0120FAF7D7FEFBF7AFF800285B
:1054A000EBD0013D002DF5D1A034EEE7114A954235
:1054B000CBD10133A9E72B000833DA6F0E4BFC6523
:1054C0001A42E2D1032C01D0532CDED1C820FAF7C6
:1054D000BBFEFBF793F80028CFD0012379352B7062
:1054E000CBE7C04648040010C80C0010D1070000EC
:1054F000E90300005902000000FFFF0010B50C4C4A
:1055000000232100A83100228868C96806F020FE27
:1055100003000120002B09D0B8340023A068E16803
:10552000002206F015FE43425841400010BDC0461F
:10553000C80C001070B5FFF7E1FF03000020012B3D
:1055400016D00C4B0022A8331C685D680A4B200063
:10555000290006F00DFE00280AD0084B002220008A
:10556000290006F019FE431E9841434201201840CD
:1055700070BDC046C80C00100000F03F0000F0BF36
:10558000F0B585B002900C0003921F0006F086FA79
:10559000451E002D01DB002C01DC05B0F0BD029B97
:1055A0002100585D0123039A00933B00FFF70EFC96
:1055B000241A002F02D1013C013DEAE70026B54242
:1055C000F9D0064B5B789E42F5DA039BE0B299195D
:1055D000C9B2FFF7E7FB0136F3E7C0460000001051
:1055E000F0B50500012789B0280006F057FA2B789E
:1055F00001902D2B08D000242600019B9C4206DB45
:105600003800704309B0F0BD01357F42ECE7285DFA
:10561000303809F02FF8019B02900391581E001BAF
:1056200009F028F802000B0000200D49FDF760F991
:1056300004900591300009F01DF8049A059B06902E
:1056400007910298039908F025FA02000B000698CA
:10565000079907F0F9FA08F0D7FF01340600CCE704
:1056600000002440F0B5060087B006F017FA337842
:1056700003902D2B25D1701CFFF7F4FF80231B0610
:10568000C91807B0F0BDF25C2E2A18D0452A00D107
:105690001F000133039A9342F5DB8C4205D1A742E8
:1056A00014D1300006F0FAF904000022002300258E
:1056B00000920193039B9D420ADB00200EE01C0038
:1056C000E7E72A4C002327002100E3E73C00ECE752
:1056D000AF4210D1781C3018FFF782FF08F0CAFFE4
:1056E00002000B0000202249FDF702F9009A019BFD
:1056F00008F0D0F9C5E7AC421FDD705D303808F026
:10570000B9FF04900591601E401B08F0B3FF020032
:105710000B0000201649FDF7EBF802000B0004987F
:10572000059908F0B7F902000B000098019907F0FD
:105730008BFA009001910135BCE7AC42FBDA705D59
:10574000303808F097FF04900591281B08F092FF6D
:1057500002000B0000200649FDF7CAF802000B000A
:105760000498059907F08CFDDDE7C046E7030000CB
:1057700000002440F0B5264D85B02C006434200094
:1057800006F08CF90023C2B2A275E3752376637626
:10579000A376E3769A4201D00133237664352B78E1
:1057A0002D2B01D12C3BAB760022C3B20393160004
:1057B00015001400110001230292019203988842FF
:1057C00012DC002D02D0124B6433DC75002E03D0A6
:1057D0000F4B019964335976002A03D00C4B029A7F
:1057E0006433DA7605B0F0BD094864300F5C0131EE
:1057F0002E2F07D0452FE1D1085CCCB201942D2883
:1058000003D01E001D001C00D8E71A000293F8E721
:10581000480400107FB51C4C0600230064331B7E37
:10582000002B1DD1194D2B009C331B78002B17D159
:10583000174BA835196C5A6C009101929A6CDB6C6D
:105840000098019902920393029A039BFFF74CFD83
:10585000009A019B2A606B60029A039BAA60EB602E
:105860000A4964347831A07DE27D0978821A8A423F
:1058700004DB637E002B01D1452E02D1024B643341
:105880001E54FFF777FF7FBD48040010C80C0010BE
:1058900050E8000010B50B4C230064331B7E002B36
:1058A00006D13120FFF7B6FF0122074BA4331A704F
:1058B0006434637E002B04D14520FFF7ABFFA37D4A
:1058C000637610BD48040010C80C001010B5074BDB
:1058D0006433DA7D002A08D11B78002B02D13020F6
:1058E000FFF798FF2E20FFF795FF10BD480400102A
:1058F00010B53920FFF78EFF10BD10B53820FFF727
:1059000089FF10BD10B53720FFF784FF10BD10B51B
:105910003620FFF77FFF10BD10B53520FFF77AFF67
:1059200010BD10B53420FFF775FF10BD10B5332042
:10593000FFF770FF10BD10B53220FFF76BFF10BDF1
:1059400010B53120FFF766FF10BD10B53020FFF70E
:1059500061FF10BDF0B5060085B00F0006F09EF89F
:10596000350000240390039AAB1B9A4201DD832C7F
:1059700001DD05B0F0BD00232878210000933A0036
:10598000FFF724FA241801340135ECE7802273B5BF
:10599000002107252B4B2C4C920301912000DA6744
:1059A000902206F043F8019B284EA360284B1A680A
:1059B000AA431A600122196811431960254B19681E
:1059C000A9431960196811431960802322495B01BA
:1059D000086803430B60214B1A6082323260204A10
:1059E000126819681F4B1868504306F09BF8E121B4
:1059F000090306F097F810221B4B1C491A60030A92
:105A00000B6003231A4AC0B210603360194B1D604B
:105A1000194B593518680190080011001A682A407E
:105A2000602AFBD15F3A1D68154207D1227080229F
:105A3000124B92031A600523036073BD0D68019534
:105A4000F1E7C04604E100E0481400100C8000407B
:105A5000A4400440A8400440808004409880044052
:105A600078800440480400102880004004800040F2
:105A700000800040088000401480004000E100E009
:105A8000FA2110B50C4C8900206806F067FA0B4B20
:105A9000984209D800230A4A013863611060094A14
:105AA00013600722084B1A60FFF770FFFAF708FB34
:105AB000FAF7EEFC10BDC04648040010FFFFFF00DF
:105AC00014E000E018E000E010E000E010B500286D
:105AD00039D080211D4A13688B43136001231C4970
:105AE0000A681A42FCD003221A4B1A6001230021D3
:105AF000194A13601160136011681942FCD0174AEB
:105B00001749136080230C685B0223430B6011006C
:105B1000002804D180230D4A146823431360114BDD
:105B20009A6882420ED09860431E98410E4B4042C4
:105B300018400E4B0968C01805F0F4FF0C4B1860B4
:105B4000FFF79EFF10BD034B1860CFE7388204407B
:105B50000C800440708004407480044078800440CD
:105B6000808004400000001000512502001BB70097
:105B700048040010F0B587B00190039172B68022FE
:105B80007E4B1202DA676C2200247D4B7D481A603E
:105B90007D4B1968014019601A6804211A607B4B1B
:105BA0001A6802401A601A6800201A600122FAF787
:105BB000D7FB012204210020FAF7AEFB01220521C8
:105BC0000020FAF7CDFB012205210020FAF7A4FB03
:105BD0006F4B704D1C6022352B19665D5F7801227A
:105BE00039003000FAF7BCFB0234002239003000E3
:105BF000FAF792FB142CEFD100240020FAF78EFC68
:105C0000654B210065485C65FAF772FB210064482A
:105C1000FAF76EFB21006348FAF76AFB210062483D
:105C2000FAF766FB21006148FAF762FB604B614DB1
:105C30001A68614B614E1A60019B5A1E93413F22C4
:105C40005B4293435E4A9B185E4A136004235E4A9C
:105C500011680B4313605D4B2C601A685C490A4065
:105C60001A600293039B2A689B0700D481E0EC230F
:105C70005B0113432B6080233360DB183360802388
:105C8000DB00336080235B01336080231B013360C2
:105C9000019B002B56D000244E4B4F4F1C604F4BA6
:105CA00021001C604E4B38001C604E4B1C60FAF704
:105CB0001FFB220009212000FAF752FB22000921D4
:105CC0002000FAF729FB8021474A484813680B4314
:105CD000136007223B68763993433B603B68053A83
:105CE00013433B60019B584305F01CFF0322404BCC
:105CF00040491860404B02981C60404B1A60404B72
:105D00001A680A4080211A601A680A431A608023C0
:105D100080229B0052023360326002687E391A434F
:105D200002602A6813432B600123364A1360364A07
:105D30001160364A274913601460136010681842D6
:105D4000FCD00B600122324B52421A60314B1A6870
:105D5000059262B630BFC046059A1B689A4206D1CA
:105D600030BF2D4B9868FFF7B1FEFAF783FA07B002
:105D7000F0BD80231B0113432B6086E704E100E0A4
:105D800018000040F8FCFFFF30400440344004405D
:105D90000480044050E7000048040010084004401C
:105DA00000400440AC400440144004401C40044007
:105DB00038820440048204403482044000E100E060
:105DC000FF1800003082044010ED00E00082044023
:105DD0007FE2FFFF04C00040644004400400014033
:105DE000044001400480014080800440841E000083
:105DF00018C000400FF0FFFF08C0004014C0004072
:105E00003CC00040788004407080044074800440AE
:105E100008820440C804001000000010842210B55D
:105E200052000021014805F001FE10BDD8140010F9
:105E300010B508210120FFF749F802210020FFF7E3
:105E400045F800210220FFF741F806210220FFF764
:105E50003DF803210800FFF739F80321002208006C
:105E6000FAF75AFA002206210220FAF755FA01221F
:105E700006210220FAF750FAFFF7D0FFFFF75BF890
:105E8000A220FFF74DF8A020FFF74AF8C020FFF747
:105E900047F8F820FFF744F80020FFF741F80A2000
:105EA000FAF7D2F94020FFF73BF82C20FFF738F83B
:105EB0003220FAF7C9F92E20FFF732F83220FAF72C
:105EC000C3F92F20FFF72CF80A20FAF7BDF9252097
:105ED000FFF726F80A20FAF7B7F98120FFF720F834
:105EE0000020FFF71DF8AF20FFF71AF8A420FFF7F6
:105EF00017F810BD70B50A20FAF7A6F9FFF73EFAB9
:105F00000128F8D01D4D2C0048342379002B19D0DE
:105F1000002323712372E3706379002B07D1C12220
:105F2000022152000E20FAF795FA012363710C2228
:105F3000012148352B7908001A43AB795B001A43DD
:105F4000FAF788FAAC20FEF7EBFFAE20FEF7E8FF89
:105F5000A520FEF7E5FF00200121FFF70BFE002042
:105F6000FAF710FB002802D10121FFF703FEFFF72B
:105F70005FFFFFF753FFFEF7DEFF70BD4804001020
:105F8000CC2210B5D2000021014805F04FFD10BD14
:105F9000D00D001010B5044816220021643005F021
:105FA00045FDFFF7E7FB10BD4804001070B50E4C2F
:105FB00023009C331B78002B14D10C4D6435280032
:105FC00005F06CFD00280DD02800FFF74BFB2300E7
:105FD000A8331860596000220023B0342260636047
:105FE000FFF7D8FF70BDC046C80C00104804001071
:105FF000F0B589B0FFF7DAFF464B5C681B68009389
:10600000019400980199434BDC689B6802930394C8
:10601000029A039BFFF768F93F4B1C6C5D6C9E6C0A
:10602000DF6C2000290032003B00FFF73DF93B4BBD
:106030002933FF331C685D68384B20003933FF3348
:106040001A685B6800920193344B29004933FF338F
:106050001A685B6804920593304B00225933FF3372
:106060001E685F682E4B07F087FF22002B0007F0A9
:1060700011FD2A4B029003916933FF331A685B6864
:106080002000290007F006FD3200069007913B0032
:106090003000390007F0FEFC02000B00069807995B
:1060A00007F06AFF029A039B07F0EAF8FBF7C0F8D3
:1060B00000260027194BB83318605960174B200091
:1060C000C0331E605F60049A059B290007F0E2FC64
:1060D000009A019B04000D001000190007F0DAFC83
:1060E00002000B002000290007F046FF029A039BE4
:1060F00007F0C6F8FBF79CF80122064B18605960C0
:10610000064BB0331E605F60044BA4331A7009B0B5
:10611000F0BDC046700D001050E80000C80C001023
:106120000000F03FF7B5FFF741FF204C2500A835F0
:1061300028686968AA68EB68FFF7D6F81C4B1E6CE4
:106140005F6C9A6CDB6C00920193009A019B3000AB
:106150003900FFF7A9F82300210029335931FF3313
:10616000FF311A685B68260008684968009201934D
:1061700007F086F8B83630607160210023000026F1
:1061800000273931C033FF311E605F6008684968FD
:10619000009A019B07F074F82300B0331E605F6023
:1061A0000123A434286069602370F7BDC80C001077
:1061B00050E8000070B5FFF7F9FE0B4C2500A8353C
:1061C000AA68EB6828686968FFF78EF82300E8334F
:1061D00019685A6829606A609A68DB68AA60EB608F
:1061E0000123A434237070BDC80C0010F8B5FFF76C
:1061F000DDFE084BD8331E685F689C68DD683000A0
:106200002B0039002200FFF76FF80123014CA43462
:106210002370F8BDC80C001070B5FFF7C7FE0B4C1B
:106220002500A835AA68EB6828686968FFF75CF85C
:10623000074BA434996ADA6A29606A601A6B5B6B4F
:10624000AA60EB600123237070BDC046C80C00102B
:10625000D0E80000F0B587B0FFF7A8FE484B1C68F7
:106260005D68484B20001E685F68474B2900793302
:10627000FF331A685B6807F00DFC444B00900191F6
:106280001A685B683000390007F004FC02000B005C
:106290000098019907F070FE3B4B0290039149333F
:1062A000FF331A685B682000290007F0F3FB320017
:1062B00004000D003B003000390007F0EBFB02004A
:1062C0000B002000290007F057FE2F4E009001918F
:1062D000A83630687168B268F368FFF705F82C4B90
:1062E0001C6C5D6C9A6CDB6C04920593049A059BA4
:1062F00020002900FEF7D8FF009A019B029803991D
:1063000006F0BEFF204C0022B834206061600021FE
:106310001D4BC03319605A60009801991B4B1A68D5
:106320005B6807F0B7FB174B04001A685B680D0049
:106330000298039907F0AEFB02000B002000290031
:1063400007F01AFE0E4B04001A685B680D000098F7
:10635000019907F09FFB02000B002000290006F0C6
:106360008FFF0022306071600021074BB03319604D
:106370005A600122044BA4331A7007B0F0BDC04626
:10638000F00D0010000E0010C80C0010200E0010C0
:1063900050E80000F8B5FFF709FE0D4C002225007B
:1063A000A8352E686F6800233000390007F072FBB3
:1063B00002000B00A868E96806F046FC2300B03331
:1063C0001E605F600123A434286069602370F8BDFB
:1063D000C80C001073B5FFF7E9FD124B1E00A8367C
:1063E000B168F2680091019234687568009801996B
:1063F0001A00F832146055609060D1601A00B8320B
:106400001068516814605560306071609068D168A0
:10641000B060F160009801999060D1600122A433CE
:106420001A7073BDC80C0010F7B5FFF7BFFD144C10
:1064300025002300F835A83319685A6829606A6076
:106440009A68DB68AA60EB602300B8331E685F6857
:106450009A68DB6800920193009A019B3900300032
:10646000FEF7FCFE29686A682300D83319605A6079
:10647000A968EA689960DA600123A4342370F7BD43
:10648000C80C0010D0B52A4C8CB02200833213788F
:10649000002B07D0012B03D10B3313700CB0D0BDF0
:1064A000013BFAE7FFF782FD2300A83319685A6819
:1064B000069107929E68DF680698079900220023DC
:1064C00005F046FE00280BD00022002330003900E2
:1064D00005F03EFE002803D0873401232370DDE75A
:1064E00023000699079AE83319605A602300F033B5
:1064F0001E605F6013000A000292039300220023D3
:10650000049605970092019308A80022094B06F013
:10651000C1F80899099A2300A83319605A600A99AA
:106520000B9A2300B03319605A60A434D5E7C046F3
:10653000C80C00100000F03F10B5FFF737FD064B08
:106540001A00A833E83218685968106051609868DA
:10655000D9689060D16010BDC80C0010F7B5FEF787
:10656000CDFF284E002803D0022387363370F7BDB5
:10657000FFF7E2FF3300A836B833776836681C6847
:106580005D6832003B002000290007F0F5FC009018
:10659000019102000B003000390005F0E9FD0022F6
:1065A000194B00282AD00098019906F04DFB0200F3
:1065B0000B0020002900FEF7C5FD009A019B040096
:1065C0000D003000390005F0D3FD002801D1009EF8
:1065D000019F00220C4B30003900FEF7B3FD020092
:1065E0000B002000290006F04BFE00220023FEF7DE
:1065F00035FE0122034BA4331A70B8E7300039008E
:10660000D3E7C046C80C00100000F03FF0B589B0D9
:10661000FEF774FF394C0590002804D0022387341C
:10662000237009B0F0BD26002936FF36FFF784FF3E
:10663000306871680022324B07F09EFC069007918B
:106640000B0021002500270002003931F835A8375A
:10665000FF312A636B63086849683A687B68009277
:10666000019307F089FC009A019B2864696410007B
:10667000190007F00FFA0B00224902000868496868
:1066800007F07AFC28656965210023005931B83389
:10669000FF311A685B68086849680292039307F043
:1066A0006BFC029A039B286669661000190007F0CC
:1066B000F1F90B00144902000868496807F05CFC16
:1066C000029A039B2867696700980199250007F0E3
:1066D000E1F97935FF3502000B002868696807F099
:1066E0004BFC069A079B286069603A607B60B26841
:1066F000F368A434BA60FB60059B91E7C80C0010F6
:106700000000F03F100E0010300E0010F7B5FFF73C
:1067100013FF134C2500A835A868E968FEF714F9A3
:106720002E686F680090019130003900FEF70CF977
:1067300006000F00009801990022002307F0AAF933
:1067400032003B0006F080FA2300B0332860696015
:106750000099019A19605A600123A4342370F7BD8F
:10676000C80C001070B5FEF7C9FE104C012803D10B
:1067700002238734237070BD2500A835FFF7DCFEA7
:106780002868696800220A4B07F084F9094B0A4A15
:1067900006F076FD23002860696000200021B033F8
:1067A00018605960A4340123E4E7C046C80C001007
:1067B00000807640FB211940182D4454F0B587B075
:1067C000FEF79CFE334C012804D10223873423704A
:1067D00007B0F0BD2500A835FFF7AEFE2E686F6844
:1067E00030003900FEF7B0F80090019102000B0074
:1067F0003000390007F0C0FB0022274B07F04AF9B0
:106800000022264B07F046F9F9F766FF0022234BDA
:1068100006F036FD23000290039100200021B033E2
:10682000186059600298039907F0EEFE07F022FF06
:106830001B4A1C4B06000F0007F02CF9F9F74CFF20
:10684000320004900591029803993B0007F094FBF5
:106850000022114B07F01EF9134A144B07F01AF9E6
:10686000F9F73AFF02000B000498059906F0ECF9DD
:1068700000220F4B06F004FD00220E4B06F000FD37
:10688000009A019B06F0E0F9A434286069600123B6
:106890009DE7C046C80C00100000594084D79741BE
:1068A0005555555543DEA341E4388EE358314541F3
:1068B00080842E410088C34010B5084C23008633E5
:1068C0001B78002B04D185342278002A01D0237054
:1068D00010BDFFF731FE0123F9E7C046C80C0010D8
:1068E000F0B587B0FFF728FE144D02A82C00A8349D
:1068F000E3680193A368009322686368FCF744FF90
:10690000029E039F26606760049A059BA260E36075
:10691000FEF7F4FD01280BD030003900FEF79EF899
:106920002B002060616000200021B03318605960A6
:106930000123A4352B7007B0F0BDC046C80C001071
:10694000F0B58BB0FFF7F8FDFEF7F4FD204E070021
:106950003500A835A968E8682A686B68019000913D
:1069600006A8FDF73DF8089B099C1A48029303947A
:10697000069A079B184907F0FFFA00220490059138
:1069800002980399002307F085F802000B00049891
:10699000059907F0F1FA340028606960B034002FDF
:1069A0000CD1029A039B0020002107F0E5FA206039
:1069B00061600123A43633700BB0F0BD00220023C8
:1069C00022606360FEF74AF828606960F1E7C0461C
:1069D000C80C0010182D4454FB21F93F70B586B047
:1069E000FFF7AAFDFEF7A6FD124E05003400A834FD
:1069F000E36802A80193A368009322686368FCF728
:106A0000EFFF0298039920606160049A059BA260E1
:106A1000E360002D09D0350000220023B0352A6044
:106A20006B60FEF71BF8206061600123A4363370B1
:106A300006B070BDC80C001070B5FFF77DFD0A4CA4
:106A40002500A835AA68EB6828686968FAF7A4FCED
:106A500023002860696000200021B033186059606D
:106A60000123A434237070BDC80C0010F8B5FEF7E4
:106A700045FD144C002803D0022387342370F8BD51
:106A8000FFF75AFD25002300A835B8331E685F685C
:106A90002868696832003B0007F06EFA00220A4B52
:106AA00006F0F8FF3B00320006F0EAFB2300286006
:106AB000696000200021B03318605960A4340123BC
:106AC000DCE7C046C80C00100000594070B5FEF766
:106AD00015FD114C002803D002238734237070BDAC
:106AE000FFF72AFD25002100A835B8312A686B6818
:106AF0000868496806F0CEFF084B002206F0C0FB8C
:106B000023002860696000200021B03318605960BC
:106B1000A4340123E2E7C046C80C0010000059402D
:106B2000F0B58DB0FFF708FD1D4C2500A835A9680C
:106B3000E8682A686B680190009108A8FCF728FFB4
:106B40000A9A0B9B089E099F164906920793086CA8
:106B50008A6BCB6B496C0090019108A8FCF718FF79
:106B60000A9A0B9B08A804920593089A099B029223
:106B70000393069A079B0092019332003B0005F0B5
:106B800089FD089A099B2A606B600A990B9A230079
:106B9000B03319605A600123A43423700DB0F0BDE6
:106BA000C80C0010D0E8000030B587B0FFF7C4FC77
:106BB0000C4D02A82C00A834E368A4350193A36807
:106BC000009322686368FCF7E3FE029A039B22604D
:106BD0006360049A059BA260E36001232B7007B0F9
:106BE00030BDC046C80C001030B58BB0FFF7A4FC18
:106BF000104C2500A835AA68EB6804920593286814
:106C00006968009201930290039106A82A686B6854
:106C100005F0CCFA069A079B2A606B600899099ADE
:106C20002300B03319605A600123A43423700BB0E1
:106C300030BDC046C80C0010D0B5FEF75FFC134C49
:106C4000002803D0022387342370D0BDFFF774FCE3
:106C50002300B8331E685F682300A8331A685B6896
:106C60003000390007F088F90022094B05F0ECFFED
:106C700002000B0030003900FEF764FA0023002206
:106C8000FEF7ECFAA4340123DEE7C046C80C00107E
:106C90000000F03FF0B591B0FFF74EFC644E3300BA
:106CA0002933FF335C681B680093019400980199B5
:106CB00033003933FF335C681B680293039433005D
:106CC0005933FF335C681B680493059433007933B0
:106CD000FF331A685B6806F0DDFE049A059B04002A
:106CE0000D000298039906F0D5FE02000B0020006B
:106CF000290007F041F933004933FF330A900B9123
:106D00001A685B680098019906F0C4FE029A039B1A
:106D100004000D001000190006F0BCFE02000B007C
:106D20002000290007F028F933006933FF3306906B
:106D300007911A685B680098019906F0ABFE049A07
:106D4000059B04000D001000190006F0A3FE37009B
:106D500002000B002000290007F00EF9A8373B685D
:106D60007C6808930994BA68FB680C900D910898A8
:106D70000999FEF7B9FA2F4B1C6C5D6C9A6CDB6CB1
:106D80000E920F930E9A0F9B20002900FEF78CFAAB
:106D90000C9A0D9B0698079906F07CFEFAF748FAC4
:106DA000340002000B000A980B9906F069FAB83417
:106DB00033002060616000220021C03319605A60F6
:106DC000089A099B0098019906F064FE029A039BB9
:106DD00007F0D2F80A9A0B9B06F05CFE069A079B16
:106DE00004000D000498059906F054FE02000B0003
:106DF0002000290005F028FF069A079B04000D00DB
:106E00000098019906F046FE02000B0020002900C0
:106E100006F036FA33003860796000220021B03382
:106E200019605A6033000122A4331A7011B0F0BD0A
:106E3000C80C001050E80000F0B587B0FFF77CFBED
:106E4000FEF75CFB244C012819D02500A8352E68DC
:106E50006F680022214B3000390005F07FF90028CF
:106E60000DD13900300007F0CFFB07F003FC020022
:106E70000B003000390005F06BF900281DD125000A
:106E8000A835286869680022144B05F0DDFE020071
:106E90000B00E868A9680190009102A8FDF7B8FB13
:106EA000029A039B2A606B60049A059BAA60EB60C0
:106EB0000123A434237007B0F0BD084B002230003A
:106EC0003900FEF73FF923002860696000200021A7
:106ED000B03318605960EBE7C80C00100000F03FB9
:106EE000F0B587B0FFF728FB1A4C2500A835AE682F
:106EF000EF6830002A686B68390002920393FDF74F
:106F000023FD0090019102980399FDF71DFD0022D9
:106F10000490059100980199002306F0BBFD049AA6
:106F2000059B05F091FE02000B000298039907F003
:106F300023F8009A019B2860696025003000390021
:106F400007F01AF80123B035A43428606960237073
:106F500007B0F0BDC80C0010F8B5FEF7CFFA194C19
:106F6000012803D1022387342370F8BD2500A835FA
:106F7000FFF7E2FAA868E9680022134B06F080F9EF
:106F800002000B0005F060FE104A114B06F082FD76
:106F9000002206000F00286869680B4B06F070F9A4
:106FA00002000B0005F050FE094B084A06F072FD86
:106FB0002300B0331E605F6028606960A434012341
:106FC000D2E7C046C80C001000807640182D44540B
:106FD000FB210940F0B585B0FEF790FA3D4C012841
:106FE00004D102238734237005B0F0BDA834FFF725
:106FF000A3FA6568246820002900FDF7A5FC00902D
:10700000019102000B002000290006F0B5FF0022CC
:10701000314B06F03FFD0F00060007F0F5FA0400C3
:1070200007F028FB02000B003000390006F0A4FF37
:107030000022294B06F02EFD0022284B06F02AFDE7
:10704000F9F74AFB0022254B06F01AF90022224BE1
:1070500006000F0005F0A0F8002808D03000390025
:1070600000221D4B06F088FF06000F0001343B2C68
:1070700008DD009801990022194B05F0E5FD00900C
:1070800001913C3C6420604307F0F4FA0022029036
:10709000039100980199134B06F0FCFC02000B00D1
:1070A0000298039905F0D0FD32003B0005F0CCFDBD
:1070B0000C4B002206F0E4F8064D0B4B18605960AB
:1070C0002B0000200021B033186059600123A43543
:1070D0002B7089E7C80C001000004E4080842E41C0
:1070E0000000F03F0088C340700D0010F7B5154C4C
:1070F00023009C331B78DB0603D52B22124BE25472
:10710000F7BD25002600B835A836FFF715FA326816
:1071100073682868696805F097FDB268F3680090A5
:107120000191A868E96805F08FFD06000F0000983E
:1071300001993B003200FEF791F80123A43423703B
:10714000DEE7C046C80C001072070000F0B589B039
:10715000FEF7D4F9394C0590002804D00223873477
:10716000237009B0F0BD26002936FF36FFF7E4F999
:10717000306871680022324B05F066FD0690079179
:107180000B0021002500270002003931F835A8370F
:10719000FF312A636B63086849683A687B6800922C
:1071A000019305F051FD009A019B28646964100069
:1071B000190006F06FFC0B002249020008684968BC
:1071C00005F042FD28656965210023005931B83377
:1071D000FF311A685B68086849680292039305F0FA
:1071E00033FD029A039B286669661000190006F0B9
:1071F00051FC0B00144902000868496805F024FDA1
:10720000029A039B2867696700980199250006F098
:1072100041FC7935FF3502000B002868696805F0EC
:1072200013FD069A079B286069603A607B60B2682C
:10723000F368A434BA60FB60059B91E7C80C0010AA
:107240000000F03F100E0010300E0010F7B5154C86
:1072500023009C331B78DB0603D52D22124BE2540E
:10726000F7BD25002600B835A836FFF765F9326866
:1072700073682868696806F07FFEB268F36800905A
:107280000191A868E96806F077FE06000F000098F3
:1072900001993B003200FDF7E1FF0123A434237084
:1072A000DEE7C046C80C001072070000D0B5184CCD
:1072B0008AB023009C331B78DB0604D52A22154BA9
:1072C000E2540AB0D0BDFFF737F923002100B833EC
:1072D00018001E685F68A8318A68CB68049205931D
:1072E0000A684B68029203938268C36806A80092FA
:1072F000019332003B0004F059FF089A099B06985D
:107300000799FDF7ABFF0123A4342370D9E7C046EA
:10731000C80C001072070000F0B5A1B0FFF70CF91F
:107320007B4D2B002C0084331B78A8345BB2069372
:10733000012B4CD122686368A668E7681000190029
:1073400005F082FC08900991FAF7F4FF32003B0047
:107350000C900D913000390005F076FC0A900B91ED
:10736000FDF7A8F802000B000C980D9905F06CFCD5
:1073700006000F000A980B99FDF756F832003B0003
:1073800005F07EFF0A900B9108980999FBF76AF8BF
:1073900032003B0005F074FF002206000F000A983F
:1073A0000B99002306F076FB02000B003000390039
:1073B00005F04AFC2B00B033206061600A990B9AFB
:1073C00019605A60069BA4352B7021B0F0BD069B56
:1073D00027686668013338D100224E4B18A8049202
:1073E00005930022002302920393A268E3680092AF
:1073F00001933A00330004F0D9FE1A99189A0091CB
:107400001B99199B019118A8FCF7BEF90022424B69
:1074100018A804920593802300221B06029203936E
:107420001A9A1B9B00920193189A199B04F0BEFEB6
:10743000189A199B226063601A991B9A2B00B0332B
:1074400019605A60A4350123BEE7FEF757F80128FA
:107450006ED02B007E331B78002B34D02F4A730064
:107460005B08934208DC01230022009338000023CC
:107470003100FCF707FC08E0294A934213DD3A008B
:1074800033003800310006F077FD2B00A833186078
:107490005960B035002300242B606C6001221C4B26
:1074A000A4331A7091E71CAA31003800FCF7DCFD08
:1074B0001E9A1F9B0221400008400139081A0090C3
:1074C0001C981D99D5E72B007F331B78B03500221F
:1074D000002B1BD0134B3800310005F0D1FE060005
:1074E0000F00FAF7CFF93200069007913B00002019
:1074F0000D4906F041FDFAF7C5F902000B000698A8
:10750000079905F0BDFE20606160C3E7074BE2E725
:10751000C80C00100000F03F0000F0BFFB21E93F65
:10752000FFFFEF7F000069400000E03F0080664001
:107530003A00E568A46833003800310005F084FBA8
:1075400006900791FCF7B6FF220006000F002B0003
:107550002000290005F078FB08900991FAF7EAFE6F
:1075600002000B003000390005F06EFB06000F0032
:10757000FAF7DCFE00229C4B04F0F0FD002800D15D
:10758000F7E006980799FAF7D1FE0A900B91089850
:107590000999FAF7CBFE954A0C900D910A980B9930
:1075A000934B05F06DFE0022002304000D0004F053
:1075B000F3FD00228F4B002800D10BE120002900B1
:1075C00005F042FB07F020F807F054F8A822884B9A
:1075D000D20506000F0006F05DFA02000B000A98C3
:1075E0000B9906F0C9FC802204000D005205824B65
:1075F0003000390006F04EFA02000B00200029008E
:1076000006F0BAFC7D4A04000D007D4B30003900C5
:1076100006F040FA02000B002000290006F0ACFC46
:1076200002000B0006F036FA0C9A0D9B002600278C
:10763000109011911000190006F02CFA002234006D
:107640003D00704B129013910E920F930C920D937C
:107650000A920B9300226B4B2000290005F0F4FAEC
:107660000A9A0B9B04000D0006F014FA00220A90FF
:107670000B91644B2000290005F0E6FA04000D0090
:1076800002000B000A980B9906F004FA0C9A0D9B65
:107690000A900B911098119906F0FCF90E9A0F9B25
:1076A0000C900D911298139906F0F4F902000B005A
:1076B0000E900F910C980D9905F0C6FA0A9A0B9B43
:1076C00005F0DEFD32003B0005F0BEFA0022169008
:1076D00017914C4B2000290005F0B6FA04000D006C
:1076E00002000B000A980B9906F0D4F9002206005C
:1076F0000F00444B2000290005F0A6FA02000B0001
:1077000004000D003000390006F0C4F90C9A0D9BFE
:107710000A900B911098119906F0BCF90E9A0F9BE4
:107720000C900D911298139906F0B4F90C9A0D9BD8
:107730000E900F9106F020FC0A9A0B9B05F0A0FD1D
:1077400002000B00149015911698179905F07CFA19
:1077500002000B0006000F001498159905F090FD2B
:10776000FAF7E4FD284A294B04F00CFD002800D06C
:1077700070E7002200233000390004F0E9FC002803
:107780002DD108980999FAF76DFE32003B0005F0FB
:1077900077FD04000D0006980799FCF745FE3200BE
:1077A0003B0005F06DFD002206000F0000232000C5
:1077B000290006F06FF902000B003000390005F0D7
:1077C00043FA134B1A00B033A832106051601C60AA
:1077D0005D6063E62000290006F0CEFBF2E600249F
:1077E0000C4D00200C49ECE70000D03F182D44540C
:1077F000FB2109400000E03F460B213E6EC04531B1
:1078000063626A3C0000F03F4F64A14091B49F3C2A
:10781000C80C00100000F07F0000F87FF0B5842550
:1078200097B0FEF789FE824B814C5D57A834012D3D
:1078300042D126686768A268E36830003900069282
:107840000793FAF70FFE0890099106980799FCF73D
:10785000EBFD02000B000898099906F01BF908904F
:10786000099130003900FAF765FD06000F0006980F
:107870000799FCF71FFE02000B003000390006F0EC
:1078800009F9002206000F0008980999002306F064
:1078900001F902000B003000390005F0D5F9644B06
:1078A000206061600899099AB03319605A60604B92
:1078B000A4331D7017B0F0BD226863680692079369
:1078C0006B1C5AD106980799E36800220893594B1C
:1078D00005F0BAF9A768089D02000B0001950EA8F3
:1078E0000097FAF7B5FE0E9A0F9B069807990A9231
:1078F0000B93109A119B0C920D9300224D4B06F0A6
:107900003BFB01950B00020000970EA8FAF7A0FEC2
:10791000109A119B0EA8049205930E9A0F9B029247
:1079200003930C9A0D9B009201930A9A0B9B04F00F
:107930003DFC069A079B0E980F9905F085F9089B68
:1079400006000D00109811993A0005F07DF93200FB
:107950002B00019100900EA8FCF71AF80E9A0F9BCD
:10796000226063601099119A314BB03319605A60EC
:1079700001222F4BA4331A709CE7FDF7BFFD2C4D5D
:10798000B035012825D02A4B00267E331B780027EE
:10799000002B08D006980799FCF78CFD20606160E9
:1079A0002E606F60E4E7224B00227F331B78002BB0
:1079B0000DD0214B0698079905F062FC02000B00E0
:1079C00000201E4906F0D8FAF9F75CFFE6E71C4BE9
:1079D000F0E714AB12AAA068E168FAF7F7FD069881
:1079E0000799FCF721FD149A159B06F053F8070040
:1079F0000E00089106980799FCF75CFD129A139BFC
:107A000006F048F8002206900791002338000899F4
:107A100006F040F80B0002000698079906F0ACFA51
:107A200080231B06F618206061602F606E609FE760
:107A3000C80C00100000F03F000069400000E03F6B
:107A400000806640F0B591B0FEF776FD684D2B00E2
:107A50002C0084331B78A8345BB20893012B42D1ED
:107A600026686768A268E3683000390006920793C9
:107A7000FAF760FC0A900B9106980799FCF7D4FC82
:107A800002000B000A980B9906F004F80A900B917B
:107A900030003900FAF7E6FC06000F000698079957
:107AA000FCF708FD02000B003000390005F0F2FF82
:107AB000002206000F000A980B99002305F0EAFF48
:107AC00002000B003000390005F0BEF82B00B03387
:107AD000206061600A990B9A19605A60089BA4356E
:107AE0002B7011B0F0BD636826680693089B0133C4
:107AF00044D1A268E3680892099304920593320086
:107B0000069B0CA802920393089A099B009201938A
:107B10003200069B04F04AFB0C980D990022354B6D
:107B200005F092F80B000E99020000910F990CA835
:107B30000191FAF78DFD0C980D993200069B05F026
:107B400083F8089A099B06000F000E980F9905F01C
:107B50007BF832003B00019100900CA8FBF718FF66
:107B60000C9A0D9B226063600E990F9A2B00B03324
:107B700019605A600122A4352A70B2E72F00FDF780
:107B8000BDFCB037012823D02B007E331B78002B9F
:107B90000ED030000699FCF747FC2060616000239E
:107BA00000243B607C602B000122A4331A7098E70C
:107BB0002B007F331B780022002B07D00E4B3000A8
:107BC000069905F05DFBF9F75DFEE6E70B4BF6E77E
:107BD000E068A1683200069B019000910CA8FCF7B8
:107BE000ABFC0C9A0D9B226063600E9B0F9CD8E748
:107BF000C80C00100000F03F0000694000806640A3
:107C0000D0B5224C8CB023009C331B78DB0604D506
:107C10002F221F4BE2540CB0D0BDFEF78DFC230089
:107C2000A83319685A68069107929E68DF6806981B
:107C300007990022002304F08BFA00280BD00022C1
:107C400000233000390004F083FA002803D0873481
:107C500001232370DFE72300B833186859680496BE
:107C60000597069E079F029603979A68DB68009225
:107C7000019302000B0008A804F00CFD0898099974
:107C80000A9A0B9BFDF7EAFAA434E1E7C80C00104E
:107C90007207000070B58AB0FEF74EFC154C21004B
:107CA000B83188680A684B680090C9680191210062
:107CB000A8310D684E68029503968868C9680490DB
:107CC000059106A8FBF730FF0699079A2300F833C1
:107CD00019605A600899099A9960DA60089A099BB4
:107CE00006980799FDF7BAFA0123A43423700AB065
:107CF00070BDC046C80C001070B58AB0FEF71CFC01
:107D0000134C144925002600086C8A6BCB6B496C18
:107D1000A835009001912868696802900391F836AF
:107D2000A868E9680490059106A8FBF7FDFE069A8D
:107D3000079B08980999326073602A606B60012381
:107D4000A434B060F160A860E96023700AB070BD2F
:107D5000C80C0010D0E8000030B587B0FEF7ECFB8F
:107D60000C4D02A82C00A834E368A4350193A36845
:107D7000009322686368FCF715FC029A039B22605B
:107D80006360049A059BA260E36001232B7007B037
:107D900030BDC046C80C001030B587B0FEF7CCFB34
:107DA0000C4D02A82C00A834E368A4350193A36805
:107DB000009322686368FAF74BFC029A039B2260E7
:107DC0006360049A059BA260E36001232B7007B0F7
:107DD00030BDC046C80C001070B5FEF7DBF8084B8C
:107DE00008491A000C6C4D6C886CC96CA832146080
:107DF00055609060D1600022A4331A7070BDC046F7
:107E0000C80C001050E800001B4B1C491A00293216
:107E1000FF3270B50C6C4D6C886CC96C1460556089
:107E20009060D1601A003932FF3214605560906062
:107E3000D1601A004932FF32146055609060D16001
:107E40001A005932FF32146055609060D1601A00F8
:107E500079336932FF33FF329860D960146055601E
:107E60009060D1601C605D60FEF794F840220021B4
:107E7000034803F0DBFD70BDC80C001050E80000A3
:107E8000700D001082B070B505930492144B6528F4
:107E900008DD0322012487331A70200070BC08BC5F
:107EA00002B0184702019A180932FF32049C059D5E
:107EB00014605560069C079D9460D5600024652879
:107EC000EBD1EB22D200991808684968054A064BA5
:107ED00005F0E0FD04F066FE03F0C0FFDDE7C046FC
:107EE000C80C00100000C0FFFFFFDF4110B50928DB
:107EF0000BD9094BFE2809D1E922D2009B1818683A
:107F0000596806F081FB03F0A5FF10BD03228733FB
:107F10001A700020F9E7C046C80C001010B5030025
:107F20000E280CD90F20FE2B09D1E922044BD200D8
:107F30009B181868596806F067FB03F08BFF10BDAB
:107F4000C80C001010B5682802D8FCF7F7FE10BD69
:107F5000094BFE280AD1E922D2009B1818685968FB
:107F600006F052FB03F076FFC0B2EEE70322873340
:107F70001A700020EBE7C046C80C001010B50300D3
:107F800063280CD96420FE2B09D00130FD2B06D0CC
:107F9000094CFF2B04D0032300208734237010BD2D
:107FA000E923DB00E3181868596806F02DFB03F09D
:107FB00051FF6328EFDCF2E7C80C0010F7B50C00A6
:107FC0000500170002684368100019000092019331
:107FD000FCF7D2FC634A20601300A5331B7806002F
:107FE000012B35D1A6321378BB4200DB7B1E0F2F4D
:107FF00000DD0F27BE4203DA5B429E4200DB9CE0BD
:10800000300006F037FB02000B0000205649FAF75B
:108010006FFC02000B000098019905F031F9012670
:108020002860696028686968FCF7A6FCB04258DBE4
:108030004C4BA5331B78032B00D081E0032E00D0DE
:108040007EE00022494B2A606B602368033375E0B1
:10805000022BD5D0032B5CD1009801990022444B10
:1080600004F09AF8002807D10098019900223F4BAC
:1080700004F07EF8002860D0300006F0FBFA020021
:108080000B0000203849FAF733FC02000B0000987F
:10809000019905F0F5F828606960206803F0DAFEC0
:1080A000032104F041F80E1E1BD02A686B68009271
:1080B00001932368002B15DD080006F0DBFA0200AF
:1080C0000B0000202849FAF713FC009A019B05F0E9
:1080D000E1FC2368286069609B1B01362360002E49
:1080E000A0D1F7BD03277F1A380006F0C3FA0200BB
:1080F0000B0000201C49FAF7FBFB009A019B05F0DE
:10810000C9FC2860696004202368861BDF1B276088
:1081100088E7042BE5D10E20801B06F0ABFA0200A5
:108120000B0000201049FAF7E3FB02000B00009857
:10813000019905F0AFFC2860696000232360D0E757
:10814000701E06F097FA0B00020007490020FAF7AC
:10815000CFFB04F045FD04F061FD236828606960F1
:108160000133EBE7C80C0010000024400000F03F92
:1081700000408F40F0B58BB0FEF7DEF9454C08A803
:1081800023002500A83319685A68089109929A6853
:10819000DB68069207930223A5352E780F2205A9E6
:1081A0002B70FFF70BFF0F2204A906A8FFF706FFAD
:1081B000A6342E70207806F097FA0B00020036499C
:1081C0000020FAF795FB04F00BFD2B78032B03D16D
:1081D0000A22002303F032FD04F020FD089A099BD7
:1081E00004000D0005F056FCF8F776FA22002B008B
:1081F00005F046F8069A079B08900991200029008F
:1082000005F048FCF8F768FA22002B0005F038F872
:1082100006900791059806F02DFA02000B00002049
:108220001D49FAF765FB089A099B05F033FC069B8C
:10823000079C0290039104980093019406F01AFAA7
:1082400002000B0000201449FAF752FB06000F0051
:10825000009801990F4C0022002305F01BFC32000E
:108260003B0005F017FC029A039B250004F0ECFC90
:10827000A83528606960009801993B00250032000C
:1082800005F008FC0123B035A43428606960237030
:108290000BB0F0BDC80C001000002440F0B5384B06
:1082A00089B004930023374E0D00745C02A903903B
:1082B0000B739A4204D01522334904A803F0ABFB98
:1082C0002000FCF7EBFB07002800FCF761FC002F07
:1082D0001ED000281ED12F007619767806AD052213
:1082E0000021280003F0A2FBFE2E17D12749280009
:1082F00003F091FB762C2DD13A00254BB6009E1948
:10830000B36C2449009304AB039803F084FB2CE086
:1083100000282CD06F1EF45D765DDFE7FF2E01D1C3
:108320001D49E4E71D49FD2EE1D0632E0FD923003E
:108330004F3B012B04D92B2C02D0A31F012B06D8B5
:1083400032001149233A280003F065FBD2E73200DE
:108350001349F8E7134BA400E358019500933A0042
:1083600004AB1149039803F056FB09B0F0BD0D4B67
:10837000A400E3582A0000930C4904ABC4E7C046AC
:1083800020200000F804001071F200003DF200000F
:10839000D0E800008DF1000080F1000084F10000C1
:1083A0008AF10000F0EB000096F10000A1F100005E
:1083B000F0B597B0019010000892099316001C00C8
:1083C0005A0043420343CF495208DB0F1343CB1AF1
:1083D000CD490BD4CD4BDA420DD42100002200232D
:1083E00003F0D0FECA49002800D1CA49019803F021
:1083F00012FB17B0F0BD00220023210003F0AEFEF7
:10840000002800D115E1C44BA5331878089604382C
:108410000300581E8341059380231B06E4181C9B10
:108420000994013B1C931C9A0BA908A8FFF7C6FDF1
:10843000089B099C180021000293039404F0D0FBD0
:1084400004000D000E900F9104F0E8FB0F000600F1
:10845000FCF792FA03000133049000933200029873
:1084600003993B0005F088FD2C43069007910F27E8
:10847000002C00D11027009BFF1A380006F0FAF8F4
:1084800002000B000020A549FAF732FA02000B00A7
:10849000029003910698079905F0FCFAF8F71CF989
:1084A00004F09EFB04000D0004F0B8FB029A039B4D
:1084B00003F072FE002800D0BDE00C940D950B9ED9
:1084C000002E07D0300006F0D5F8FCF755FAF60F6D
:1084D00036180236904B1A00A533A63214781B7852
:1084E0002200032B03D1009BE21A9C4200DB0F24E5
:1084F000002F00D1CBE03B00974200DD13001C9A17
:10850000961B009AB11A1A008B4200DD0A00D5436F
:10851000ED171540AF4200DCC0E07A1B39000CA813
:10852000FCF752FE002827D0002200230120002162
:108530000C920D930E9A0F9B801859410E900F913B
:1085400004F06CFBFCF718FA009B984214DB0B9BC1
:10855000002B00D19EE0009B581E06F08BF80B000C
:1085600002006E490020FAF7C3F904F039FB0B9BB7
:108570000E900F9101330B93002E00DC0126009B1F
:10858000B34200DC8CE09E1B320019000EA8FCF701
:108590001BFE002809D00E980F990B2364220B9321
:1085A000002303F04BFB0E900F910B9B9E190B9633
:1085B0001422002111A803F039FA2A00584911A801
:1085C00003F029FA059B012B08D1019803F066FA04
:1085D000019B2D221818534903F01DFA019803F04E
:1085E0005DFA019B504918180E9A0F9B03F013FA7D
:1085F000002D00DC9AE0019803F050FA019B11A9CC
:1086000018180C9A0D9B03F006FA0B9B002B00D157
:10861000EFE6414B0198A5331B78042B00D092E084
:1086200003F03CFA2E22019B3E49181803F0F3F99F
:10863000DFE60590F7E600220023012000210C92DE
:108640000D930E9B0F9CC01861410E900F9104F08A
:10865000E5FAFCF791F9009B984200DA2FE70B9BB3
:10866000002B10D0049806F005F80B0002002B49EF
:108670000020FAF73DF904F0B3FA0B9B0E900F912E
:1086800001330B931BE7049B0233009317E701238D
:108690005B4234E7009B013300936DE71D006BE7FD
:1086A000009BA34284DD1C1B200005F0E3FF0200B9
:1086B0000B0000201949FAF71BF9009B06000F0078
:1086C0002200022B10DC19000EA8FCF77DFD0E988D
:1086D0000F9904F0A3FA32003B0005F0DBF904F037
:1086E0007FFA0E900F9163E700990EA8FCF76CFDDE
:1086F0000028ECD0002301220E920F930B9B033332
:108700000B9355E70000F07FA9F1000000001080F6
:10871000AEF10000ADF10000C80C001000002440D4
:10872000B2F1000071F20000BCF10000002D00D099
:108730006BE7019803F0B2F9019B2E221818054946
:1087400003F069F961E703F0A9F9019B0B9A181886
:1087500001496BE771F20000C1F1000082B0F0B591
:1087600093B019931C9B1892023BDA0FD3185B103D
:108770000390162200210CA8029303F057F9162249
:10878000002106A803F052F91A9C1B9D404E3300AD
:1087900080331B78002B5DD01898199922002B008C
:1087A000F8F7FAFD189A199B04900591200029000A
:1087B000FAF738FF33007E367F331A7833780400B7
:1087C0000D00134338D10022324B05F063F9324AD1
:1087D000324B04F055FD1E2604000D00029B0CA830
:1087E0000093049A059BFFF7E3FD0CA803F056F9EC
:1087F000029B984206D20CA803F050F9029B5B0042
:108800001B1A0293029B06AF009322002B00380034
:10881000FFF7CEFD1E4B1A00A5321278042A1FD195
:1088200033001F4900970CAA039803F0F4F813B023
:10883000F0BC08BC02B018471E26002ACED0002289
:10884000184B05F027F9144A144B04F019FD0400E5
:108850000D00C3E7189A199B692604920593BDE79A
:1088600080331B78002B04D0009733000CAA0E49EC
:10887000DAE7002200232900200003F083FC0096A1
:108880003B000CAA09490028CED10949CCE7C046D3
:10889000C80C001000807640182D4454FB2119406C
:1088A000C6F1000000007940CDF10000D6F10000D3
:1088B000E0F1000070B50F4C0F2223000E4E78330C
:1088C0001A7030000532002103F0B0F823000025B3
:1088D0009C330A4A1D700A4B0C320A493000E55499
:1088E00003F099F823008334A0331D602570FDF751
:1088F00051FB70BDC80C0010500D0010000000109E
:10890000720700009EF10000F7B5384C23009C333D
:108910001D78002D56D03648364D030064331B7841
:10892000002B0FD12300A0331B68AB4202D0324A88
:1089300093421DD1314BE35C002B19D16430304997
:1089400003F069F82300A0331A68AA4222D12B4A07
:10895000A25C2B2A12D12B4A1A602300A0331B6879
:10896000873498472378002B29D0FDF713FB04E0C8
:10897000230083331B78002BE4D1F7BD2D2A01D1CE
:10898000214AE9E72A2A01D1204AE5E72F2AE4D142
:108990001F4AE1E718498A42DFD1184AA25C2B2A14
:1089A00001D11C4AD8E72D2A01D11B4AD4E72A2A33
:1089B00001D11A4AD0E72F2ACFD1194ACCE7FFF7C5
:1089C00079FFDAE7FDF7F2FA2300A8331E685F6843
:1089D0009A68DB6800920193009A019B300039008D
:1089E000A434FCF761FC2570C7E7C046C80C001032
:1089F00048040010A18F00003D90000072070000A5
:108A0000E9F1000091910000ED9100004992000011
:108A1000AD9200001193000059930000A193000053
:108A2000F5930000F0B56D4C91B023009C331B789A
:108A30005B070BD56A4B64331B7E002B02D14920A8
:108A4000FCF7E8FEFFF760FF11B0F0BDFDF7AEFAEE
:108A5000FCF754FD012835D12500A835AA68EB683C
:108A600006920793230080331B78B034002600273A
:108A7000002B22D02A686B680892099308980999FC
:108A8000069A079BF8F788FC089A099B0A900B91B5
:108A900006980799FAF7C6FD0A9A0B9B266067604D
:108AA0002A606B60FBF7DAFF32003B00FCF7FCFB4F
:108AB00001224A4BA4331A70C6E726606760069805
:108AC0000799F1E7022802D187342070BCE7220021
:108AD000B832106851689568D66822002300089063
:108AE00009910695079680321278A833186859685C
:108AF00000260027002A4CD023007E331B78002B51
:108B00000FD17F3423780022002B40D0354B04F066
:108B1000B7FB02000B0004F097F8334A334B04F024
:108B2000B9FF2E4B324C1A00B0331E605F60002339
:108B3000A832106051600493059402000B000CA849
:108B4000029603970096019703F030FB0E990C9A5A
:108B500000910F990D9B01910CA8FBF723FD0E9B33
:108B60000F9C0CA8049305940C9B0D9C02930394FA
:108B7000069B079C00930194089A099B03F016FB3F
:108B80000C980D990E9A0F9BFCF768FB90E7194B18
:108B9000BDE70024164D0296039704940595020044
:108BA000DC689B680CA8009301940B0003F0FEFAAC
:108BB000089A099B0C980D9904F046F8069A079BB1
:108BC00004000D000E980F9904F03EF806000F0007
:108BD0002000290032003B00D6E7C046C80C001038
:108BE0004804001000007940182D4454FB2109402E
:108BF0000000F03F008076401FB5124C23009C33EC
:108C00001B789B070AD510486430037E002B02D1E5
:108C10000E4902F000FFFFF777FE1FBDFDF78CFC49
:108C200023008021A8339A6809060292DA68A434E6
:108C3000521803920299039A9960DA600123237013
:108C4000EBE7C046C80C00104804001080F100009B
:108C5000F7B56B4C260083363378002B16D02300F3
:108C600085331B78002B10D0664D6435280002F048
:108C700015FF012804D12800FCF7B2FC0130307048
:108C8000833421787620FCF731F8F7BD2300863352
:108C90001B78002B00D19AE0FDF788F923007C3384
:108CA0001A88594B9B185D78FCF728FC002809D0DE
:108CB0000C2D03D8554BEB40DB0703D4022387343C
:108CC0002370E2E72300A8331E685F682300681E54
:108CD000B8331A685B68009201930B2819D803F027
:108CE00033F9061B262D343B4E5D60636669210017
:108CF000A83100228868C968002303F029FA0028F7
:108D000012D0002200233000390003F021FA00289D
:108D10000AD0FBF7A5FF07E000220023300039004E
:108D200003F030FA0028F4D0A4340123C8E700226D
:108D300000233000390003F011FAF3E7002200238A
:108D40003000390003F028FAECE70022002330005D
:108D5000390003F00DFAE5E721002300A831B8330C
:108D60009A68DB688868C96803F0F2F90028D0D0F7
:108D7000009A019B3000390003F0EAF9D2E72100A4
:108D80002300A831B8339A68DB688868C96803F0A3
:108D9000DFF90028C8D0009A019BB4E7009A019B34
:108DA000BCE7009A019BC4E7009A019BC8E7009AC0
:108DB000019BCCE72100A83100228868C968002304
:108DC00003F0C6F90028A4D000220023D2E7230034
:108DD00085331B78002B00D157E7FFF76BFD22008E
:108DE00020219C321170220001230949A032116018
:108DF0007834084908483370237002F00CFE44E7C9
:108E0000C80C001048040010F8040010C210000044
:108E1000518C0000EDF10000500D001070B51B4E9C
:108E200033009C331B785B060AD519486430037EF7
:108E3000002B02D1174902F0EEFDFFF765FD70BD72
:108E40003400A834FDF7B2F8A268E36820686168CE
:108E5000FCF74AFA03F00CF8EB23DB00F51805F0F9
:108E600009FC0D4A0D4B04F00BFAEC23DB002860E3
:108E700069600022F51800232A606B60A260E3603D
:108E80000123A436206061603370D8E7C80C00105D
:108E900048040010E9F100000000C0FFFFFFDF41BF
:108EA00010B5284C28496434200002F009FE00283F
:108EB00002D1FDF76FF810BD200002F0EFFD002891
:108EC0000FD0200002F0EAFD0023201801380370C3
:108ED000200002F0E3FD0028EDD11C4BA4331870F4
:108EE000E9E71A4B1A009C321278002A02D0FFF7E9
:108EF000E1FCE0E71A0085321278002A1AD07C33B0
:108F00001C88002CD7D0124B185DFBF7C7FD00283A
:108F100002D0A01C022107E02000FBF739FE01214E
:108F20000300601C002BF5D14942FBF7FBFDFBF76A
:108F30005BFEC0E7200002F0B1FD0028BBD1FEF7C8
:108F40004BFFB8E74804001080F10000C80C001087
:108F5000F804001010B50F4CFE2064342378492B20
:108F600013D00D49200002F0ABFD0300FF20002BC1
:108F70000BD00A49200002F0A3FD0300FD20002BC6
:108F800003D02078402801D9233010BD2000FCF701
:108F900027FBFAE74804001080F10000E9F1000027
:108FA00037B5214C25009C352B78002B0CD0FFF7D2
:108FB000D1FF230085331B78C0B2002B11D00100F4
:108FC0000D20FBF793FE37BD230086331B78002B63
:108FD00017D0FCF7EBFF23007C331A88134B9B1848
:108FE0005878FEF7CBFF2100A8318D684B680A68DE
:108FF0000095C968A4340191FEF744FF0123237052
:10900000E1E7FCF7D3FFFFF755FC56232B70230055
:10901000074AA0331A6002237834064906482370B1
:1090200002F0F9FCCFE7C046C80C0010F8040010AD
:10903000A18F0000F3F10000500D001030B5314C4D
:1090400085B025009C352B78002B26D0FFF782FFBA
:10905000230085331B78C5B2002B05D029001120D1
:10906000FBF744FE05B030BD274B196C5A6C0091DC
:1090700001929A6CDB6C0098019902920393029A18
:10908000039BFCF731F92800FEF778FF1F49FBF737
:1090900043FC0123A4342370E4E7230086331B78C8
:1090A000002B1CD0FCF782FF23007C331A88184B5E
:1090B0009B185878FEF762FF0500134B196C5A6C29
:1090C000009101929A6CDB6C0098019902920393D3
:1090D000029A039BFCF708F90C492800D7E7FCF734
:1090E00065FFFFF7E7FB56232B702300094AA033E7
:1090F0001A600223783408490848237002F08BFC78
:10910000B0E7C046C80C001050E80000700D001019
:10911000F80400103D900000F7F10000500D001021
:1091200070B5174C01222300A4331A702300863334
:109130001B780500002B0ED07C34FCF737FF22880B
:10914000104B9B185878FEF719FF04000E492000B9
:10915000FBF7E2FB10E023009C331B78002B0DD0C3
:10916000FFF7F8FE85342378C0B2002BEBD0010066
:109170002800FBF7BBFD054C200070BD034CE5E764
:10918000C80C0010F8040010C00D0010FFFFFF7F96
:10919000F0B5792085B0FFF7C3FF0700642820DC15
:1091A000114C2600A834F83622686368306871686C
:1091B00003F04AFDA268E36805000391B068F16816
:1091C00003F042FD2A00039B3260736002000B0033
:1091D000B260F36000902A00039B01913800FEF713
:1091E00051FE05B0F0BDC046C80C0010F0B57A20A5
:1091F00085B0FFF795FF0700642820DC114C26009E
:10920000A834F836226863683068716804F0B4FEE8
:10921000A268E36805000391B068F16804F0ACFE51
:109220002A00039B3260736002000B00B260F3609F
:1092300000902A00039B01913800FEF723FE05B041
:10924000F0BDC046C80C001030B57B208BB0FFF7D6
:1092500067FF0500642825DC134B06A81C00A83313
:109260009968DA68049105921A685B680292039320
:10927000F834A268E368009201932268636802F000
:1092800095FF069A079B22606360089A099BA2607B
:10929000E360099808990190069A079B00912800BD
:1092A000FEF7F0FD0BB030BDC80C001030B57C20CF
:1092B0008BB0FFF735FF0500642825DC134B06A8AB
:1092C0001C00A8339968DA68049105921A685B68F3
:1092D00002920393F834A268E36800920193226833
:1092E000636803F0D7F9069A079B22606360089AC7
:1092F000099BA260E360099808990190069A079B70
:1093000000912800FEF7BEFD0BB030BDC80C001068
:1093100073B57D20FFF704FF642819DC0D4C250090
:109320002600A835F836B268F368A868E96803F043
:109330008BFC32687368009001912868696803F0BB
:1093400083FC009A019BB0342860696022606360EE
:1093500073BDC046C80C001073B57E20FFF7E0FE59
:10936000642819DC0D4C25002600A835F836B268B3
:10937000F368A868E96804F0FFFD3268736800903C
:1093800001912868696804F0F7FD009A019BB034E8
:10939000286069602260636073BDC046C80C00101D
:1093A00030B57F208BB0FFF7BBFE64281EDC104C6D
:1093B00006A823002500F8339968DA68049105921D
:1093C0001A685B6802920393A835AA68EB6800925A
:1093D00001932A686B6802F0E9FE069A079BB03495
:1093E0002A606B60089A099B226063600BB030BDF5
:1093F000C80C001030B580208BB0FFF791FE6428B8
:109400001EDC104C06A823002500F8339968DA68A2
:10941000049105921A685B6802920393A835AA68C2
:10942000EB68009201932A686B6803F033F9069A9F
:10943000079BB0342A606B60089A099B22606360C6
:109440000BB030BDC80C001070B5FCF7AFFD1E4C62
:1094500025009C352B78002B0AD08534FFF77AFD48
:109460002378002B03D0C1B27320FBF73FFC70BD03
:10947000230086331B78002B16D023007C331A88F8
:10948000124B9B185878FEF731FD230087331B7869
:10949000002BECD1ED232418DB00E4182378002BFB
:1094A000E5D1FBF7DDFBE2E7FFF704FA05232B70BC
:1094B0002300074AA0331A6001237834054906487F
:1094C000237002F0A8FAD2E7C80C0010F8040010CC
:1094D00049940000FBF10000500D001070B5FCF73E
:1094E00065FD234C25009C352B78002B17D0FFF70A
:1094F00031FD230085331D78C0B2002D04D001005A
:109500006F20FBF7F3FB70BDFEF7F0FCED23201896
:10951000DB00C01805700123A4342370F3E7230097
:1095200086331B78002B12D023007C331A88114B12
:109530009B185878FEF7DAFC230087331B78002B42
:10954000E1D1ED222018D20080180370E3E7FFF785
:10955000B1F905232B702300074AA0331A600123B9
:10956000783406490648237002F055FACBE7C04626
:10957000C80C0010F8040010DD94000007F2000091
:10958000500D001070B5FCF711FD204C25009C35E6
:109590002B78002B17D0FFF7DDFC230085331B78D9
:1095A000C0B2002B04D001006B20FBF79FFB70BD05
:1095B000FEF79CFCED232018DB00C0180123A43427
:1095C00003702370F3E7230086331B78002B0DD044
:1095D00023007C331A880E4B9B185878FEF786FCC4
:1095E000230087331B78002BE1D1E3E7FFF762F913
:1095F00005232B702300074AA0331A600123783417
:1096000005490648237002F006FAD0E7C80C00109E
:10961000F80400108595000013F20000500D0010B2
:10962000F8B5FCF7C3FC1D4C25009C352B78002BAE
:1096300023D0FFF78FFCC0B2FBF780FB184B98429A
:1096400017DC0222012103009446164F091AFA2260
:10965000CD18D200934206D0FA5C562A03D0664653
:109660000133B243F3D102214942491B4019FBF7B0
:1096700059FA00237C342380F8BDFFF71BF9082337
:109680002B702300084AA0331A600223783407495C
:109690000748237002F0BFF9EEE7C046C80C00107F
:1096A000CF070000F8040010219600001DF2000012
:1096B000500D0010F0B5334C89B025009C352B7847
:1096C000002B0BD08534FFF745FC2378002B03D00B
:1096D000C1B24B20FBF70AFB09B0F0BD2300863373
:1096E0001B78002B3CD0FCF761FC23007C331A88EC
:1096F000254B9B185878FEF741FC05002D01651994
:109700002F00224E09373100FBF706F930687168E7
:1097100007AB009305AA06ABFBF7C8F8059A079BB1
:10972000FF379E180798BA68FB6805960292039364
:1097300004F0A0FF02000B003868796803F084FA97
:10974000029A039BF835AA61EB61069B2861696167
:109750009E4201DDFBF784FA0123A4342370BBE7AA
:10976000FCF724FCFFF7A6F807232B702300084A18
:10977000A0331A600223783406490748237002F0A8
:109780004AF9A9E7C80C0010F8040010C00D001039
:10979000B59600002AF20000500D0010F0B5334CD1
:1097A00089B025009C352B78002B0BD08534FFF732
:1097B000D1FB2378002B03D0C1B24720FBF796FAE8
:1097C00009B0F0BD230086331B78002B3CD0FCF79A
:1097D000EDFB23007C331A88254B9B185878FEF745
:1097E000CDFB05002D0165192F00224E09373100F0
:1097F000FBF792F83068716807AB009305AA06ABD7
:10980000FBF754F8059B079AFF379E1A0798BA682A
:10981000FB6805960292039304F02CFF02000B00F4
:109820003868796804F0A8FB029A039BF835AA61AE
:10983000EB61069B286169619E4201DCFBF710FA2F
:109840000123A4342370BBE7FCF7B0FBFFF732F829
:1098500007232B702300084AA0331A6002237834B0
:1098600006490748237002F0D6F8A9E7C80C001093
:10987000F8040010C00D00109D9700002EF20000AB
:10988000500D001073B5284C25009C352B78002B0B
:109890000CD0FFF75FFB230085331B78C0B2002B91
:1098A00011D001004320FBF721FA73BD230086335A
:1098B0001B78002B25D0FCF779FB23007C331A881A
:1098C0001A4B9B185878FEF759FB2500210006001B
:1098D000F835A8310A684B682A606B608A68CB68E3
:1098E000AA60EB60FBF718F8A9686B682A6800911A
:1098F000E96830000191FEF7C5FA0123A434237012
:10990000D3E7FCF753FBFEF7D5FF07232B702300AB
:10991000074AA0331A6002237834064906482370A8
:1099200002F079F8C1E7C046C80C0010F804001036
:109930008598000032F20000500D001070B51F4CE9
:1099400025009C352B78002B12D0FFF703FB23005A
:1099500085331B78C0B2002B15D001004C20FBF7DB
:10996000C5F970BD01221A700323A5342370F8E7EE
:10997000230086331B78002B0DD023007C331A88FC
:109980000F4B9B185878FEF7C9FA2300A63300281E
:10999000E8DD1870E8E7FCF709FBFEF78BFF230012
:1099A00002227833074908481A7002F034F8074B4E
:1099B000A034236005232B70D3E7C046C80C0010E9
:1099C000F804001037F20000500D00103D9900001F
:1099D00070B51C4C25009C352B78002B0CD0FFF764
:1099E000B9FA230085331B78C0B2002B0FD00100D9
:1099F0004820FBF77BF970BD230086331B78002BD2
:109A00000ED023007C331A880F4B9B185878FEF732
:109A100085FA2300A63318700223A5342370EAE7E1
:109A2000FCF7C4FAFEF746FF230002227833074909
:109A300007481A7001F0EFFF064BA034236005239E
:109A40002B70D8E7C80C0010F80400103BF200009F
:109A5000500D0010D199000070B51C4C25009C35AC
:109A60002B78002B0CD0FFF775FA230085331B7879
:109A7000C0B2002B0FD001004420FBF737F970BDB6
:109A8000230086331B78002B0ED023007C331A88EA
:109A90000F4B9B185878FEF741FA2300A633187035
:109AA0000123A5342370EAE7FCF780FAFEF702FFF2
:109AB000230002227833074907481A7001F0ABFFF0
:109AC000064BA034236005232B70D8E7C80C001088
:109AD000F80400103FF20000500D0010599A0000E9
:109AE00070B5114C114E2500A0352B68B3420DD135
:109AF000FFF730FAC0B2FBF737F9002803D104238F
:109B00008734237001E07C34208070BDFEF7D2FEE4
:109B1000230002227833064906481A709C3401F06B
:109B20007AFF2E600923ECE7C80C0010E19A0000D0
:109B300043F20000500D001070B5FCF737FA244CCA
:109B400025009C352B78002B0AD085342378002BF8
:109B500005D0FFF7FFF9C1B20720FBF7C7F870BDCA
:109B6000230086331B78002B19D023000122250007
:109B7000A4331A707C352A88164B9B185878FBF74B
:109B8000F3F8002807D12300042287331A70012339
:109B9000A4342370E3E72880FBF726F8F7E72300D7
:109BA00085331B78002B0FD0FEF784FE0C232B701F
:109BB0002300094AA0331A60022378340749084871
:109BC000237001F028FFCAE7FFF78AFFC7E7C04606
:109BD000C80C0010F8040010399B00004EF2000081
:109BE000500D001070B5184C184E2500A0352B688C
:109BF000B34213D1FFF7AEF9061E00D10136FAF7D2
:109C000079FF0500B04200DD35002800FAF7C0FFFB
:109C1000431E98417C342D18258070BDFEF74AFE06
:109C2000FAF768FF04F026FDFAF7A6FE23000130DC
:109C3000783318700649074801F0EDFE01239C3483
:109C40002E602370E9E7C046C80C0010E59B0000B9
:109C500057F20000500D0010F7B52F4C2200833250
:109C60001378002B06D00C2B02D10B3B1370F7BDE1
:109C70000133FBE7294D64352B7E002B17D06E7E18
:109C8000A97E744274410C40E97E701C2818AB19FF
:109C9000AA7D0C4304D00100180001F0EAFEE6E7BB
:109CA000190001F0E6FE2D236C75AB55DFE72300AC
:109CB0000122A4331A702300A8331A685E68019247
:109CC0009F68DD68002200230198310002F040FA0D
:109CD000002802D180231B06F6180022002338003A
:109CE000290002F035FA002802D180231B06ED1866
:109CF000002200233800290003F0CCFE019A330033
:109D000002F0A2FF064B3A00186059602B00B034F5
:109D100022606360ABE7C046C80C00104804001026
:109D2000700D0010F0B5504D89B0280001F0B6FE5E
:109D30004E4E009028220021300001F077FE4C4F5B
:109D40004C4CE35D002B0FD0280001F0A7FE20183B
:109D5000873003782B2B39D1280001F09FFE444B2C
:109D60002018E35C87300370230083331B78424F55
:109D7000002B4AD0414A9B00D3189A6C390002A8A4
:109D800001F049FE23009C331B78DB0603D53C49D8
:109D9000300002F087F802A9300002F083F82300B7
:109DA0009C331B78002B55D02200A032354B126813
:109DB00000259A4208D0344F6437230078331B784B
:109DC000BA7D9B1AAB423FDC09B0F0BD280001F020
:109DD00065FE2018873003782D2BBDD0280001F0B8
:109DE0005DFE2018873003782A2BB5D0280001F0BB
:109DF00055FE2018873003782F2BADD0280001F0B6
:109E00004DFE20188830E35DADE71222009BD31A87
:109E10001D4A019364320092937D019A93420CDDB6
:109E20001A4A1B490F32300001F0F5FD009B9A7D64
:109E3000019BD21A009B9A18A0E72A003900300033
:109E400001F0E9FD009A99E71249300002F02AF882
:109E50000135B2E70C4B64339B7D0E2BB4D80D4912
:109E6000300002F01FF8AFE7500D0010F00C0010AA
:109E700072070000C80C00109EF10000D0E800003E
:109E800000F30000518C0000480400100000001096
:109E900063F2000067F20000F0B5C54E89B02822D9
:109EA0000021300001F0C2FDC24D2822002128000F
:109EB00001F0BCFDC04C14220021200001F0B6FDD1
:109EC00014220021BD4801F0B1FD330085331B7819
:109ED000002B05D1330079331B78002B00D1D3E060
:109EE00033007C331988002904D001390022300066
:109EF000FEF7D4F937007C37012239882800FEF7B5
:109F0000CDF93888FAF756FE0200692807DCAC491B
:109F1000632801DDAB49233A200001F07CFD9C362B
:109F20003378002B01D0FFF7FDFEA14C23008733CF
:109F30001B78002B32D0012B03D1A349200001F064
:109F40006AFD230087331B78022B03D19F49200031
:109F500001F061FD230087331B78042B03D19C495A
:109F6000200001F058FD230087331B78052B03D117
:109F70009849200001F04FFD230087331B78032B05
:109F800003D19549200001F046FD230087331B785B
:109F9000062B03D19149200001F03DFD23007A33C7
:109FA0001B78002B03D08E49200001F034FD2300E4
:109FB00086331B78002B14D12300A5331B78042B88
:109FC0000FD0230084331B7886495BB2012B00D16C
:109FD000E6E0013300D0D6E01D228349774801F046
:109FE0001AFD230085331B78734D002B27D12300E6
:109FF000A5331B78042B22D023007E331B78002B43
:10A0000003D07A49280001F04DFF23007F331B78ED
:10A01000002B03D07649280001F044FF754BE35C28
:10A02000002B03D07449654801F03CFF23008033C6
:10A030001B78002B03D07149280001F033FFFBF798
:10A04000EDFE20000021FBF785FC08215948FBF7B5
:10A0500081FC002383211A0028008334FBF790FA47
:10A060002378002B00D19FE0012308226821644857
:10A07000FBF786FA0123082252216248FBF780FA97
:10A08000FAF759FF09B0F0BD330086331B78002B77
:10A090000FD033007C331B885B4AD35C2A2B08D05B
:10A0A0005A49300001F0B7FC5949280001F0B3FCCF
:10A0B0003BE73300A53357481B780C30042B50D1B5
:10A0C00001F0ECFC16245449241A300001F0A3FCE2
:10A0D000384F5249380001F09EFC300001F0DEFCA0
:10A0E0003300B8331A68351805929E685A68DB68E1
:10A0F00006920793002200233000079902F028F807
:10A10000002832D10799059A069B02940191009686
:10A110002800FEF723FB380001F0C0FC244B3F1859
:10A12000A8331A689D68DE6805925A68280006926E
:10A1300000230022310002F00BF800281CD1059A00
:10A14000069B0294019600953800FEF707FB344BFE
:10A1500064331B7E002B00D0E5E6154B9C331B7847
:10A16000DFE601F09BFC1224ADE70094059A069B04
:10A170002800FEF71DF9CEE70094059A069B3800EB
:10A18000FEF716F9E3E7230082331B782549002BFD
:10A1900006D1230081331B78002B00D121E722490F
:10A1A000064801F07FFE1CE708228321034865E78B
:10A1B000C80C0010F00C0010180D00102C0D001031
:10A1C00074F2000069F2000093F200009FF20000B8
:10A1D000ACF20000B5F20000C2F20000CDF20000C7
:10A1E000DFF20000E5F20000E7F20000EDF200000F
:10A1F000F1F2000074070000F4F20000F7F2000032
:10A20000FAF20000FEF20000F80400107FF20000F5
:10A2100087F20000000000108DF2000090F20000B4
:10A220004804001085F20000EBF20000F0B5A34BEB
:10A2300085B0984200DDC4E0EF23002874D10122EC
:10A2400086247C209E4D9F4E6F6901956D69DB00D1
:10A250000297F55032553252002904D19A4BF35CE3
:10A26000002B00D1C9E00124984B00935D780027B2
:10A2700002E00137A74207D0E31B009A013BD05C04
:10A28000FAF70CFC0028F4D1FB0700D5BAE0904B9C
:10A29000904F0393002D00D1ECE02B2D00D188E0EE
:10A2A000802D69D8AD00EB59002B65D09847019BF4
:10A2B000029A5B699B1A632B00D972E08623F35CD8
:10A2C000002B00D1ECE08723F35C002B54D17C33CE
:10A2D000F45A009B08211A5D1300473B8B43DBB205
:10A2E000012B3CD9130004206F3B8343DBB2002BCE
:10A2F00035D01300763B0A2B31D9402315009D43FE
:10A300002B2D2CD0931F012B29D9073B8343DBB284
:10A31000002B24D08A43433A012A20D96E4B9C4219
:10A3200027D87C2301341FE07C2786220125644C3A
:10A33000644E019484B20198F453B554476942695C
:10A34000DB000297F250002903D15F4BF35C002B36
:10A3500053D05E4B00931D5D002C88D197E75F4B77
:10A360009C4206D87C230234A4B2F452009B1D5DAB
:10A3700090E787230322F254EF2300229C218620BA
:10A380000124DB00715CF2503254002906D1019D9A
:10A390006435280001F082FB00281FD1200005B0A1
:10A3A000F0BDFAF7EBFF0028E6D1019B5B69029351
:10A3B00084E74A4B9C420AD987230322F254039B29
:10A3C00074E7872203213F4B01249954E6E77C235D
:10A3D0000234009AA4B2155DF45261E72800FBF73D
:10A3E00041F93300A8331860596000220023B036C9
:10A3F00032607360FBF7CEFDD0E7FFF74DFD7C23A5
:10A40000F45AA6E72B000822473B9343DBB2012B0B
:10A4100022D92B0004216F3B8B43DBB2002B1BD0D6
:10A420002B00763B0A2B17D94023280098432B2872
:10A4300012D0AB1F012B0FD9073B8B43DBB2002B94
:10A440000AD02B009343433B012B05D9224B9C425E
:10A450000CD87C23013404E0204B9C4206D87C239A
:10A460000234A4B2F452009B1D5D10E7872303223F
:10A47000F2540CE7012C0ED9671E02E00135BD42F3
:10A4800007D0631B009A023BD05CFAF707FB002859
:10A49000F4D1EB070ED4002C02D07C23013CF45203
:10A4A000EF2300229C218620DB00715C0024F25007
:10A4B00032546AE77C23023CF452F1E7CF070000F4
:10A4C00048040010C80C001073070000F8040010C6
:10A4D000E1A40000F4ED0000CE070000CD0700006D
:10A4E000F8B5244C25009C352B78002B25D0FEF7A1
:10A4F00031FDC5B22800FDF725FD230085331F7807
:10A500000600002F0AD0002803D0052387342370CB
:10A5100003E029002B20FAF7E9FBF8BD002809D059
:10A52000FEF7C8F90123A434390030002370FFF787
:10A530007DFEF2E787340423E9E7230086331B78A6
:10A54000002BEAD1FBF732FDFEF7B4F908232B709C
:10A550002300094AA0331A602300022278331A70BC
:10A560008534237805480649002B00D1054901F0C0
:10A5700052FAD2E7C80C0010E1A40000500D001000
:10A5800002F300000CF3000070B5184D2B009C3353
:10A590001B781A0709D5164B64331B7E002B03D199
:10A5A000FBF738F9FEF7B0F970BD002BFCD12B009A
:10A5B00085331E782330C4B2002E04D0210007203A
:10A5C000FAF794FBF0E7FBF7F1FC2B000122A43330
:10A5D00020001A70FDF7B6FC002803D03100FFF709
:10A5E00025FEE1E7042287352A70DDE7C80C00105C
:10A5F0004804001010B54520FFF7C6FF10BD10B588
:10A600004420FFF7C1FF10BD10B54320FFF7BCFF8A
:10A6100010BD10B54220FFF7B7FF10BD10B54120A7
:10A62000FFF7B2FF10BDF7B5FBF7C0FC264C2500C5
:10A630009C352F78002F0AD085342378002B05D045
:10A64000FEF788FCC1B20620FAF750FBF7BD2600E2
:10A6500086363378002B1ED025007C352A881B4B8C
:10A660009B185878FDF76EFC002803D1042387342B
:10A670002370EBE72B883900019323000124A433D6
:10A680001C70FFF7D3FD002801D03770DEE7019B77
:10A6900034702B80DAE7230085331B78002B0FD032
:10A6A000FEF708F90C232B702300094AA0331A6027
:10A6B0000223783407490848237001F0ACF9C5E754
:10A6C000FFF790FAC2E7C046C80C0010F80400106B
:10A6D00027A6000015F30000500D001010B5FBF781
:10A6E00065FC084B1A0086321178002904D000233B
:10A6F0001370FAF7B5FA10BD7C331888FFF796FD92
:10A70000F9E7C046C80C0010F8B50A4C0026250031
:10A710000027094BE835186059609E60DF601033F0
:10A72000AB42F8D101211000A834FFF77FFD20686B
:10A730006168F8BDC80C0010700D0010F0B57E4BBC
:10A7400089B05B69069007937C4BA8331E685F68ED
:10A750007A4B3000B8331C685D68390022002B004A
:10A7600001F010FD00280DD0002200237349F831BC
:10A770008A60CB6032003B000C604D6026002F00E9
:10A7800014001D00069A30003900FFF7BDFF6B4B27
:10A790000290039187331B78002B00D1C5E0012084
:10A7A000404209B0F0BD059B069A01332000290004
:10A7B0000593FFF7A9FF614B0090019187331B7848
:10A7C000002BECD1029A039B03F0D6FBF7F7AEFD0A
:10A7D0005B4A5C4B01F0C2FC002819D022002B0020
:10A7E0003000390002F030FA574B002203F052F9E2
:10A7F000069A06000F00FFF787FF02900391F7F714
:10A8000095FD4F4A4F4B01F0A9FC002800D087E08E
:10A8100032003B002000290003F0AEFB009A019BB0
:10A8200003F038F9029A039B06000F000098019983
:10A8300003F0A2FB02000B003000390002F020FD03
:10A8400002000B002000290003F096FB22002B00E1
:10A850000290039103F090FBF7F768FD384A394BFB
:10A8600001F07CFC002806D1059B652B39D106221E
:10A87000324B87331A70314E0598370003F0FAFED9
:10A88000D83738607960310000220023E0310A6057
:10A890004B60009A019B3100C8310A604B60310067
:10A8A00000220023D0310A604B603100B8310C60C7
:10A8B0004D603100C0310A604B60029B039C310047
:10A8C000A8310B604C60310000230022B0310A60D7
:10A8D0004B60873633781800062B00D161E70020E3
:10A8E0005FE7154E079A73699B1A632B05D9FAF730
:10A8F00045FD0028BFD1736907932600009A019B8C
:10A900002F00029C039D0292039300980199F7F790
:10A910000DFD0B4A0B4B01F035FC002800D042E73F
:10A920000294039534003D00A5E700220593074BF0
:10A9300000920193E9E7C04648040010C80C0010DB
:10A940001656E79EAF03D23C0000E03F0000F03F08
:10A95000F7B5FBF72BFB2C4C26009C363578002DE9
:10A960001BD0FEF7F7FAC5B22800FDF7EBFA23007B
:10A9700085331B780600002B04D029005020FAF7FD
:10A98000B5F9F7BDFDF796FF002E02D03000FFF7B6
:10A99000D5FEA43401232370F3E7270086373B78E4
:10A9A000002B20D026007C363288184B9B18587814
:10A9B000FDF7C8FA0028E4D033880193FFF7BEFE04
:10A9C000019B012233802300A4331A70002801DA8E
:10A9D0003D70D6E7062804D1FAF742F92300873301
:10A9E0001D708634D6E7FDF765FF09233370230019
:10A9F000074AA0331A6002237834064906482370B8
:10AA000001F009F8BDE7C046C80C0010F8040010BA
:10AA100051A900001EF30000500D001010B5064BA8
:10AA200086331B78002B05D0FFF736FAFA2080001A
:10AA3000F5F70AFC10BDC046C80C0010F0B5BE4BBF
:10AA4000DDB05B6912901393BC4BA6331B78181CC6
:10AA50000F2B00D90F20C0B2404203F00BFE0200C2
:10AA60000B000020B649F7F743FFB44E1A901B9134
:10AA70003300A8335C681B68009301940098019927
:10AA80003300B8331C685D6822002B0001F07AFBAC
:10AA900000280CD000220023F83634607560B260C4
:10AAA000F360009A019B0094019514001D00009A28
:10AAB000019B2000290002F0C7F80022A14B02F000
:10AAC000E9FF0A900B918021002300220020C90594
:10AAD000F7F70EFF0A980B99129AFFF715FE974B9E
:10AAE0000690079187331E78002E04D0012305932A
:10AAF00005985DB0F0BD009A019B2000290003F08D
:10AB00003BFA0022904B02F0C5FF00228F4B0C90C5
:10AB10000D9102F0BFFF069A079B1490159102F069
:10AB2000B9FF3CAB04931CAB109301231C901D9107
:10AB300000960E930123009A9B1A501E119303F066
:10AB400099FD169017910B0080210200C905002085
:10AB5000F7F7CEFE00227E4B03F00EFA02000B0048
:10AB600004000D0002F096FF02000B0006000F002B
:10AB70000020764903F000FA22002B0002F08AFF41
:10AB80000C9A0D9B02F086FF0A9A0B9B02F05CF870
:10AB9000129AFFF7B9FD694B0890099187331B782A
:10ABA0000593002BA2D10E9B3200013303930020AA
:10ABB0003B00674903F0E0F9089A099B02F06AFF3D
:10ABC00008900991119803F055FD0B0080210200B7
:10ABD000C9050020F7F78CFE039B0E9A1890199177
:10ABE000981A03F047FD002206000F0018981999E3
:10ABF000574B03F0C1F902000B003000390001F09F
:10AC0000B7FA002800D0A7E0089A099B0698079990
:10AC100002F01AF8169A179B0690079180210020DF
:10AC2000C905F7F765FE02000B001498159902F0AC
:10AC300031FF069A079B02F02DFF0124049B186048
:10AC400059601D00109B089308992E686F680CC905
:10AC500030000891390003F08FF90E900F91200019
:10AC600003F008FD02000B0000203A49F7F740FE10
:10AC70000022374B03F080F902000B000E980F9969
:10AC800002F0FEFA3B00320001F0DEFF119B0134BE
:10AC9000A860E96008359C42D6DD009BD900049B82
:10ACA00049425A189368D46808930994109B59181C
:10ACB00008684968089A099B03F05EF9089A099B9D
:10ACC0000E900F9102F0DCFAF7F730FB0B001199B0
:10ACD0000200012900D1CDE01A981B9901F052FA27
:10ACE000002803D1059B002B00D18DE0134C039865
:10ACF000250003F0BFFC230000260027C835D03311
:10AD0000286069600E980F991E605F60F7F70EFB70
:10AD10002300B833186059600899099A2300C0339A
:10AD20001E605F602300B034A83319605A6026604B
:10AD300067600023DBE6C04648040010C80C001022
:10AD4000000024400000E03F0000D03F0000084029
:10AD50000000F03F00001040039B00980133039374
:10AD600003F088FC0B0080210200C9050020F7F7E2
:10AD7000BFFD02000B002000290001F065FF02006A
:10AD80000B0004000D0002F085FE02000B0006001F
:10AD90000F0000203E4903F0EFF822002B0002F0E4
:10ADA00079FE0C9A0D9B02F075FE0A9A0B9B01F03E
:10ADB0004BFF129AFFF7A8FC364B18901991873376
:10ADC0001B78002B00D091E6334B139A5B699B1ADA
:10ADD000632B08D9FAF7D2FA002801D00123059392
:10ADE0002D4B5B69139332003B0000202B4903F08D
:10ADF000C3F8189A199B02F04DFE02000B00089848
:10AE0000099901F021FFDBE6009B0F3336D1214C7D
:10AE10000622230087331A70039803F02BFC2300CB
:10AE2000002600272500D0331E605F60049BC835D4
:10AE30009A6FDB6F00920193109B28606960009805
:10AE4000019980331A685B6803F096F8F7F76EFA99
:10AE50002300B833186059600099019A2300C03369
:10AE60001E605F602300B034A83319605A6026600A
:10AE700067603DE6059B002B00D037E7009B049AF6
:10AE8000013B0093109B10920493039B51E6C04634
:10AE900000000840C80C0010480400100000F03FFB
:10AEA000F8B5FBF783F8294C25009C352B78002B4F
:10AEB00022D0FEF74FF8C5B22800FDF743F8230073
:10AEC00085331E780700002E04D029004F20F9F7A3
:10AED0000DFFF8BDFDF7EEFC002F09D02500012382
:10AEE00086352B70FEF7D8FF3800FFF7A7FD2E70D0
:10AEF0000123A4342370ECE7230086331B78002B56
:10AF000014D023007C331D88114B5B195878FDF752
:10AF100019F8002801D0FFF791FD230022007C33AF
:10AF20001D80012386321370A434E3E7FDF7C2FCD1
:10AF300009232B702300074AA0331A6002237834B8
:10AF400005490648237000F066FDC2E7C80C0010F2
:10AF5000F8040010A1AE000029F30000500D00100D
:10AF60004F4B10B51A694F4901321A614E4A1268A7
:10AF7000D2B2302A66D01AD8182A0ED005D8082A9C
:10AF800036D0102A44D008234EE0202A69D0282A3F
:10AF9000F9D1D8689A69904248D2DA68501CD860D2
:10AFA00001339B18DB7F414ADBB21360EBE7482A91
:10AFB00057D009D8382A4DD0402AE4D1DA69042381
:10AFC000012A4BD10B60DEE7502A53D0582ADAD140
:10AFD000364A12689868D2B2441C9C601C0038340F
:10AFE00022540222FF325A608023F13ADB0552E0FC
:10AFF0000022DA60D868421CDA605A1C1218D27F2C
:10B000002A48D2B2026028220A60273A5A6010BD4C
:10B0100000229A60DA68501CD86001339B18DB7FED
:10B02000224ADBB2136028230B60F0E78022D86944
:10B03000D205002801D02023B7E70220FF30586056
:10B040001023B2E780221020D205106008220A6087
:10B05000FA32DBE7822252005A6094E78022D2055E
:10B06000A3E780221020D205106008220A60042283
:10B07000FF32CBE70D4A12689868D2B2441C9C603C
:10B080001C0038342254DA699868531E0422834223
:10B0900003D98023DB051A6075E70A6073E7C046B1
:10B0A0004804001018000040040000400800004060
:10B0B000202130B5064A074C0378002B01D1180037
:10B0C00030BD013015680D42FCD02360F4E7C04666
:10B0D00014800040008000400E22174B10B51B6802
:10B0E0001340062B12D1154B90321B68134205D02A
:10B0F000134ADBB25360134B1B6810BDDB07FCD552
:10B10000104B1868C0B2F5F78FF8F6E7042BF7D0AC
:10B110000C2B05D10A4AF43351680B435360ECE71A
:10B12000022BEAD1054B1A68054B920602D5002284
:10B130009A60E2E70122FBE70880004014800040AB
:10B1400048140010008000400122034B1A60034A9B
:10B15000536801335360704700800140C8040010F9
:10B160000122034B1A60034A9368013393607047CE
:10B1700000400140C80400100122034B1A60034A3A
:10B18000D3680133D360704700000140C804001049
:10B190000122034B1A60034A13690133136170479C
:10B1A00000C00040C8040010074A084B5169013133
:10B1B00002D15969013159615169013151619A696D
:10B1C00001329A617047C04648040010C80400105C
:10B1D000064A10B5136801331360054B9868FAF7F7
:10B1E00075FCF5F747F8C046C04610BDC80400100E
:10B1F00000000010F7B5F5F76DF8B64A01241368A2
:10B200001B0B1B031360B44A13681B0B1B03136057
:10B21000B24A13681B0B1B031360B14A13681B0B64
:10B220001B0313600022AF4B1A60AF4B1C601A6007
:10B230001C601A682242FCD02322AC4B01201A6009
:10B24000FAF744FCF5F746F840213F20A84B1A686E
:10B250008A431A60A74A1060A74A14601A688A4392
:10B260001A60FAF7E5FDFAF7D9FDFAF709FCA34BE6
:10B270005B6D0193002B01D1F5F764F90021A04823
:10B28000F5F736F800219F48F5F732F8F5F730F971
:10B29000F5F7FEF8994C092248340021200000F00F
:10B2A000C5FB0020E071F5F76DF9974F002822D01B
:10B2B000F5F7B2F80C23184002D023781843207019
:10B2C0008E4C483423785B0711D5F5F76FF8A378D7
:10B2D000002B03D0237A012B02D80133237201E023
:10B2E000BB69FB610023854ABB614832D3700022F1
:10B2F000824B48331A70814B4833DB79002B01D1E4
:10B30000F5F754F8FA2300259B00BD61FB61FAF7BD
:10B310003DFBF0227D4CD2002900200000F086FB8E
:10B3200023000222A433FF321A802300FD3AA63301
:10B330001A7023000B3278331A70754A75490C3233
:10B34000754800F068FBFAF725FEFAF713FAFEF7E6
:10B35000A3FDFAF713F8051E00D12AE16F4AA35C9A
:10B36000002B04D00023A35422007C32138000223F
:10B3700023003A6187331E78964215D01A70FAF787
:10B38000F9F93A69664B9A4203D9FAF7B3FD0023FB
:10B390003B61FEF781FD614BE35C002BD9D10321BA
:10B3A0000A20FAF7E7FBD4E7A02D4EDDA021280004
:10B3B00000F0BAFE0D2917D1FDF77CFA594800F0CC
:10B3C0001FFB0125584B5948595D00F019FBFA2322
:10B3D0000135DB009D42F5D1554D280000F010FBF2
:10B3E000280000F00DFBCAE711290CD1FDF762FA25
:10B3F00023007C331E800123484A4E48A35400F0AA
:10B40000FFFA4B48EDE7072907D1230086331B7865
:10B41000002BB4D1FEF764FBB1E7062907D1230066
:10B4200086331B78002BAAD1FEF7DCFBA7E7322975
:10B43000A5D1FA223100D2003B4800F0F7FA2300F0
:10B440007C331E80FDF736FA99E723009C331B7886
:10B45000002B75D02B003D3B012B21D92821280042
:10B4600000F062FE12291BD004230A009A43012A2D
:10B4700016D02A00153A132A03D82F4BD340DB07E6
:10B480000ED42B000422143B934304D123008333B6
:10B490001B78002B04D12B000422373B93430FD1A0
:10B4A000E8B2F9F7CDFB1548643000F0F7FA230055
:10B4B00078331B78984200D061E7FDF725FA5EE704
:10B4C0001429F0D81D4BCB40DB07ECD52831C8B28E
:10B4D000E7E7C04600800050008001500080025025
:10B4E00000800350408004404480044008800440B1
:10B4F0003882044024800440D8800440480400106E
:10B50000984004409C400440C8040010C80C00103F
:10B51000000000109EF10000500D001074070000A4
:10B520005702000042F30000F804001038F3000056
:10B530004CF300003CF30000F3EE0F0010911900F3
:10B54000230085331B78EDB22800002B29D0F9F7B2
:10B55000A5FA002824D120232A009A43122A1FD0BA
:10B560002B0002229343012B1AD02B00523B012BBC
:10B5700016D9612D14D02633DBB2102B03D84E4AD6
:10B58000DA40D3070CD42821280000F051FBFB231C
:10B590000539194204D02B007F33DBB21E2B03D8B0
:10B5A0002800F9F74DFBEAE600212800F9F79EFB99
:10B5B000E5E6424BE35C002B00D1E2E6404A917B9A
:10B5C000537B994200D1C4E6937BD318DD7B937BF8
:10B5D0000133DBB293735BB2002B01DA0023937368
:10B5E0000D2D03D00A2D01D0202D2FD13E00203665
:10B5F0003000F9F7F5FF0A2201900021300000F039
:10B6000015FA304B5E61304BE35C002B03D129000F
:10B610002E4800F0F5F9019BFF2B00D999E6260092
:10B620007C363588002D06D1FA222900D200284820
:10B6300000F0FCF9358022007C32138825498B42CA
:10B6400033D1002313801D4AA35482E6082D01D074
:10B650007F2D18D11C4BE35C002B14D13B00194EFD
:10B66000203372699A420ED90821184800F0C8F9AF
:10B670002021164800F0C4F90821144800F0C0F950
:10B680007369013B73612B00303B092B96D80E4B3D
:10B69000E35C002B03D129000C4800F0B1F9094A02
:10B6A0005369591C51611D7088E701339BB21380A7
:10B6B0000199074AD1544CE611310100740700008A
:10B6C00048140010000000107307000071F2000021
:10B6D000F8040010CF07000070B500241E5D0519A6
:10B6E000002E08D1121B1300002B07DCD043C0171B
:10B6F0001040001970BD06550134EFE72970013B79
:10B700000135F1E7F8B505000C001E00571E092BA6
:10B7100016D90A21180000F005FA210003003A00AA
:10B720002800FFF7EFFF04002D1830000A2100F079
:10B730007FFA30312970601CF8BD2C70013F013553
:10B74000002FFADC141E00DC0124013CEDE7F0B50B
:10B7500085B00B9E040003910A9F551E002E01D157
:10B76000092F1DD90A2200233800310000F066FAA3
:10B770002A000090019120000399FFF7E8FF0500DF
:10B780002418380031000A22002300F057FA681C00
:10B790003032227005B0F0BD039B013D23700134AF
:10B7A000002DF9DC151E00DC0125013DE9E7F7B5A8
:10B7B0000F00D9171E005B184B4004000193551E63
:10B7C000092B16D918000A2100F0ACF90300002E4D
:10B7D00000DA43422A0020003900FFF7E8FF0500A5
:10B7E000241801980A2100F023FA3031681C2170D6
:10B7F000FEBD002E00DA951E23006119CA1A002A28
:10B800000BDCE843C017054064196B1C002EE8DA16
:10B810002D221D0022700134E3E71F700133EDE794
:10B8200073B5069E04001D0010003309013A002B79
:10B8300011D0009320002B00FFF7F2FF24180F23F4
:10B840001E40F3B2092E0DD830330130237076BD7F
:10B850002170013A0134002AFADC002800DC0120C2
:10B860000138ECE7002D01D03733EEE75733ECE732
:10B87000F0B585B0040003911D00002801D000231D
:10B880000370002630001378002B00D092E0039A5A
:10B89000B24200D99AE00023013C2370013E96E0B9
:10B8A0005178252902D1217002328CE0302924D030
:10B8B000531C029320239C46029B1B782D3B5A422B
:10B8C0005341029AD31800220293029B1B781F0057
:10B8D000303F092F15D9039997198F4201D98A1B37
:10B8E000D2B2692B46D015D8632B5ED0642B41D0E1
:10B8F000582B4ED00126764269E0931C02938C4669
:10B90000DAE70A214A439A18029B303A0133D2B24D
:10B910000293DAE7732B41D01FD86C2BEAD1029B3C
:10B920005B786C2B14D1029B9B78752B10D1029BFA
:10B9300007350233072102932B008B431D00186843
:10B94000596800900191614620000835FFF7FFFE1D
:10B95000029A24180132361895E7752B12D0782BED
:10B96000C8D12B682F1D0093002361462000FFF7EC
:10B9700057FF05E02B68614620002F1DFFF717FFDA
:10B980003D00E5E72B68614620002F1DFFF7BAFE5A
:10B99000F6E72B682F1D00930123E6E72B6861462D
:10B9A00020002F1DFFF798FEEAE72B680120237087
:10B9B0000435CDE70399B14200D86CE7252B00D1BF
:10B9C0006EE701322370013601345CE723703000EA
:10B9D00005B0F0BD10B513000A006421FFF748FF61
:10B9E00010BD00B59BB00A00010001A8FFF7F2FFEF
:10B9F000632800DDFEE701A8FFF75AFB1BB000BD7E
:10BA00000FB407B504A901C90191FFF7EAFF03B01C
:10BA100008BC04B018470EB403B503AA02CA0192C9
:10BA2000FFF7D8FF02B008BC03B01847F0B5050017
:10BA3000830704D003009A189A4217D1F0BD03007F
:10BA4000032AF8D9131F0F049B080C063C439E00E1
:10BA500036180C430F0204363C4310C5B542FCD1E6
:10BA6000032401339B00C3182240E4E7197001331B
:10BA7000E2E710B5814208D20139431E002A00D105
:10BA800010BD8C5C9C54013AF8E700238142F7D941
:10BA90009A42F5D0CC5CC4540133F9E702000300AC
:10BAA000981A0133591E09780029F9D1704703000B
:10BAB0000A781A70002A00D1704701310133F7E784
:10BAC000002210B5835C8C5CA34201D0181B10BD12
:10BAD0000132002BF6D11800F9E7FEE7FEE700007F
:10BAE000002370B50A480B490B4C1A188A4207D339
:10BAF00000210A4B0A4A934206D3FFF77BFBFEE77D
:10BB0000E55C01331570F0E719700133F3E7C046C7
:10BB100000000010480400109CF5000048040010CC
:10BB2000E0150010002243088B4274D303098B42B6
:10BB30005FD3030A8B4244D3030B8B4228D3030CFD
:10BB40008B420DD3FF22090212BA030C8B4202D39F
:10BB50001212090265D0030B8B4219D300E0090AC7
:10BB6000C30B8B4201D3CB03C01A5241830B8B42D0
:10BB700001D38B03C01A5241430B8B4201D34B03B9
:10BB8000C01A5241030B8B4201D30B03C01A52411E
:10BB9000C30A8B4201D3CB02C01A5241830A8B42A3
:10BBA00001D38B02C01A5241430A8B4201D34B028C
:10BBB000C01A5241030A8B4201D30B02C01A5241F0
:10BBC000CDD2C3098B4201D3CB01C01A52418309A4
:10BBD0008B4201D38B01C01A524143098B4201D3DE
:10BBE0004B01C01A524103098B4201D30B01C01A09
:10BBF0005241C3088B4201D3CB00C01A5241830883
:10BC00008B4201D38B00C01A524143088B4201D3AF
:10BC10004B00C01A5241411A00D20146524110460F
:10BC20007047FFE701B5002000F006F802BDC046EE
:10BC30000029F7D076E770477047C046002B11D136
:10BC4000002A0FD1002900D1002802D00021C943C9
:10BC5000081C07B4024802A14018029003BDC04668
:10BC6000D9FFFFFF03B4684601B5029800F006F85B
:10BC7000019B9E4602B00CBC7047C046F0B54F46D3
:10BC80004646D646C0B5040082B00D00914698469F
:10BC90008B422FD82CD04146484600F0B1F82900FD
:10BCA0000600200000F0ACF8331A9C46203B9A4670
:10BCB00000D576E04B46524693401F004B46624605
:10BCC00093401E00AF4228D825D05346A41BBD4147
:10BCD000002B00DA7BE00022002300920193012375
:10BCE000524693400193012362469340009318E02B
:10BCF0008242D0D900220023009201930A9B002B9C
:10BD000001D01C605D600098019902B01CBC904697
:10BD10009946A246F0BDA342D7D900220023009243
:10BD200001936346002BE9D0FB0798464146720811
:10BD30000A437B0866460EE0AB4201D1A2420CD812
:10BD4000A41A9D41012024196D410021013E2418AF
:10BD50004D41002E06D0AB42EED9013E24196D4173
:10BD6000002EF8D100980199534600196941002B23
:10BD700023DB2B005246D3402A006446E2401C00DD
:10BD800053461500002B2DDB26005746BE403300DE
:10BD900026006746BE403200801A9941009001910A
:10BDA000ACE7624620239B1A4A46DA4061461300FC
:10BDB00042468A4017001F4380E7624620239B1AB1
:10BDC0002A0066469A402300F3401343D4E76246B4
:10BDD000202300219B1A0022009101920122DA40C7
:10BDE000019280E72023624626009B1ADE402F0046
:10BDF000B0466646B74046463B003343C8E7C046B8
:10BE000010B5002903D100F007F8203002E0081C2B
:10BE100000F002F810BDC0461C2101231B0498420B
:10BE200001D3000C10391B0A984201D3000A0839CB
:10BE30001B09984201D30009043902A2105C401882
:10BE40007047C04604030202010101010000000026
:10BE500000000000C317C018584070470022034B71
:10BE60001B68A83318605A607047C046180000105D
:10BE7000094B10B51C68094AA83420686168084B52
:10BE800000F038F8012200238018594120606160D9
:10BE90004800400810BDC046180000102D7F954C8A
:10BEA0002DF4515870B50400830717D102680F4B69
:10BEB000D31893430E4A150013420FD10430026881
:10BEC0000A4BD31893432B4208D104300268074B26
:10BED000D31893432B42F1D000E001300378002BBC
:10BEE000FBD1FFF7E4FD200070BDC046FFFEFEFE63
:10BEF00080808080F0B5CE46474615042D0C2E007C
:10BF000080B50704140C3F0C9946030C7E435D4337
:10BF1000674363437F19340CE4199C46A54203D957
:10BF200080235B029846C4444B4643435143250C4F
:10BF300036046544360C2404A4195B1959182000F2
:10BF40000CBC90469946F0BD02B4714649084900C0
:10BF5000095C49008E4402BC7047C04603460B434F
:10BF60007FD4002243088B4274D303098B425FD3F2
:10BF7000030A8B4244D3030B8B4228D3030C8B421E
:10BF80000DD3FF22090212BA030C8B4202D3121204
:10BF9000090265D0030B8B4219D300E0090AC30BD9
:10BFA0008B4201D3CB03C01A5241830B8B4201D386
:10BFB0008B03C01A5241430B8B4201D34B03C01A6F
:10BFC0005241030B8B4201D30B03C01A5241C30AE7
:10BFD0008B4201D3CB02C01A5241830A8B4201D358
:10BFE0008B02C01A5241430A8B4201D34B02C01A42
:10BFF0005241030A8B4201D30B02C01A5241CDD2E7
:10C00000C3098B4201D3CB01C01A524183098B4231
:10C0100001D38B01C01A524143098B4201D34B011A
:10C02000C01A524103098B4201D30B01C01A52417D
:10C03000C3088B4201D3CB00C01A524183088B4204
:10C0400001D38B00C01A524143088B4201D34B00ED
:10C05000C01A5241411A00D201465241104670475F
:10C060005DE0CA0F00D04942031000D34042534064
:10C0700000229C4603098B422DD3030A8B4212D324
:10C08000FC22890112BA030A8B420CD38901921156
:10C090008B4208D3890192118B4204D389013AD093
:10C0A000921100E08909C3098B4201D3CB01C01A68
:10C0B000524183098B4201D38B01C01A524143097B
:10C0C0008B4201D34B01C01A524103098B4201D369
:10C0D0000B01C01A5241C3088B4201D3CB00C01AD6
:10C0E000524183088B4201D38B00C01A5241D9D2EE
:10C0F00043088B4201D34B00C01A5241411A00D26F
:10C100000146634652415B10104601D34042002B6A
:10C1100000D54942704763465B1000D3404201B5E9
:10C120000020FFF789FD02BD0029F8D016E770470F
:10C130008446101C62468C46191C634600E0C046CB
:10C140001FB501F03FFC002801D40021C8421FBDEB
:10C1500010B501F097FB4042013010BD10B501F061
:10C1600031FC002801DB002010BD012010BDC046BD
:10C1700010B501F027FC002801DD002010BD0120D2
:10C1800010BDC04610B501F0B9FB002801DC00204D
:10C1900010BD012010BDC04610B501F0AFFB002856
:10C1A00001DA002010BD012010BDC046F0B5DE460A
:10C1B00057464E4645469446E0B595B09B461E9B75
:10C1C000654699461F9B04009846209B6046029353
:10C1D000219B029A9A46594653460A9501F05AFC09
:10C1E000239F229E0490059132003B004846414621
:10C1F00003960B9701F04EFC3D0006000F00039ADA
:10C200002B000A9859460C960D9701F043FC4A46BC
:10C210000690079143460298514601F03BFC3200DC
:10C220003B00089009910498059901F0A5FE089A31
:10C23000099B06000F000698079900F005FD3200E3
:10C24000009001913B0030003900FFF781FF00288A
:10C250000DD0009A019B200026606760A260E36019
:10C2600015B03CBC90469946A246AB46F0BD00983E
:10C27000019902000B00FFF76BFF0028E9D10A9932
:10C280005B468C460A0060465946654601F074FEDE
:10C290004A461090119143464846414601F06CFED3
:10C2A0000B000200FFF754FF3822434258416B460F
:10C2B0009B1818704A46434641464846FFF748FFD8
:10C2C0003822431E98416B469B181B782A00034076
:10C2D0000E9328005B465946FFF73AFF002800D12D
:10C2E00023E11098119902000B00FFF731FF00289D
:10C2F00000D01AE159460022D34B002900DAD34B73
:10C300009B460E9B0A925A425341D14A5B421340CC
:10C31000CD4A94466344424600215B00D20FD207C7
:10C320005B08134389469846029A53460298514641
:10C33000FFF70EFF002800D168E10B99039D8C46A2
:10C340000B002A0028006146FFF702FF002800D1F9
:10C3500050E101230E93029A53460298514601F090
:10C360000BFE129013910B99039D8C462A000B0033
:10C3700028006146654601F0FFFD0B000200FFF753
:10C38000E7FE4022434258416B469B181870039ABF
:10C390002B0029000398FFF7DBFE4022431E984143
:10C3A0006B469B181B78029A0340109302985346E1
:10C3B0005146FFF7CDFE002868D01298139902006D
:10C3C0000B00FFF7C5FE002860D1524600259E4BAA
:10C3D000002A00DA9D4B9A46109B9D4A013B134070
:10C3E000994A0295944663440B9A5B00D70F00224A
:10C3F0000A9E5B08FF073B4303920B9332005B46A8
:10C4000030005946FFF7A4FE002800D138E14A4623
:10C41000434648464146FFF79BFE002800D125E1F0
:10C42000029A53460A98594601F034FB0B9D0600C8
:10C430000F00039A2B004846414601F02BFB0200F7
:10C440000B003000390001F097FD0022814B01F014
:10C4500021FB039A2B0006000F000A98594601F0B1
:10C4600019FB029A0090019153464846414601F05B
:10C4700011FB02000B000098019900F0E5FB00227F
:10C48000744B01F007FB00900191E2E6109B002B3A
:10C4900000D0A4E00E9B002BC2D1049805990200A5
:10C4A0000B0001F069FD0E900F91049805990200B0
:10C4B0000B00FFF74DFE002846D00E980F990200A2
:10C4C0000B00FFF745FE00283ED10A9E5B46320076
:10C4D00030005946FFF73CFE002800D1A0E04A4654
:10C4E000434648464146FFF733FE002800D1B3E0FB
:10C4F000029A534602985146FFF72AFE002800D1BF
:10C5000098E0039F0B9E3A00330038003100FFF79C
:10C510001FFE002884D100220B991300914201DAFA
:10C5200080231B0603920B937AE70E9B002B00D10E
:10C5300011E7002259461300914201DA80231B06BD
:10C540009B460A92404BE6E60C980D9902000B00C0
:10C5500001F012FD049005910C980D9902000B005A
:10C56000FFF7F6FD002807D00498059902000B009C
:10C57000FFF7EEFD0028A8D00698079902000B00EF
:10C5800001F0FAFC049005910698079902000B004F
:10C59000FFF7DEFD002807D00498059902000B0084
:10C5A000FFF7D6FD002890D00898099902000B00EB
:10C5B00001F0E2FC049005910898099902000B0033
:10C5C000FFF7C6FD002800D143E604980599020054
:10C5D0000B00FFF7BDFD002800D03AE675E7002507
:10C5E00052462B00AA4201DA80231B069A46029586
:10C5F000154BF9E600220B991300914201DA8023D2
:10C600001B060B93012303920E93A4E652464D465C
:10C610004B464A4501DA80231B0602959A468CE672
:10C6200000265A463300B24201DA80231B060A96DE
:10C630009B4654E7002552462B00AA4201DA80238C
:10C640001B0602959A465CE70000F03F0000F0BF31
:10C65000000010C00000F07F00224146130091420C
:10C6600001DA80231B069146984641E700224146A5
:10C670001300914201DA80231B0691469846CFE6CB
:10C6800000265A463300B24201DA80231B060A967E
:10C690009B46BCE6F0B557464E464546DE46E0B5FD
:10C6A0008BB0169982468946179918988846199929
:10C6B000149E8B4641464C005946159F49000192F5
:10C6C00003930500059002004B0848466108029656
:10C6D0000497FFF743FD00284BD02A005B464846ED
:10C6E0004146059500F0CCFD04000D0002000B0052
:10C6F0004846414601F0CEF9059A5B4600F0A4FA9F
:10C700002200069007912B000198039901F0C2F9CD
:10C7100032003B000296049700F096FA069A079BB7
:10C7200000F0AEFD22002B0006000F0002980499D5
:10C7300001F0B0F9019A039B01F01EFC069A079BD9
:10C7400000F09EFD320004000D003B003000390077
:10C75000FFF7FEFC00283ED0534650461E605F6047
:10C760009C60DD600BB03CBC90469946A246AB464F
:10C77000F0BD059E4A4643463000594600F080FD14
:10C7800004000D0002000B003000594601F082F950
:10C790004A46434600F058FA06000F00029A049BEE
:10C7A0002000290001F076F9019A039B00F04CFA71
:10C7B00032003B000696079700F062FD019A039B4A
:10C7C00006000F002000290001F064F902000B00B0
:10C7D00002980499B0E722002B0020002900FFF7FF
:10C7E000B7FC0028B8D10022002348464146FFF795
:10C7F000AFFC002828D00022002305985946FFF7F7
:10C80000A7FC002820D00399019A0B000198FFF79C
:10C810009FFC002800D176E143460024DE4D002B2A
:10C8200001DA0024DD4D019A039B2000290001F06C
:10C8300031F9029A06000F0020002900049B01F044
:10C8400029F904000D0087E70198039906900791E4
:10C8500002000B000698079901F08EFB08900991E1
:10C860000399019A0B000198FFF772FC00287ED013
:10C870000898099902000B00FFF76AFC002876D19E
:10C880004A4643464846414601F076FB02000B000B
:10C89000FFF75EFC002800D146E105995B460A00DF
:10C8A0000800594601F068FB02000B00FFF750FC3E
:10C8B000002800D195E0BA4B039A029FD20F049E44
:10C8C000D207134301933A0033003800310001F0DE
:10C8D00053FB3A0004000D00330038003100FFF72D
:10C8E00037FC002800D153E122002B002000290052
:10C8F000FFF72EFC002800D04AE1A94C049B00223F
:10C90000DB0FDB071C434846019B414601F0C2F8A0
:10C91000230006000F0000220598594601F0BAF8DE
:10C9200002000B003000390000F08EF900229A4B13
:10C9300001F0B0F82300002206000F0048464146EF
:10C9400001F0A8F8002204000D00019B059859464B
:10C9500001F0A0F802000B002000290001F00CFB00
:10C9600000228D4B01F096F804000D00F4E60298C9
:10C9700004990690079102000B000698079901F0B0
:10C98000FBFA069007910499029A0B000298FFF7B0
:10C99000DFFB002800D1C7E00698079902000B00D2
:10C9A000FFF7D6FB002800D0BEE04A464346484683
:10C9B000414601F0E1FA02000B00FFF7C9FB002835
:10C9C00000D1B1E005995B460A000800594601F024
:10C9D000D3FA0B000200FFF7BBFB0023984200D004
:10C9E0006AE705995B4689460A000800594601F046
:10C9F000C3FA4A46069007915B4648465946FFF7F8
:10CA0000A7FB002800D1A7E60698079902000B00B3
:10CA1000FFF79EFB002800D09EE6089809990200C7
:10CA20000B00FFF795FB002800D195E60299894697
:10CA30000A00049948460B0001F09EFA0B00020020
:10CA4000FFF786FB0023984200D185E64246D70FC8
:10CA5000059EFF073B433200994630005B4659462E
:10CA600001F08AFA320004000D005B46300059469E
:10CA7000FFF76EFB002800D18CE022002B00200085
:10CA80002900FFF765FB002800D083E0444E5B4699
:10CA9000DB0FDB071E4300224B460198039900F091
:10CAA000F9FFB0463300049E04000D00002231005F
:10CAB000029800F0EFFF02000B002000290000F0B8
:10CAC000C3F80022002300F0E5FFB34600224B46E6
:10CAD00006000F000298594600F0DCFF0022040017
:10CAE0000D0043460198039900F0D4FF02000B00AB
:10CAF0002000290001F040FA0022002300F0CAFFC4
:10CB000004000D0028E60499029A0B000298FFF732
:10CB10001FFB002800D07FE60399019A0B000198C3
:10CB200001F02AFA089009914A4643464846414690
:10CB300001F022FA4A46069007914346484641468C
:10CB4000FFF706FB002800D14BE706980799020083
:10CB50000B00FFF7FDFA002800D042E7089809997A
:10CB600002000B00FFF7F4FA002800D1F4E5029967
:10CB700089460A00049948460B0001F0FDF90200BD
:10CB80000B00FFF7E5FA002800D1E5E5044B5DE76F
:10CB90000024B3E600267AE70000F07F0000F0FFF3
:10CBA0000000F03F70B500220C4B04000D00FFF7B1
:10CBB000F3FA002804D12000290001F025FD70BD02
:10CBC000064B00222000290001F0D6F901F01CFDDF
:10CBD00080231B069C466044F1E7C0460000E0410C
:10CBE00070B500220B4B0D00040000F053FFFFF75F
:10CBF000D9FF060001F078FD0022074B00F04AFF44
:10CC000002000B002000290001F0B6F9FFF7CAFF6F
:10CC1000310070BD0000F03D0000F04170B506002D
:10CC2000080001F061FD0022064B00F033FF0D000B
:10CC30000400300001F058FD2B00220000F004F841
:10CC400070BDC0460000F041F0B54F464646D6469E
:10CC50000C000903C0B5490A470F5E0039431F03A2
:10CC6000DB0F9C4665007B0A570F1F436D0DE40FD9
:10CC7000760DA146C000B846D200AB1B64457BD000
:10CC8000002B5FDD002E00D0A4E03E00164300D153
:10CC900012E15E1E002E00D09EE1871A4346B84284
:10CCA00080410125C91A4042091A0B0200D431E122
:10CCB00049024E0A002E00D16EE13000FFF7ACF8B9
:10CCC0000300083B1F2B00DD61E120223900D21A4E
:10CCD0009E40D1409F400E439D4200DD51E15D1BCF
:10CCE0006B1C1F2B00DD7CE12021C91A3D003000A8
:10CCF0008F408840DD40791E8F4131000722284354
:10CD0000D940002507433A40002A09D00F233B4071
:10CD1000042B05D03B1DBB42BF417F42C9191F00F8
:10CD20000B0200D426E26A1CC64B55056D0D9A42D3
:10CD300000D106E1C44AFF080A40530752023B43B0
:10CD4000120B8EE0002B00D0B8E06B1C5B055B0D76
:10CD5000012B00DC30E1871A4346B842B641CB1ABA
:10CD600076429E1B330200D54CE13B003343A1D1F8
:10CD700000220024002570E0002B00DCE5E0002EFE
:10CD800000D183E0AF4EB54260D0802636043743F1
:10CD9000B846382B00DC3EE1434613431F007A1EA1
:10CDA00097413F1887428041404209180B0200D446
:10CDB000B0E0A44B01359D4200D1C3E0A24A7B08FC
:10CDC0000A4001210F401F435108D30707221F4388
:10CDD0003A4099E79B4EB54238D080263604374317
:10CDE000B846382B00DDDCE01F2B00DC30E11E00F4
:10CDF0004746203EF740BC46202B04D04026F31A7D
:10CE000046469E403243170063467A1E97411F43B1
:10CE1000CCE0002B00D104E24346134300D159E19A
:10CE20004B07C00818438023C9081B03194208D0C8
:10CE30004546ED081D4204D14346D0085907084332
:10CE40002900420FC9007F4D1143C0004B07CA089B
:10CE50007C49C00803438D4268D012036D05120B54
:10CE60006D0D002112031800130B0A0D12051A4351
:10CE7000764B2D0513402B435B00E4075B082343EF
:10CE800019001CBC90469946A246F0BD3E001643D0
:10CE900012D05E1E002E00D000E18718874280412C
:10CEA00041444042091801250B0233D5022585E78C
:10CEB00064463300414610001D00C7E7002D00D036
:10CEC000DAE00C000443F3D05C1C00D19FE15D4C20
:10CED000A64200D12FE1DB43382B00DD66E11F2B9A
:10CEE00000DD83E120240500E41A0F00DD40D94075
:10CEF000A0404346A7405B1A441EA04198462F43DA
:10CF00003843171ABA42924143465242991A64462C
:10CF10003500CAE607223A40002A00D0F6E64B0761
:10CF2000CA084849FF083B438D4296D11900114376
:10CF300000D19EE1802109030A431203120B414DE7
:10CF40008FE71500002200238BE7002B00D0C7E0FD
:10CF50006B1C5F057F0D012F00DCF1E0394DAB420A
:10CF600000D1B9E085180A0085428941424449420E
:10CF700051180722CF076D082F4349083A401D007A
:10CF8000C2E607223049ED1A31403A40BCE63E0085
:10CF90002838864000279FE63800FEF73DFF203006
:10CFA0008EE6434613431F007A1E9741C71BB842C3
:10CFB00080414042091A78E60E003B0006431343C5
:10CFC000002D61D1002E00D0F4E0002B00D11BE138
:10CFD00064463900100039E71A4FBB427AD033005B
:10CFE000FFE630001F3DE840202B03D04021CB1A44
:10CFF0009E4037437B1E9F41072207433A40002152
:10D00000002589E7171A4346BA42B641591A7642B3
:10D010008E1B64464EE61F2B00DDADE02026474602
:10D02000F61AB740B9461700B246DF404E463E43B7
:10D0300037005646B240561EB24117434246DA40C8
:10D040008918AEE6FF070000FFFF7FFFFFFF0F809C
:10D0500020264746F61AB740B9461700B246DF40C9
:10D060004E463E4337005646B240561EB241174325
:10D070004246DA40891A99E77F4CA6425BD0802469
:10D0800024045B42214327E7002E0CD1002B00D162
:10D09000CBE0644639001000774DD7E6764FBB42AF
:10D0A00018D0330075E6002B14D04B07C008184386
:10D0B0008023C9081B03194207D0FC081C4204D175
:10D0C0007907D0080843E14621004C46420FC900C9
:10D0D0001143C000684DB9E61D0000220023C0E6E0
:10D0E000002D5BD10D00054300D1E2E65D1C00D1AF
:10D0F000B0E0614DAE421FD0DB43382B71DC1F2BFB
:10D1000000DD96E020250F00ED1AAF40B94607007C
:10D11000AA46DF404D463D432F005546A840D94022
:10D12000451EA84188440743BF1897429241514287
:10D13000414435003AE6644635004146100085E634
:10D140000B000343002D00D063E6002BF5D04346CF
:10D15000134300D17AE68718874280410722414471
:10D16000404209183A400B0200D4D5E6434B013542
:10D170001940C9E5380069E61E004746203EF740E1
:10D18000BC46202B04D04026F31A46469E4032432C
:10D19000170063467A1E97411F4302E6364DAE42A2
:10D1A000CAD080252D045B422943A6E70843411ECF
:10D1B0008841A6E6002B00D148E6871A4346B842CC
:10D1C000B641CB1A76429E1B33024BD5171A434603
:10D1D000BA429241591A5242891A072264463A4089
:10D1E00092E501430F00791E8F419DE71C000F005F
:10D1F000203CE740202B03D04024E31A9940084309
:10D20000411E884138437CE60022002425E6171A97
:10D210004346BA429241591A5242891A644635002D
:10D2200043E541461000144D10E68022002412030D
:10D2300080E61D000F00203DEF40BC46202B03D0B0
:10D240004025EB1A9940084307006346781E874142
:10D250001F4369E7871897429B4141445B42C918C5
:10D260003500A3E53B003343CED0072231003A40DE
:10D2700052E600231A00F4E5FF070000FFFF7FFFDE
:10D28000F0B55746DE464E464546E0B583460700B4
:10D290000E03480085B092461C00360B400DCD0FA2
:10D2A000002800D19DE0954B984239D08023F600AC
:10D2B0001B041E43924A7B0F334399469446030056
:10D2C0006344009300230026FF00029323031B0BFB
:10D2D00098466300E40F52465B0D019400D1B3E021
:10D2E00086498B4200D19EE04246D1008022120442
:10D2F0000A435146490F11438B46814952468C4699
:10D3000000996344CB1A0021D20000932B006340A4
:10D310009A460F2E00D905E17A4BB6009B599F46DD
:10D320005B463343994600D0B8E002230826002725
:10D3300000900293CAE7CB463A0002990195019BFF
:10D340009A46022927D0032900D180E2012944D03E
:10D350006D49009B8C4663441C00002C38DD53074C
:10D3600000D013E2D2085B46DB0109D55946674B72
:10D3700019408B468021C9008C46009B63441C00E9
:10D38000634B9C4207DC5B4664055F075B02174307
:10D390001B0B620D02E000230027584A00211B03EB
:10D3A0001C0B0B0D1B05234314055A4A3800134070
:10D3B0001C4353466400DB0764081C43210005B08E
:10D3C0003CBC90469946A246AB46F0BD0122524273
:10D3D00001231B1B382B00DCADE1002200230027BA
:10D3E000DCE75B46334399465ED0002E00D18AE1EC
:10D3F0003000FEF711FD03000B3B1C2B00DD7BE131
:10D400001D22D31A5A460100DA4008398E40130013
:10D410005F46334399468F403F4B00261B1A0093CB
:10D420000023029352E7414653460B433B499B4638
:10D430008C46009B634400935B46002B3BD1022348
:10D4400000221E43022161E7434613439B4637D027
:10D450004346002B00D162E14046FEF7DDFC0300AD
:10D460000B3B1C2B00DD53E102004146083A914082
:10D4700088461D21CB1A5146D9400B0041460B432B
:10D480009B46534693401A00009B25499C466044A6
:10D4900003008C4663440093002137E70323B14621
:10D4A00000900C26029311E7002300930133042619
:10D4B000002702930AE70323C3461E43032125E7FF
:10D4C00001331E430022012120E700239A468023D6
:10D4D00000271B03094A61E7802349461B031942C1
:10D4E00000D1E2E05946194200D0DEE00B431B03B5
:10D4F00017001B0BA246014A50E7C046FF07000079
:10D5000001FCFFFF14F50000FF030000FFFFFFFE1A
:10D51000FE070000FFFF0F800DFCFFFF01F8FFFF7B
:10D52000F3030000D94500D9CBE000D1C6E03C00B0
:10D5300048460027009B013B00935B46160E1B02EA
:10D540001E431302984633041B0C9946310C01917B
:10D55000FEF76EFB4A4642430B04210C05001943BB
:10D560008A4207D98919013D8E4203D88A4201D9DE
:10D57000851E8919881A0199FEF75AFB09048C4601
:10D580004A46210464464243090C030021438A426F
:10D5900004D98919013B8E4200D8F1E02D041D43C6
:10D5A000AB464346891A4246280C12041D0C5B46C2
:10D5B000140C22001B041B0C5A4303946B4344437A
:10D5C000029568431B19150CEB189C4203D9802463
:10D5D0006402A44660441C0C15041B042D0C201886
:10D5E0005D19814277D373D00C1AA24A7D1BAF42DA
:10D5F000BF419446009B7F426344E01B1C0086426F
:10D6000000D1DBE00199FEF713FB4A4642430B04CD
:10D61000290C070019438A4207D98919013F8E4214
:10D6200003D88A4201D9871E8919881A0199FEF701
:10D63000FFFA09044A46894629044D464243090C2B
:10D64000030029438A4207D98919013B8E4203D836
:10D650008A4201D9831E89193F04891A3A00039F1F
:10D660001A43380013041B0C584381460298150CCA
:10D670006F43434345434846000C8446DB196344EB
:10D680009F4203D9802040028446654448461F0CCF
:10D6900000041B04000C7D191818A94200D284E074
:10D6A00000D17FE001231A4357E680234A461B033B
:10D6B00013431B031B0BAA466F4A6FE6BA4200D9FD
:10D6C00035E74B46DC0758087B081C43FF0734E767
:10D6D0000024AF4289D247444745A4415B46644297
:10D6E000A4196418013BA6421ED2A0426DD800D1F5
:10D6F000B6E0241A9B4678E703005A46283B9A4036
:10D700000027914688E65846FEF786FB203072E6F1
:10D7100003005246283B9A4093460022B4E6504606
:10D72000FEF77AFB20309AE6A642E2D1B845DCD972
:10D73000341A9B4659E71F2B65DC504C0099A446D0
:10D740005C46614408008C4011008240D940501E64
:10D7500082410C4314435A46DA401300620709D051
:10D760000F222240042A05D02200141D9442894130
:10D7700049425B181A0262D50122002300270DE6F8
:10D780008A4200D80AE7831E891907E70F2313404E
:10D79000042B00D1E6E5171D9742924153429B446A
:10D7A000FA08E0E5002800D1D7E57118531EB14210
:10D7B00027D3A94215D358D01A0073E7002B00DCF9
:10D7C00004E6012300229B44CDE50223474447455C
:10D7D00089415B429C46494289190C19E344241A49
:10D7E00003E743465F0047459B41B8465B429E19AD
:10D7F000023A8919A94200D054E7404500D051E7C8
:10D80000ABE51A00F6E71F215F4649420C1BE740D3
:10D81000202B07D01A49009B8C46634418005B46B6
:10D8200083401A43501E82413A4307270023174082
:10D8300009D00F21002311401400042995D12200A2
:10D840005F075B021B0BD20817430022A6E580236B
:10D8500059461B030B431B0317001B0B064A9DE590
:10D86000BD42B2D89B460024BFE68045B9D31A001A
:10D87000C3E7C046FF030000FF0700001E040000CE
:10D880003E040000F0B54F464646D6468446C0B535
:10D890008046194E18030F034D00000B5C008246B2
:10D8A0003F0B6D0DC90F9146640DDB0F0120B54292
:10D8B0000AD0B44203D0A54201D157450CD01CBCBC
:10D8C00090469946A246F0BD66463E43F7D1AC422B
:10D8D000F5D154461443F2D10120C845EFD1994205
:10D8E00007D0002DEBD163461F433800471EB841D7
:10D8F000E5E70020E3E7C046FF070000F0B54F462C
:10D900004646D6464D00C0B50E03C90F8A462C497F
:10D910001F035C008046360B6D0D91463F0B640D76
:10D92000DB0F8D421ED08C4216D0002D1ED130430D
:10D930008446002C01D13A4323D06246002A1AD0F3
:10D940009A4529D0514602200139084001381CBCB3
:10D9500090469946A246F0BD39001143E5D0022019
:10D960004042F4E73043FAD1AC420FD0002C0FD143
:10D970003A43E7D00CE00122013B93431800013009
:10D98000E5E763460020002BE1D0DBE73A43E6D130
:10D990009A45D7D1A542D5DCA54205DBBE42D1D8F8
:10D9A00008D00020BE42D2D250460123013898430D
:10D9B0000130CCE7C845C5D80020C845F4D3C6E738
:10D9C000FF070000F0B54F464646D6464D00C0B5AD
:10D9D0000E03C90F8A462E491F035C008046360B92
:10D9E0006D0D91463F0B640DDB0F8D4218D08C42BC
:10D9F00011D0002D18D130438446002C1ED13A435B
:10DA00001CD163460020002B30D051460220013942
:10DA1000084001382AE039001143EAD0022025E00D
:10DA20003043FBD1AC4226D0002C26D13A4324D13E
:10DA30005146022001390840013817E06246002AA9
:10DA40000FD09A45E1D1A54205DBBE42DDD819D001
:10DA50000020BE420AD250460123013898430130CB
:10DA600004E00122013B9343180001301CBC9046A6
:10DA70009946A246F0BD3A43D0D19A45C5D1A542B8
:10DA8000C3DCE0E7C845C0D80020C845E3D3EDE7D4
:10DA9000FF070000F0B55746DE464E464546E0B566
:10DAA000834606000F03480087B092461D003F0BD7
:10DAB000400DCC0F002800D16FE0DE4B984238D0EB
:10DAC0008023FF001B041F43730F3B430193DA4B7A
:10DAD0000027994600239B46F60081442B036900EA
:10DAE0001B0B52469846490DED0F002900D185E0E9
:10DAF000D04B994200D173E04346DA0080231B04E7
:10DB000013435246CC48520F8446134352460020DA
:10DB10006144D20089442100694000918C46012172
:10DB200049448A460F2F00D990E0C449BF00CF591D
:10DB3000BF465B463B43019300D06AE102230827BE
:10DB4000002681469B46C9E732005846019B614644
:10DB50000091022800D175E0032800D1FEE10128E0
:10DB600000D02CE100230027002600253F032A0DCA
:10DB70003F0BB34812053A4302401B051343009A7A
:10DB80005B00D1075B080B433000190007B03CBCB9
:10DB900090469946A246AB46F0BD5B463B43019397
:10DBA00000D12FE1002F00D1A5E13800FEF734F9B4
:10DBB00003000B3B1C2B00DD96E11D22D31A5A46B5
:10DBC0000100DA405E4608398F4013008E403B4327
:10DBD00001939C4B00271B1A994600239B467DE727
:10DBE000414653460B4393498C46E144002B00D0F9
:10DBF0001AE102220220174300228CE7134300D1CE
:10DC00000DE14346002B00D181E14046FEF704F9C7
:10DC100002000B3A1C2A00DD72E10100434608397C
:10DC20008B4098461D239A1A5346D3401A00434608
:10DC3000134352468A404946081A8249894681441C
:10DC4000002068E77B4B002700268EE7140C1204A7
:10DC5000120C1100370C3604350C794328008C4621
:10DC60002E0060436044834656432100300C8046BA
:10DC70005846794340440291844506D9884680211C
:10DC800049028C46E044414602913604010C360CB0
:10DC900000048B4681191E0C1B041B0C03911900F8
:10DCA00079438C46280075436544A8465843050CC3
:10DCB00045447743A94203D9802149028C466744F1
:10DCC000290C8C4639000004000C2D042D186144E9
:10DCD000AB4405915946049101990F043F0C080C7F
:10DCE000390051434243904602008C46090C8B4652
:10DCF00062437C4344445C44A04503D980214902EB
:10DD000088464244210C884661460904090C8C4629
:10DD100039005943434370437E430F0CF6182404E3
:10DD2000BE19644442448C46B34203D980235B024B
:10DD300098464044029B61469846049B37044344FE
:10DD40009B46AB45AD416B420D0405992D0C8C46AD
:10DD50007F196744FD18A8465D462D19A542A441C8
:10DD600093466442A446C344DC448F42BF41984575
:10DD70009B4193459241A445A4415B427F421F438E
:10DD8000360C52426442BF192243BF18624638180B
:10DD90004302D20D039913436A020A43501E824183
:10DDA0006146ED0D2A434E023243D90100D4B3E05F
:10DDB0000126500832400243DE0732435B08224C02
:10DDC0005444002C62DD510709D00F201040042874
:10DDD00005D0101D9042924152429B180200D90179
:10DDE00004D580241948E400034054441848844270
:10DDF00000DD27E75E075B02D2081F0B63051643B1
:10DE00005B0DB2E6002399460133042700269B46AA
:10DE100064E60323019781460C279B465EE60122B8
:10DE200001201743002276E6032303201F434346C5
:10DE300071E6C046FF07000001FCFFFF54F500003B
:10DE4000FFFF0F800DFCFFFFFF030000FFFFFFFE41
:10DE5000FE0700000023802700933F030026434B6A
:10DE600083E6019B3200A446584670E6AC466EE657
:10DE7000802701993F0339422DD03B422BD11F43CC
:10DE80003F033F0B00951600384B6EE601252D1B16
:10DE9000382D00DD66E61F2D40DC35481C0050445F
:10DEA000160082408440EE40501E824134431443A9
:10DEB000EB40620709D00F222240042A05D022003D
:10DEC000141D9442804140421B181A023ED5012382
:10DED0000027002649E68027019B3F031F433F039D
:10DEE0003F0B0094214B40E603005A46283B9A40E2
:10DEF000002601926DE65846FDF78EFF203057E66A
:10DF000003005246283B9A401300002293E65046F5
:10DF1000FDF782FF20307BE6CA4650E71F201E0037
:10DF20004042041BE640202D03D0124C5444A34031
:10DF30001A43501E8241324307260027164009D05B
:10DF40000F200023104014000428B9D122005E07DE
:10DF50005B021F0BD2081643002306E680273F030F
:10DF60001F433F033F0B1600004BFEE5FF07000079
:10DF70001E0400003E040000F8B557464E464546D4
:10DF8000DE460C000903E0B5490A460F5F00314345
:10DF90001E03DB0F760A9B46530F3343C84E6500C2
:10DFA000C000E40FD2006D0DA24681467F0D9C4655
:10DFB0009046B74200D1B9E05B46012673409B46CC
:10DFC000EE1BA34500D183E0002E63DD002F00D0BF
:10DFD000B1E06346134300D123E1731E002B00D050
:10DFE000BAE1861A6346B04280410125C91A40420F
:10DFF000091A0B0200D447E149024B0A98464346EE
:10E00000002B00D189E14046FDF706FF0300083BE5
:10E010001F2B00DD7CE120223000D21A4146D04087
:10E02000994002009E400A439D4200DD6AE15D1B6B
:10E030006B1C1F2B00DD94E1202110003500C91A54
:10E040008E40DA408840DD40711E8E41110007226B
:10E050002843002506433240002A09D00F233340CD
:10E06000042B05D0331DB342B641764289191E00F8
:10E070000B0200D43DE26A1C914B55056D0D9A428E
:10E0800000D119E18F4AF6080A4057075202374378
:10E09000120B9BE0002E00D0C5E06E1C7605760DBD
:10E0A000012E00DC48E16746861ACB1BB042BF4117
:10E0B0007F42B8461F004346FF1A3B00B8461B028A
:10E0C00000D55FE137439AD100220024002579E092
:10E0D000002E00DCFAE0002F00D18DE0784B9D424D
:10E0E00067D0802367461B041F43BC46382E00DCE4
:10E0F00052E1634613435A1E93411E1886428041E3
:10E10000404209180B0200D4BEE06D4B01359D4220
:10E1100000D1D2E06B4A73080A4001210E401E4331
:10E120005108D30707221E43324095E71E001643CD
:10E1300000D045E740E7624B9D423AD080236746D6
:10E140001B041F43BC46382E00DDEBE01F2E00DC15
:10E150003AE133006746203BDF403B00202E05D0EC
:10E160004027BF1B6646BE40324390464646721E5D
:10E1700096413343DAE0002B00D114E263461343A7
:10E1800000D168E180234E07C008C9081B0306437D
:10E19000194208D06046C008184204D16346010005
:10E1A000D2085E071643F3009946C900720F444D2A
:10E1B00011434B46DE08424B4F073743CA089D4286
:10E1C00000D16EE012036D05120B6D0D00211203DC
:10E1D000130B0A0D12051A433B4B2D0513402B431D
:10E1E0005B00E4075B082343380019003CBC904601
:10E1F0009946A246AB46F8BD6346134311D0731E41
:10E20000002B00D007E186188642804161444042DD
:10E21000091801250B0237D502257BE73E00614630
:10E2200091463500C5E75C46002D00D0E1E00B00CB
:10E230000343F3D0731C00D1ACE1214B9F4200D1CA
:10E240003AE1F343382B00DD6FE11F2B00DD8CE159
:10E2500020250E00ED1AAE40B0460600AA46DE406C
:10E26000454635432E005546D940A8406346451ED5
:10E27000A8415B1A9C463043161AB242924163464B
:10E280005242991A3D00B4E607223240002A00D0DB
:10E29000E4E60B4BF6084F073743CA089D4200D00F
:10E2A00090E73B00134300D1A6E180231B031A43F0
:10E2B0001203120B024D89E715000022002785E7A3
:10E2C000FF070000FFFF7FFFFFFF0F80002E00D041
:10E2D000C7E06B1C5E05760D012E00DCF0E0C84D3A
:10E2E000AB4200D1B9E085180A00854289416244F9
:10E2F000494251180722CE076D082E434908324083
:10E300001D00A9E6BF49ED1A114007223240A3E6DD
:10E31000320028388240002686E63000FDF77CFD7A
:10E32000203073E6634613435A1E9341C61AB04227
:10E3300080414042091A5CE60E00674606431743D7
:10E34000002D5ED1002E00D0F3E0002F00D11EE1A1
:10E350005C46614691462CE7A94FBE427BD01E0029
:10E36000F1E610001F3DE840202B03D04021CB1ADE
:10E370009A401643731E9E410722064332400021F5
:10E38000002583E7161A6346B2428041591A40427B
:10E390000B1A98465C4632E61F2E00DDABE02027C4
:10E3A000BB1B9A4663465746BB40994613004F46EF
:10E3B000F3401F433B005746BA40571EBA41134330
:10E3C0006246F240891898E62027BB1B9A466346AE
:10E3D0005746BB40994613004F46F3401F433B004E
:10E3E0005746BA40571EBA4113436246F240891A53
:10E3F0009CE7834B9F425FD080252D0473422943C5
:10E4000020E7002E0CD1002F00D1D0E05C46614601
:10E4100091467B4DCDE67A4FBE421CD01E0065E68C
:10E42000002F18D0C0084E0706438020C9080003FB
:10E43000014208D06346DC08044204D12100DA46D8
:10E44000D2085E071643F300994601245346C900DB
:10E45000720F11431C406A4DABE61D0000220027DD
:10E46000B4E6002D59D10B00034300D1D6E6731C4E
:10E4700000D1B2E0624B9F421ED0F343382B6FDCD9
:10E480001F2B00DD97E020250E00ED1AAE40B046B0
:10E490000600AA46DE40454635432E005546A840B4
:10E4A000D940451EA8418C440643B6189642924175
:10E4B000514261443D0025E63D006146914678E6C3
:10E4C0000B000343002D00D055E6002BF5D063462A
:10E4D000134300D16DE68618864280416144404274
:10E4E000091800220B0200D4D0E6464B0135194032
:10E4F000B2E5B1465DE633006746203BDF403B00B6
:10E50000202E05D04027BF1B6646BE4032439046B2
:10E510004646721E96413343EFE5394B9F42CBD0BE
:10E5200080252D0473422943A8E70843411E8841F2
:10E53000A2E6002F00D13CE66346861ACF1AB0420D
:10E540009B415B42FB1A98461B024ED5161A634646
:10E55000B2429241591A5242891A5C4600227BE526
:10E5600001430E00711E8E419FE71D000E00203DED
:10E57000EE40B046202B04D04025EB1A99400843CA
:10E58000814648464346411E8841184374E60022AE
:10E59000002417E6161A6346B2429241591A5242B3
:10E5A000891A3D0025E561469146154D01E6802218
:10E5B0000024120379E61D000E00203DEE40B04617
:10E5C000202B04D04025EB1A9940084381464E4643
:10E5D0004346711E8E411E4367E7861896429B4153
:10E5E00061445B42C9183D008CE547463743CED0B5
:10E5F00007224146324049E600273A00E6E5C04698
:10E60000FF070000FFFF7FFF30B5144D0A034B00EA
:10E61000120B5B0DC90F0024AB4211DD104CA3425D
:10E6200010DC8024640322430E4CE41A1F2C0CDD02
:10E630000D48C31ADA4013005C42002900D11C00C7
:10E64000200030BD094BCC18FAE7094DE040AC463C
:10E6500063449A4013000343EEE7C046FE03000004
:10E660001D0400003304000013040000FFFFFF7FBF
:10E67000EDFBFFFF70B500282DD0C317C5185D4016
:10E68000C40F2800FDF7C8FB154B1B1A5B055B0D7B
:10E690000A2815DD0B38854000222D032D0B0021A3
:10E6A00010002D030A0D2D0B12052A430D4D1B05DD
:10E6B0002A4013435B00E4075B082343190070BD45
:10E6C00002002900153291400A000B21081AC540AA
:10E6D0002D032D0BE3E70024002300250022DEE7B5
:10E6E0001E040000FFFF0F8010B5041E25D0FDF7AB
:10E6F00093FB144B1B1A5B055B0D0A2812DD0B38CC
:10E70000844000222403240B0021100024030A0D5E
:10E71000240B120522430C4C1B05224013435B00C3
:10E72000590810BD02002100153291400A000B214A
:10E73000081AC4402403240BE6E700230024002227
:10E74000E2E7C0461E040000FFFF0F80A3000000A8
:10E75000FC3F0150FC3F0250FC3F03500080015041
:10E7600000800250008003502024282C383C404474
:10E77000484C0207020802010003010903040204D5
:10E7800002050305000600070008000A010000005A
:10E790000000E0FE422EE63F0000E0FE422EE6BF13
:10E7A000763C7935EF39EA3D763C7935EF39EABD8B
:10E7B000000000000000E03F000000000000E0BF9B
:10E7C00000000000000000000000000000000080C9
:10E7D00000000040FB21F93F000000002D44743E82
:10E7E000000000809846F83C0000006051CC783B67
:10E7F00000000080831BF0390000004020257A389B
:10E80000000000802282E336000000001DF369351D
:10E81000000000000000F03F000000000000F83F92
:10E82000000000000000000006D0CF43EBFD4C3E8E
:10E8300000000000000000000000004003B8E23FBC
:10E840004FBB610567ACDD3F182D4454FB21E93F08
:10E850009BF681D20B73EF3F182D4454FB21F93FF7
:10E86000E2652F227F2B7A3C075C143326A6813C7D
:10E87000BDCBF07A8807703C075C143326A6913C28
:10E88000000000000000F87F000000000000F07FA2
:10E890000000000000000000000000000000000078
:10E8A000010000000000F03F8A1EBD726654B640B1
:10E8B0004E543EF2A6EFCCC078844D13BFE9CB4056
:10E8C0004FFA050429CCB8C06C5C8AE26E569440BD
:10E8D000CC5CF6234F0B5BC0563BD76877D804401F
:10E8E000AC5913DC0D687EBFA38C9F98E6E76C3EA5
:10E8F0005610B1E5EB4731BE182D4454FB210940B9
:10E9000000000000000000000000000000002440A3
:10E91000000000000000000000000000CAF4000039
:10E92000D0F40000D6F40000DCF40000E2F40000B3
:10E93000E8F40000EEF40000F4F40000FAF4000043
:10E9400000F5000006F500000CF500000606103882
:10E950007C101010050554341C1615060611514A7A
:10E960002A2410060610242A4A5111080804423E9F
:10E9700002023E42200505007F3E1C080303403E84
:10E9800001070760584641465860040463554941F1
:10E99000020225520505080C7E0C08050510307E84
:10E9A000301006061010107C381004040404000E09
:10E9B0000505605068444005056000600060000285
:10E9C00001015F03030600060505147F147F14058B
:10E9D00005042A7F2A1005052313086462050536FD
:10E9E0004951225001010602023E410202413E0508
:10E9F000054428102844050510107C101002024020
:10EA0000300505101010101002026060030360183A
:10EA10000605053E5149453E050500427F4000057B
:10EA200005625149494605052241494936050518FF
:10EA300014127F100505274545453905053C4A490F
:10EA4000493005050171090503050536494949366F
:10EA50000505064949291E0202420002024022051C
:10EA60000508141422220505141414141405052293
:10EA7000221414080505020151090608083C023950
:10EA800045453D417E05057E0909097E05057F490D
:10EA900049493605053E4141412205057F41412254
:10EAA0001C05057F4949494105057F0909090105FB
:10EAB000053E4141513205057F0808087F030341A7
:10EAC0007F410505304040403F05057F0814224145
:10EAD00005057F4040404005057F020C027F05058B
:10EAE0007F0408107F05053E4141413E05057F0931
:10EAF00009090605053E4151215E05057F091929D1
:10EB00004605052649494932050501017F010105F0
:10EB1000053F4040403F0505071860180705057F81
:10EB20002018207F05056314081463050503047885
:10EB300004030505615149454302027F4103030671
:10EB400018600202417F050508040204080505401B
:10EB5000404040400202020404042054547804045B
:10EB60007F44443804043844444404043844447F13
:10EB70000404385454580303087C0A040418A4A459
:10EB80007C04047F0404780303447D400202847DF6
:10EB900004047C10284401017F05057C0438047CB2
:10EBA00004047C0404780404384444380404FC4419
:10EBB00044380404384444FC04047C080404050577
:10EBC00008545454200303047E4404043C40407C15
:10EBD00005050C3040300C05053C403C403C05052B
:10EBE0004464384C4404041CA0A07C030364544CCB
:10EBF0004FF300000000000055F30000000000008B
:10EC000059F30000000000005EF3000062F3000012
:10EC100066F30000000000006AF300006DF30000DE
:10EC200071F30000F3F1000076F300007CF30000C4
:10EC300080F30000F7F100000000000084F3000002
:10EC400088F300008CF300008CF3000092F30000C6
:10EC500096F30000CEF400009AF300009CF300004D
:10EC60009EF300008BF2000030F40000A0F30000DF
:10EC7000A2F30000A4F30000A7F30000A9F3000032
:10EC8000ABF30000A5F3000089F40000C3F400001A
:10EC9000C8F4000000000000ADF30000B1F3000074
:10ECA000B5F3000000000000B7F30000BFF3000060
:10ECB00060F300000000000000000000C3F300004B
:10ECC000CAF30000C7F30000CCF30000D6F3000045
:10ECD00017F4000000000000E0F30000E8F300007B
:10ECE00030F2000084F1000084F10000F1F3000034
:10ECF000F8F30000FFF3000002F40000EDF3000061
:10ED00003FF2000005F4000009F400002EF20000BC
:10ED10003BF200000FF4000014F400002AF200009F
:10ED200037F2000019F400001EF4000026F4000081
:10ED300028F40000000000000000000000000000B7
:10ED40002EF400000000000032F4000036F4000051
:10ED50003CF40000000000003FF4000042F400001A
:10ED600048F400004CF40000E9F1000050F4000009
:10ED700062F400000000000056F400005BF40000A4
:10ED800061F4000064F4000064F400006BF400001F
:10ED90006DF4000071F4000076F4000079F40000D6
:10EDA0008CF400007CF4000082F4000085F4000084
:10EDB00015F4000088F400008BF4000090F40000CB
:10EDC00093F4000098F400009DF40000000000009F
:10EDD00000000000A2F40000A7F40000ACF4000062
:10EDE000B1F40000B6F40000BBF40000C0F4000071
:10EDF000C5F4000000000000F55E0000DDA6000084
:10EE0000F5500000997D0000D950000027A60000B1
:10EE1000399B0000597D0000BD50000029640000AE
:10EE2000457A0000F97C0000A18F0000D563000046
:10EE30001D780000957C00003D900000A18E000030
:10EE40001973000085640000098900000989000029
:10EE500095580000599C00004B5900004159000092
:10EE60002359000005590000CD5800003759000013
:10EE700019590000FB5800004D7100002D59000089
:10EE80000F590000F1580000ED7000004D720000B5
:10EE9000AD720000017C0000F55E00001DAA0000BC
:10EEA000E1A400001DA6000000000000097E000093
:10EEB000A150000013A600000000000021960000F1
:10EEC0008150000009A60000E16E0000815F000093
:10EED000F98B0000FFA500007150000011530000E5
:10EEE000258A0000F5A500001D8E00001D8E000083
:10EEF00091500000914F0000396E000073500000E7
:10EF000085980000599A0000956C0000D56F0000AC
:10EF10009D970000D199000055620000596F0000D4
:10EF2000B59600003D990000396C00009563000023
:10EF3000A1AE000051A90000F55E0000B968000014
:10EF4000FD4F0000E96B000000000000A54F00002D
:10EF5000E54F0000A96B000000000000ED6100001B
:10EF6000DD690000216B00000D6700007581000065
:10EF700041690000CD6A0000934F0000D97D000078
:10EF8000E16800006D6A0000B5610000B561000035
:10EF900019620000396A000025610000954F0000E9
:10EFA0008595000061500000F15F0000BD67000022
:10EFB000DD940000515000000D6600006567000000
:10EFC00049940000415000005D650000518C000034
:10EFD000C14F00001D50000091910000ED91000014
:10EFE00049920000AD920000119300005993000077
:10EFF000A1930000F5930000FB21F93FFB2109409C
:10F000007CD91240FB2119407A6A1F407CD92240EA
:10F01000BBFD2540FB2129403A462C407A6A2F400F
:10F020005C4731407CD932409C6B3440BBFD35405D
:10F03000DB8F3740FB2139401BB43A403A463C4015
:10F040005AD83D407A6A3F404C7E40405C47414040
:10F050006C1042407CD942408CA243409C6B44409F
:10F06000AC344540BBFD4540CBC64640DB8F4740F6
:10F07000EB584840FB21494083F9A200444E6E0002
:10F08000FC291500D1572700DD34F50062DBC000F4
:10F090003C999500419043006351FE00BBDEAB00FC
:10F0A000B761C5003A6E2400D24D42004906E00027
:10F0B00009EA2E001C92D100EB1DFE0029B11C00B4
:10F0C000E83EA700F535820044BB2E009CE9840091
:10F0D000B4267000417E5F00D69139005383390019
:10F0E0009CF439008B5F840028F9BD00F81F3B00B9
:10F0F000DEFF97000F980500112FEF000A5A8B00D2
:10F100006D1F6D00CF7E360009CB2700464FB7003C
:10F110009E663F002DEA5F00BA277500E5EBC70049
:10F120003D7BF100F739070092528A00FB6BEA0041
:10F130001FB15F00085D8D00300356007BFC460068
:10F14000F0AB6B0020BCCF0036F49A00E3A91D00A1
:10F150005E619100081BE60085996500A0145F00C0
:10F160008D40680080D8FF0027734D0006063100EF
:10F17000CA561500C9A873007BE260006B8CC00002
:10F180002869290052414E20230025750025642559
:10F19000732025733F002564257320257320257374
:10F1A0000025642573202573004E414E002D494EE5
:10F1B00046002E25253025646C6C7500256C6C7519
:10F1C00000204525640025732563257300257320E1
:10F1D0002025632573002573202B257320256300CC
:10F1E000257320257320256300524E440054455357
:10F1F000543A0053544F0052434C00436865636BCC
:10F2000020466C61673A00436C65617220466C6110
:10F21000673A0053657420466C61673A0044656C38
:10F22000657465205072676D3A0049534700445336
:10F2300045005820192000454E47005343490046D9
:10F24000495800476F20546F204C424C3A004754B5
:10F250004F204C424C3A00476F20546F204C696E4F
:10F26000653A00257320005F0050726F6772616D10
:10F270002025630050726F6772616D202564005213
:10F28000756E6E696E67002E202E202E00593A0092
:10F29000583A0044697669646520627920300049F3
:10F2A0006E76616C69642074797065004E6F206CB5
:10F2B0006162656C004C6162656C2065786973748D
:10F2C00073004F7574206F66204D656D004D617839
:10F2D00020497465727320526561636865640041FA
:10F2E000626F727400680068256300660072616472
:10F2F00000677200201000205000201C2000201009
:10F3000020005069636B204C424C3A0052756E20CD
:10F310004C424C3A00475342204C424C3A00534F27
:10F320004C5645204C424C3A00494E5445475241B8
:10F330005445204C424C3A002564200050617374BF
:10F3400065207072674D656D6F72793A0D0A0045E0
:10F350006D70747900522F5300535152540047532B
:10F36000420047544F00655E5800521B0053494EFF
:10F370000031305E5800582019205900434F530087
:10F38000595E580054414E00312F5800454E5445A7
:10F3900052004545580043485300310034003700BF
:10F3A00035003800182B0033003600390050534523
:10F3B000004C424C004100434C454152201800484B
:10F3C00059500044494D004652414300434C454189
:10F3D000522052454700436F6D7020636F6E6A0084
:10F3E00072756E54696D650059202B20695820197B
:10F3F00000524553554C54004D41545249580078E1
:10F4000021001C5200792C72001C482E4D53004CD8
:10F410002E522E001C5241440050792C7800526527
:10F42000201920496D001600534F4C564500585E78
:10F43000320052544E00485950201D004C4E00528C
:10F440001A0053494E201D004C4F4700494E5400AE
:10F45000434F53201D00434C20580054414E201D63
:10F46000001725004C4153542058001400414253CA
:10F47000004D45414E001C50005346005354444536
:10F4800056001C4800434600182D001C4445470008
:10F49000463F00475241440043792C78005445537D
:10F4A000540053544F2B0053544F2D0053544F2AA4
:10F4B0000053544F2F0052434C2B0052434C2D000D
:10F4C00052434C2A0052434C2F0058201120300048
:10F4D00058203E20300058203C2030005820122078
:10F4E000300058201320300058203D20590058206B
:10F4F0001120590058203E20590058203C20590026
:10F5000058201220590058201320590058203D201F
:10F510003000000024D5000096D30000DAD30000AC
:10F520003ED30000DAD30000CAD40000DAD30000D2
:10F530003ED3000096D3000096D30000CAD400004A
:10F540003ED3000036D3000036D3000036D300008F
:10F55000D8D400004CDC00004EDB00004EDB000085
:10F560006CDE000048DB000048DB000054DE0000D9
:10F570006CDE000048DB000054DE000048DB0000C9
:10F580006CDE000062DE000062DE000062DE000071
:04F5900070DE000029
:08F59400E8C6FF7F0100000042
:10F59C000508107A4CE900004D000000583A001F95
:10F5AC002C000000E80400102000001000000000F7
:10F5BC00000000000C03001074030010DC030010AA
:10F5CC00000000000000000000000000000000002F
:10F5DC00000000000000000000000000000000001F
:10F5EC00000000000000000000000000000000000F
:10F5FC0000000000000000000000000000000000FF
:10F60C0000000000000000000000000000000000EE
:10F61C0000000000000000000000000000000000DE
:10F62C0000000000000000000000000000000000CE
:10F63C0000000000000000000000000000000000BE
:10F64C0000000000000000000000000000000000AE
:10F65C00000000000000000001000000000000009D
:10F66C000E33CDAB34126DE6ECDE05000B00000062
:10F67C00000000000000000000000000000000007E
:10F68C00000000000000000000000000000000006E
:10F69C00000000000000000000000000000000005E
:10F6AC00000000000000000000000000000000004E
:040000030000BAE15E
:00000001FF
